:020000040000FA
:1080000000590020D5800000F18000001B540100C1
:108010000000000000000000000000000000000060
:10802000000000000000000000000000F5800000DB
:108030000000000000000000F780000045FC010087
:10804000FB800000FB80000085C4010091C401009A
:108050006DC2000059020200C1080200CD080200F2
:1080600031670100396701000DE3010015E30100EC
:108070008D540100955401004102020049020200A2
:10808000510202000366010061020200690202005F
:108090007102020075C40100D73D0200EDD4010059
:1080A000898C00007DC401000931020011310200F9
:1080B0005F680100FB65010049CF0000F9B50000D1
:1080C0000348854600F09CFD004800477B8C00007B
:1080D0000059002009480A4A002100A1814200D924
:1080E00002440848084A0260084880470848004798
:1080F000FEE7FEE7FEE7FEE7FEE7FEE70000002002
:108100000000000008ED00E00080000069010200AE
:10811000C180000030B50B4601460020202201241A
:1081200009E00D46D5409D4205D31D469540491BAB
:108130002546954040191546521E002DF1DC30BDF4
:1081400070B500242546002801DA012440420029A8
:1081500001DA01254942FFF7DDFFAC4200D0404281
:10816000002C00D0494270BDF0B51FB40646002077
:1081700082B005464024019100901BE001992246FF
:108180000F46304600F036FC049A059B801A994150
:1081900010D310461946224600F01CFC361A8F41B7
:1081A0000197224601200021009F00F013FC38189F
:1081B0004D4100902046641E0028DFDC019B0098A2
:1081C0002946324607B0F0BD38B50446C0681821CC
:1081D000401E4843A16840183C214843616840184C
:1081E0003C2148432168451860690C2148432169B6
:1081F00040186921C900401A3021FFF7A1FF114A38
:1082000050434219084600921A2902DB0E495118C0
:1082100000910C21FFF794FF0C4A5043009A8018FC
:1082200000900B4806E0491E425C074B5A43009BF6
:10823000D21800920029F6DC2146684600F006FCC0
:10824000009838BD801F8607805101008033E1010E
:1082500048C3020003460B439B0703D009E008C94B
:10826000121F08C0042AFAD203E00B780370401CE6
:10827000491C521EF9D27047D2B201E00270401C74
:10828000491EFBD270470022F6E710B513460A4696
:1082900004461946FFF7F0FF204610BD421E5378F2
:1082A000521C002BFBD10B781370491C521C002B65
:1082B000F9D17047421C0178401C0029FBD1801A7B
:1082C000704703460A780270401C491C002AF9D105
:1082D000184670470321001D401E037812021A43FE
:1082E000491EF9D510467047034610B508330722DA
:1082F000040E090221435B1E1C7800022043521E1B
:10830000F6D510BD034603220870000A491C521E10
:10831000FAD51846704770B504460D46072310700D
:108320000E06000A3043090A521C5B1EF7D5204690
:10833000294670BDF8B502464A40D40F42004B00B2
:1083400052085B089A4202D20246084611464A0089
:1083500023D0C30D4A00DDB2120EAD1A202D35DA3E
:1083600049020126490AF6058A19002C00D052421A
:1083700020214F1B1146B9402A411018C20D9A42C4
:1083800021D0002C17D0012D08DCDA05801AD20F7D
:108390008019D207DBB200F09BFBF8BDDA05801A2A
:1083A000012340001B06C01880185A428018CA0FCB
:1083B0001043490007E04908C2071143DA05801A53
:1083C00080194008801800F07BFBF8BD6100012295
:1083D000511A001BF7E70122D2075140AAE70122F8
:1083E000D2075040A6E7024670B54A40D30FDB07DC
:1083F00040002DD04A002AD0010E140E00021202B5
:108400000919400A520A8418E50104465443000A37
:10841000120A2E045043A4194219200CC543AA186D
:10842000120C0125AD03521C521912047F39240489
:1084300000D0521C104301D44000491EC2B20C06A9
:10844000C0092018401C4008802A02D003E0002008
:1084500070BD40084000002900DA0020184370BDBC
:1084600070B502464A40D50F40004A00ED0740086B
:108470005208002814D0002A12D0C40DD30D410296
:108480000120C0055202490A520AE41A09181218BA
:108490007D34914201D3641C00E04900002C01DAD4
:1084A000002070BD0023914201D3891A0343400884
:1084B00049000028F7D100290AD0914202D10121B8
:1084C000C90705E0914201D2012101E00121C94320
:1084D000E005C018401900F0F3FA70BDF0B507468A
:1084E0000846584087B0C00F049048000E46590017
:1084F00040084908BC1A884105D2384631461E4614
:1085000017460B4602465800400810434CD0300D29
:10851000039040055900400D490D0590401A029006
:10852000402872DA18030121000B09050843019065
:1085300004980092002805D00199524200208841F9
:1085400000920190029840210A1A0199009800F0C7
:1085500041FA05460C466B4607CB00F05CFAC019A1
:108560007141039A0E0D0023D71756401A467A40E0
:10857000164344D0049A002A2DD0029A012A039A65
:1085800015DC1205C01A914101263605001C714107
:10859000D20F059ED2070093019202962A462346E7
:1085A00000F0DCFA07B0F0BD38463146FAE71605B0
:1085B000224A0F46B218C01AB74101210905001C12
:1085C0004F4100187F41114618187941E20F1043BE
:1085D0006D19644113E0E2076D0815436408C20792
:1085E0001443039A01261205C01A91413605001C56
:1085F0007141CE07400830434908C01851412A460E
:10860000234600F09EFACDE7FFE7049801224000E0
:10861000C117121A00238B4104983146C417381A27
:10862000A141EEE730B40124E407634030BC55E7D4
:1086300030B40124E407614030BC4FE70000E0FFA4
:10864000F0B51FB488B00B990998002448400999E7
:10865000C00F490049080991C0070B9900904900D3
:1086600049080B9109990898A64608431CD00B9914
:108670000A98084318D0099801244000420D480088
:10868000410D099824050003000B204309900B9825
:108690000003000B20430B9050181C494018002287
:1086A00001901446104605E0002001460DB0F0BDD3
:1086B000032801DA034600E003239C46C11A0AAEF0
:1086C0000AE05F0008ADED5B4F00F75B7D430027DC
:1086D000AA187C41491C5B1E6145F2DD410004ABD8
:1086E0005A522104120C0A43240C401C0828DFDBD8
:1086F000019802900099704601910090059B049AA0
:108700000799069800F02AFAD0E700000DFCFFFF59
:10871000F0B50C465C4085B0E40FE40703944C00D0
:1087200000266408590094464908024602962243EE
:1087300021D062460A431ED06200570D4A000E0344
:108740002303550D012402462C492405781B1B0BDD
:10875000360B401823432643614600901C46501AAE
:10876000B44103D30098401C009002E09218009896
:108770005B41002803DA0020014605B0F0BD00206F
:10878000012109050746864611E064461D46141B73
:10879000B54106D36546521BB341744607430C43AB
:1087A000A646CD0740084908284392185B41054674
:1087B0000D43EAD11046184313D060461946504085
:1087C0007140084306D06046101AB34106D2012218
:1087D000002306E000220123DB0702E00122D2434E
:1087E0005310009874460105381C6141029C039D9A
:1087F0000019694100F0A5F9BFE70000FD03000082
:10880000C217C10F504010B54018CA079623002167
:1088100000F05EF910BD10B500229623114600F05D
:1088200057F910BD0EB5C217C10F5040CA07401806
:108830000021054B0293019200910A460B4600F07D
:108840008DF903B000BD0000330400000EB50549EA
:108850000291002100910A460B46019100F07EF939
:1088600003B000BD33040000410040020122400A71
:10887000D205090E80187F2901DA00207047962959
:1088800003DC9622511AC8407047963988407047D9
:1088900041000A0E40020121400AC90510B54018E6
:1088A0007F2A02DA0020014610BD0021962A03DC4F
:1088B00096239A1AD04010BD963A00F08BF810BD5E
:1088C0004A0009030123090B1B051943094B10B585
:1088D000520D9A4201DA002010BD064B34339A4201
:1088E00003DC9A1A00F086F810BD0349511888403D
:1088F00010BD0000FF030000CDFBFFFFC20FD20739
:10890000400040080BD0C10D0723DB01C91840020D
:108910000905400A1143C20840071143704700206F
:108920000146704710B5002904DB0124E4074042EA
:108930008C412146002B04DB1C460123DB075242FD
:10894000A3418B4200D1824210BD000010B5002926
:1089500004DB0124E40740428C412146002B04DB68
:108960001C460123DB075242A341994200D19042A9
:1089700010BD0000CB0FDB07490010B549080246C7
:108980000A4307D00A0D07240903E401090B121B4F
:10899000002A01DC002010BDC900440F0C43C100B7
:1089A000E018D205801800F08BF810BD0122D20724
:1089B000002800DB101A002900DB511A81427047A1
:1089C0000122D207002800DB101A002900DB511A0F
:1089D0008842704710B5202A04DB0146203A9140B6
:1089E000002010BD914020239C1A0346E340194308
:1089F000904010BD10B5202A04DB0846203AD04034
:108A0000002110BD0B46D340D0402024A21A914033
:108A10000843194610BD10B5202A06DBCB170846BF
:108A2000203A1041C1170B4306E00B461341D040DA
:108A30002024A21A91400843194610BD10B50249DE
:108A400000F004F810BD0000D048002070B50C46BE
:108A500000683C21FFF75EFB21603C21FFF75AFBD9
:108A600061601821FFF756FB0546A1600721001D34
:108A7000FFF750FBA1610F48A90008180E49FFF746
:108A800049FB0246443288086261E0613B2802D318
:108A9000910700D0401C0021084B0A462161995CD7
:108AA000814203D8401A521C2261F8E7401CE06062
:108AB000204670BD6C0B0000B505000054C30200D9
:108AC000002904DA401C490001D1400840007047E9
:108AD00070B40024050C05D11024000402D1002933
:108AE00021D01124050E01D100020834050F01D157
:108AF0000001241D850F01D18000A41C002801DB8A
:108B00004000641C002908D020252E1B0D46F5408E
:108B1000A14000D001212943084301061B1B000A84
:108B2000DB1D02D5002070BC7047DB0518188018CB
:108B30000029F8DA401C4900F5D170BC400840001B
:108B4000704710B5002B08DA0024401C61419218D0
:108B50005B411A4301D14008400010BDF0B51FB47D
:108B600082B005460C0003D008461BF0F7FC02E07B
:108B70001BF0F4FC20300246009021462846FFF707
:108B800029FF049B059A04460F46184311430843E6
:108B900014D0184610431BD0009840210A1A1846DA
:108BA0000599FFF727FF05460E46009A0599049898
:108BB000FFF710FF084305D0012004E020463946A6
:108BC00007B0F0BD0020C11705430E432C433743C7
:108BD00000990E986305401A7905E40A00220C43B7
:108BE000FD0A0A3002D500200146E9E70105101907
:108BF00069410C9C0D9D00196941FFF7A2FFDFE759
:108C0000064C0125064E05E0E36807CC2B430C3CDF
:108C100098471034B442F7D3FFF756FA7CC50200E8
:108C20009CC5020070B58C180578401C6B075B0F63
:108C300001D10378401C2A1106D10278401C03E0C0
:108C400006780E70401C491C5B1EF9D12B0705D419
:108C50000023521E0DD40B70491CFAE70378401C08
:108C6000CB1A921C03E01D780D70491C5B1C521E30
:108C7000F9D5A142D8D3002070BD10B517F074FA11
:108C800021F0B4FA002010BD10B5C046C046C04661
:108C9000C04610BDF7B58AB00D460595059D28461E
:108CA000E917090F09180905090E0491002728E0A2
:108CB000002407E0380101190A98405C694608550C
:108CC000601CC4B2102CF5DB002605E00C98805D1A
:108CD00006A98855701CC6B2102EF7DB012206A922
:108CE00068461BF069FD002407E06846015D380115
:108CF00002190A988154601CC4B2102CF5DB781C50
:108D0000C7B204988742D3DB0DB0F0BDFFB58DB07C
:108D100014460D98002802D0012854D154E025466D
:108D20002C462046E917090F09180911491C0905A5
:108D30000E0C301BC0B2089008980790E8B206905D
:108D400007E0069A0E99079888540698401CC0B20E
:108D500006900698B042F4DB002005902CE0002736
:108D600008E005980001C1190E98405C01A9C8559A
:108D7000781CC7B2102FF4DB002705E01098C05D07
:108D800009A9C855781CC7B2102FF7DB002209A922
:108D900001A81BF011FD002708E001A8C15D05989E
:108DA0000001C2190E988154781CC7B2102FF4DB51
:108DB0000598401CC0B20590F117090F89190A11D6
:108DC00005998A42CBDC53E025462C462046E9171C
:108DD000090F09180911491C09050E0C301BC0B2F6
:108DE000089008980790069507E0069A0E9907984C
:108DF00088540698401C80B206900698B042F4DB76
:108E0000002005902CE0002708E005980001C1191A
:108E10000E98405C01A9C855781CC7B2102FF4DB2E
:108E2000002705E01098C05D09A9C855781CC7B295
:108E3000102FF7DB002209A901A81BF0BDFC0027B9
:108E400008E001A8C15D05980001C2190E9881547F
:108E5000781CC7B2102FF4DB0598401CC0B20590F7
:108E6000F117090F89190A1105998A42CBDC00BF55
:108E700000BF11B0F0BD0000FEB51746002400256C
:108E8000002600200290019000BF27E0A0002549A5
:108E9000085800280DD0A00008584B21C90088426E
:108EA00007D2A0001F490958029808180290701CA8
:108EB000C6B2A0001C49085800280DD0A0000858D0
:108EC0004B21C900884207D2A000174909580198D0
:108ED00008180190681CC5B2601CC4B2BC42D5DB46
:108EE000002D08D029460198FFF714F90F4900908A
:108EF000FFF708FA03E00D490020FFF703FA002E00
:108F000009D031460298FFF705F90849091F00907A
:108F1000FFF7F8F904E00549091F0020FFF7F2F90F
:108F2000FEBD0000741A00208C1A0020B01A002028
:108F300010B50446454800780A3803001BF025FBAD
:108F40000B070D17212B353F49535F697F002B2CF1
:108F500002D10B203D49087075E0432C03D10C2051
:108F60003A49087002E00A20384908706BE0452C45
:108F700003D10D203549087002E00A2033490870FA
:108F800061E0522C03D10E203049087002E00A2023
:108F90002E49087057E0452C03D10F202B4908704B
:108FA00002E00A20294908704DE0472C03D1102027
:108FB0002649087002E00A202449087043E03A2C50
:108FC00003D112202149087002E00A201F490870CD
:108FD00039E0202C03D112201C49087002E00A203D
:108FE0001A4908702FE0302C05DB332C03DC1320EA
:108FF0001649087002E00A201449087023E02C2C5E
:1090000003D114201149087002E00A200F490870AA
:1090100019E020463038C1B2012021F0F9FF312C8F
:1090200001D0352C07D10320C04309490875002021
:109030000649087002E00A200449087003E00A208B
:109040000249087000BF00BF10BD000030070020BB
:109050003334002010B50446384800780A3803003D
:109060001BF093FA09060C16202A343E485266007B
:109070002B2C02D10B20314908705DE0432C03D129
:109080000C202E49087002E00A202C49087053E099
:10909000472C03D10D202949087002E00A202749F6
:1090A000087049E0412C03D10E202449087002E0E9
:1090B0000A20224908703FE0542C03D10F201F4999
:1090C000087002E00A201D49087035E0542C03D1D5
:1090D00010201A49087002E00A20184908702BE095
:1090E0003A2C03D112201549087002E00A201349D6
:1090F000087021E0202C03D112201049087002E0F2
:109100000A200E49087017E020463038C1B202200C
:1091100021F07EFF312C07D10320C0430849087598
:1091200000200649087002E00A200449087003E0A4
:109130000A200249087000BF00BF10BD30070020A0
:1091400033340020224909780A2902D00B2933D16F
:1091500008E0492805D10B211D4A117000211D4A44
:10916000117033E052281CD04B280CD0302822DB61
:10917000392820DC17490A780978491C154B1970E1
:109180001549885417E00021124A11700022124933
:10919000CA730A210E4A11700321C9430F4A11757F
:1091A00009E000210B4A11700A21094A11700221BD
:1091B000C9430A4A117509E00A21054A11700021C4
:1091C000044A1170C91E054A117500BF00BF7047DF
:1091D000300700206E070020A02900203334002033
:1091E00070B50446B24800780A3803001BF0CDF988
:1091F0002C171D27313B455B6597A1ABB5BBC9E07B
:10920000F8FEEDECEBEAEAEAEAEAEAEAEAEAEAEA96
:10921000EAEAEAEAEAEAEAEAEA6F79838DEA2B2CDB
:1092200002D10B20A24908703FE14D2C03D10C2044
:109230009F49087002E00A209D49087035E1492CD9
:1092400003D10D209A49087002E00A20984908705D
:109250002BE1502C03D10E209549087002E00A2022
:109260009349087021E14C2C03D10F2090490870DC
:1092700002E00A208E49087017E1572C06D1002120
:109280008C48817210208A4908700BE0452C06D169
:1092900001218848817232208549087002E00A2045
:1092A0008349087001E1522C03D1112080490870D4
:1092B00002E00A207E490870F7E0492C03D1122011
:1092C0007B49087002E00A2079490870EDE0582CCB
:1092D00003D133207649087002E00A2074490870EF
:1092E000E3E0452C03D134207149087002E00A20E4
:1092F00071490870D9E0432C03D135206C490870BE
:1093000002E00A206A490870CFE0552C03D11220F0
:109310006749087002E00A2065490870C5E0542CCE
:1093200003D113206249087002E00A2060490870E6
:10933000BBE0452C03D114205D49087002E00A20EF
:109340005B490870B1E03A2C03D1152058490870E8
:1093500002E00A2056490870A7E0302C02D11620FE
:1093600053490870A1E02C2C0AD1172050490870ED
:109370000020504988710A214E48001FFEF783FFE4
:1093800093E02C2C10D0302C11DB392C0FDC494809
:10939000807909280BDA474881798079401C454A51
:1093A0009071101F445402E01820414908707CE07D
:1093B0002C2C14D13F48807A002809D119203C492F
:1093C00008700CE070E027E01CE015E00EE007E01C
:1093D0003848807A012802D11A203549087064E0A3
:1093E0002C2C02D11A20324908705EE02C2C02D1BC
:1093F0001B202F49087058E02C2C02D11C202C492E
:10940000087052E02C2C06D11D202949087000213B
:109410002A488172C17248E02C2C3BD00D2C39D0E7
:109420002649C87A897A00020843012189028842C4
:1094300028DA20480838FEF74DFF451C1D49083939
:109440002846FEF75FFF302C01DB392C07DD412C6D
:1094500001DB462C03DD612C25DB662C23DC174861
:10946000C17A807A09020143144AD07A927A0002C2
:109470001043401C82B211488272120AC2720C3030
:10948000445410E000210D488172C1720A2008493D
:10949000087008E000200749487201202039C8758B
:1094A0000A200349087000E000BF00BF70BD000043
:1094B000830700205334002030070020332E002083
:1094C00000B53D4909780A390B001BF05EF8090622
:1094D000101A242E384053606E002B2803D10B2124
:1094E000354A117002E00A21334A117061E04328C5
:1094F00003D10C21304A117002E00A212E4A11706A
:1095000057E0532803D10D212B4A117002E00A21A4
:10951000294A11704DE0512803D10E21264A1170BD
:1095200002E00A21244A117043E03A2803D10F21B6
:10953000214A117002E00A211F4A117039E00146E8
:1095400030391E4A117010211B4A117031E02C284D
:1095500003D11121184A11700BE0184909780A2229
:1095600051430246303A8918144A11701121124AA7
:1095700011701EE04F2809D112210F4A11700F49B6
:1095800009781F2902DD00210C4A117011E04B28D7
:1095900007D10321C9430A4A11750A21064A1170ED
:1095A00002E00A21044A117003E00A21024A117004
:1095B00000BF00BF00BD00003007002036070020BC
:1095C0003334002070B50446D44800780A380300CC
:1095D0001AF0DBFF0C070D17212B35426384A4C45E
:1095E000E4F72B2C02D10B20CC49087094E1432CDA
:1095F00003D10C20C949087002E00A20C74908704D
:109600008AE1432C03D10D20C449087002E00A20EE
:10961000C249087080E14C2C03D10E20BF4908706C
:1096200002E00A20BD49087076E14B2C03D10F20DF
:10963000BA49087002E00A20B84908706CE13A2C77
:1096400006D11020B54908700020B549087002E025
:109650000A20B24908705FE12F2C10D0302C1BDBA0
:10966000392C19DCAE4800780A214843AC4908700F
:109670002046303809784018A94908700CE0A849FC
:10968000097808466430A749FEF73CFE0020A4494B
:1096900008701120A14908703EE12F2C10D0302C09
:1096A0001BDB392C19DC9E4800780A2148439C4971
:1096B00008702046303809784018994908700CE045
:1096C00097490978481E9749091FFEF71BFE00209D
:1096D000934908701220914908701DE12C2C10D07C
:1096E000302C1ADB392C18DC8D4800780A214843CD
:1096F0008B4908702046303809784018884908702E
:109700000BE08849083986480078FEF7FBFD002009
:1097100083490870132081490870FDE03A2C10D06D
:10972000302C1ADB392C18DC7D4800780A2148439C
:109730007B4908702046303809784018784908700D
:109740000BE078490C3976480078FEF7DBFD002005
:1097500073490870142071490870DDE03A2C10D06C
:10976000302C1ADB392C18DC6D4800780A2148436C
:109770006B490870204630380978401868490870ED
:109780000BE06849103966480078FEF7BBFD002001
:1097900063490870152061490870BDE02B2C11D079
:1097A000302C0DDB392C0BDC5D4800780A21484356
:1097B0005B490870204630380978401858490870CD
:1097C000A5E0A5E05749143955480078FEF79AFD01
:1097D0005448FEF77FFD0546643D52492846FEF792
:1097E00091FD5048001FFEF775FD451C4D49091FAE
:1097F0002846FEF787FD4B481438FEF76BFD0546FB
:109800000A21FEF79DFC060146481438FEF762FD6A
:1098100005460A21FEF794FC0E4343498E714148E8
:109820001038FEF757FD05460A21FEF789FC0601B0
:109830003C481038FEF74EFD05460A21FEF780FC35
:109840000E4339494E7137480C38FEF743FD054643
:109850000A21FEF775FC060132480C38FEF73AFD86
:1098600005460A21FEF76CFC0E432F490E712D4868
:109870000838FEF72FFD05460A21FEF761FC0601B8
:1098800028480838FEF726FD05460A21FEF758FC51
:109890000E4325498E702348001FFEF71BFD054629
:1098A0000A21FEF74DFC06011E48001FFEF712FDBF
:1098B00005460A21FEF744FC0E431B494E70194829
:1098C000FEF708FD05460A21FEF73AFC0601154899
:1098D000FEF700FD05460A21FEF732FC0E43124951
:1098E0000E7008460078232807DB084614F0CFFBEB
:1098F000E121C901012014F02DF800200849087069
:109900000A20064908700320C0430849087503E08F
:109910000A200249087000BF00BF70BD7707002011
:1099200078070020B134002079070020333400206C
:10993000294909780A2906D00B290ED00C2916D0FE
:109940000D2943D11CE0492803D10B21224A117073
:1099500002E00A21204A11703CE0442803D10C2186
:109960001D4A117002E00B211B4A117032E03A28A7
:1099700005D10021194A11700D21174A117029E0F3
:1099800052281CD04B2810D0302801DB392803DDA9
:1099900041281ADB462818DC10490A780978491C46
:1099A0000E4B19700E4988540FE000210B4A1170BC
:1099B00000220B490A75111F0A4A117505E00021A2
:1099C000064A1170C91E074A117503E00A21024AAE
:1099D000117000BF00BF70473007002080070020D3
:1099E000B02900203334002000B5344909780A3901
:1099F0000B001AF0CAFD07050F19232D37415D0032
:109A00002B2803D10B212D4A117002E00A212B4A89
:109A1000117051E0432803D10C21284A117002E053
:109A20000A21264A117047E0472803D10D21234A15
:109A3000117002E00A21214A11703DE0532803D140
:109A40000E211E4A117002E00A211C4A117033E0F7
:109A50004E2803D10F21194A117002E00A21174A3A
:109A6000117029E03A2803D11021144A117002E044
:109A70000A21124A11701FE04B280CD0302816DB47
:109A8000392814DC0E490A780978491C0C4B1970E6
:109A90000C4988540BE00021094A11700A21074A39
:109AA000117000220749CA73111F074A117503E09C
:109AB0000A21024A117000BF00BF00BD300700201C
:109AC00076070020902900203334002000B53D495E
:109AD00009780A390B001AF058FD0A06101A242ECC
:109AE000384248525C6E452803D10B21354A11702B
:109AF00002E00A21334A117061E0562803D10C219B
:109B0000304A117002E00A212E4A117057E04528B0
:109B100003D10D212B4A117002E00A21294A11704C
:109B20004DE04E2803D10E21264A117002E00A2191
:109B3000244A117043E0542803D10F21214A1170A7
:109B400002E00A211F4A117039E03A2803D110219E
:109B50001C4A117002E00A211A4A11702FE03028C5
:109B600002D11121174A117029E02C2803D11221AA
:109B7000144A117002E00A21124A11701FE03128C4
:109B800003D113210F4A117002E00A210D4A11700E
:109B900015E0352807D10321C9430B4A11750A2165
:109BA000084A117006E00221C943074A11750A21CB
:109BB000044A117003E00A21024A117000BF00BF7D
:109BC00000BD0000300700203334002010B50446EB
:109BD000314800780A2804D00B280FD00C2855D122
:109BE0002DE02C2C06D10B202B49087000202B498E
:109BF000088002E00A20284908704BE02C2C1AD07B
:109C0000302C1BDB392C19DC244800880A214843FE
:109C10002249088020463038098840181F490880AA
:109C2000084600881A2809D10C201B49087000201A
:109C30001A49088002E00A20174908702AE00D2C12
:109C400020D0302C21DB392C1FDC144800880A215D
:109C500048431249088020463038098840180F4987
:109C600008801FF031FE0D49098888420DD123205C
:109C700005F094F80320C043094908750A200649F5
:109C8000087002E00A200449087003E00A20024933
:109C9000087000BF00BF10BD3007002084070020FF
:109CA0003334002000B5344909780A390B001AF022
:109CB0006CFC0906101A242E3842485260004528D0
:109CC00003D10B212C4A117002E00A212A4A11709B
:109CD00050E0562803D10C21274A117002E00A21D6
:109CE000254A117046E0452803D10D21224A117002
:109CF00002E00A21204A11703CE04E2803D10E21D7
:109D00001D4A117002E00A211B4A117032E05428EA
:109D100003D10F21184A117002E00A21164A11706E
:109D200028E03A2803D11021134A117002E00A21D9
:109D3000114A11701EE0302802D111210E4A117013
:109D400018E02C2803D112210B4A117002E00A21DD
:109D5000094A11700EE0362807D10321C943074A8A
:109D600011750021044A117002E00A21024A1170A3
:109D700000E000BF00BF00BD3007002033340020EA
:109D800010B56E4909780A390B001AF0FEFB080578
:109D90000B151F29333D9CD12B2802D10B21674A7B
:109DA0001170C9E04E2803D10C21644A117002E001
:109DB0000A21624A1170BFE04E2803D10D215F4A8B
:109DC000117002E00A215D4A1170B5E04D2803D1FF
:109DD0000E215A4A117002E00A21584A1170ABE074
:109DE000492803D10F21554A117002E00A21534A34
:109DF0001170A1E03A2803D11021504A117002E0FD
:109E00000A214E4A117097E02C284CD14C49097810
:109E1000042914D14B4909787D22D2005143494A83
:109E2000527864235A438A18464989780A23594349
:109E30005118444AD2788918434A118028E0404991
:109E4000097803290ED13F490978642251433D4ADC
:109E500052780A235A4389183A4A927889183A4A1A
:109E6000118015E036490978022909D13549097868
:109E70000A225143334A52788918334A118007E045
:109E80002F490978012903D12E4909782E4A1180DA
:109E900000212B4A117000222C498A72CA721121AA
:109EA000264A11700EE030280CDB39280ADC014606
:109EB0003039CAB222490B780978491C204C2170EC
:109EC0002049CA5438E0214AD17A927A09021143D2
:109ED00001229202914227DC1C4AD17A937A0A022B
:109EE0001A431A4BD97A9B7A09021943491C8BB23F
:109EF00016498B721B0ACB720C318854134AD17AE3
:109F0000927A09021143104A12885200914201DAF2
:109F10000D280CD100210E4A51720121203A917571
:109F20000A21064A117002E00A21044A117003E076
:109F30000A21024A117000BF00BF10BD3107002086
:109F40006F0700207207002070070020332E0020CA
:109F50005334002000B5214909780A390B001AF062
:109F600014FB07050B11171D23293600542802D1B5
:109F70000B211A4A11702EE0492802D10C21174AF0
:109F8000117028E04E2802D10D21144A117022E0F0
:109F9000442802D10E21114A11701CE03A2802D146
:109FA00010210E4A117016E0202802D110210B4A10
:109FB000117010E0332806D10321C943084A1175F6
:109FC0000121084A11700A21044A117003E00A2194
:109FD000024A117000BF00BF00BD000067070020EB
:109FE000333400206507002010B50446304800785F
:109FF0000A3803001AF0C9FA07050F19232D374153
:10A000005600462C03D10B202949087002E00A2093
:10A01000274908704AE0412C03D10C2024490870DC
:10A0200002E00A202249087040E0432C03D10D20B1
:10A030001F49087002E00A201D49087036E0452CCF
:10A0400003D10E201A49087002E00A20184908704E
:10A050002CE02C2C03D10F201549087002E00A20B7
:10A060001349087022E0312C03D1102010490870E8
:10A0700002E00A200E49087018E0302C0AD1232093
:10A0800004F08CFE0320C0430A4908750A200849E1
:10A09000087006E00220C043064908750A200449FA
:10A0A000087003E00A200249087000BF00BF10BD1D
:10A0B0003007002033340020234909780A2906D0CC
:10A0C0000B290AD00C2915D00D2939D130E00D28E3
:10A0D00002D10B211C4A117033E00A2806D130212D
:10A0E0001A4A11700C21184A117002E00A21164A0E
:10A0F000117026E00D2803D10D21134A117016E0CE
:10A1000030280BDB392809DC104908700321C943CA
:10A110000F4A11750A210C4A117008E0452806D132
:10A120000221C9430A4A11750A21074A117008E041
:10A130000222D24306490A750A21034A117000E03F
:10A1400000BF00BF704700003007002068070020F4
:10A150003334002010B5F84909780A390B001AF099
:10A1600014FA120A15F4FAEDECEBEAE98D939DACC2
:10A17000E8E7E6E5E4143A2807D10021EF4A117038
:10A18000EF4A11700B21EC4A11703FE22D285DD08F
:10A19000302801DB392859DDE8490978012904D143
:10A1A000E7494978E74A11803AE0E4490978022909
:10A1B00009D1E34949780A225143E14A9278891842
:10A1C000E04A11802CE0DD49097803290FD1DC49F0
:10A1D000497864225143DA4A92780A235A4389180B
:10A1E000D74AD278891809B2D64A118018E0D349E3
:10A1F0000978042914D1D24949787D22D2005143EB
:10A20000CF4A927864235A438A18CD49C9780A23E1
:10A2100059435118CA4A1279891809B2C94A11809A
:10A22000C7490978012905D1C6490988494209B2B7
:10A23000C44A1180C3490988002903D10A21BE4AB2
:10A2400011701AE01321BC4A117016E02D2803D1B9
:10A250000121BB4A117010E0B849097804290CDAD1
:10A2600001463039CAB2B5490978491CB44B5A5431
:10A27000B2490978491CB14A1170C7E1492802D195
:10A280001421AD4A1170C1E1442803D11521AA4A15
:10A29000117002E00021A84A1170B7E13A2808D1F4
:10A2A0000021A64A1170A84A11701621A24A117005
:10A2B00002E00021A04A1170A8E12D2820D030280A
:10A2C00001DB39281CDD00210022A04B1A6000BFF1
:10A2D0000EE09E4A12680A235A439C4B1A609A4B1E
:10A2E0004A1C9A5C994B1B68D218984B1A60491CFF
:10A2F000924A12789142ECDB0C228F4B1A7023E0C9
:10A300002D2803D10121904A11701DE08B49097855
:10A310000A2916DA89490978491C8B4A5054874919
:10A320000978491C854A11700EE02CE11CE115E109
:10A33000CCE0C0E04DE041E030E020E015E00AE094
:10A3400003E000217C4A117060E1452802D10D2113
:10A35000794A11705AE1432803D10E21764A1170CF
:10A3600002E00C21744A117050E14C2803D10F21F6
:10A37000714A117002E00A216F4A117046E13A28D1
:10A3800008D100216D4A11706D4A117010216A4A7E
:10A39000117002E00A21684A117037E1302809DBA8
:10A3A000392807DC01463039694A11801121624A97
:10A3B000117002E01121604A117027E13A2807D19B
:10A3C00000215E4A11705E4A117012215A4A1170C2
:10A3D0001CE12D2803D10121594A11706AE030286F
:10A3E00017DB392815DC5549097804290DDA0146AF
:10A3F0003039CAB251490978491C514B5A544F4916
:10A400000978491C4D4A117054E00A214A4A1170DA
:10A4100050E04A490978012904D1494949784D4A0F
:10A4200011803AE045490978022909D1444949781F
:10A430000A225143424A92788918464A11802CE0F8
:10A440003E49097803290FD13D4949786422514397
:10A450003B4A92780A235A438918394AD278891894
:10A4600009B23C4A118018E034490978042914D112
:10A47000334949787D22D2005143314A927864238E
:10A480005A438A182E49C9780A23594351182C4A2D
:10A490001279891809B22F4A1180294909780129AE
:10A4A00005D12C490988494209B22A4A118017214D
:10A4B000214A1170AAE03A2807D100211F4A1170E1
:10A4C0001F4A117018211C4A11709FE02D281ED0C0
:10A4D000302801DB39281ADD002100221E4B1A80AA
:10A4E00000BF0CE01C4A12880A235A431A4B1A80F8
:10A4F000134A525C1B88D218174B1A80491C0F4A0A
:10A5000012789142EEDB19220B4B1A7013E00B49C3
:10A5100009780A290CDA01463039CAB20849074BD2
:10A520001B78CA5405490978491C044A117002E095
:10A530000021014A117069E030070020390700202E
:10A54000683400204E070020D43400203C0700204F
:10A55000580700205407002044070020492802D152
:10A560001A212B4A117051E03A2808D10021294ABA
:10A570001170294A11701B21254A117002E0002137
:10A58000234A117042E02D2824D0302801DB3928DD
:10A5900020DD00210022214B1A8000BF0EE01F4A5F
:10A5A00012880A235A431D4B1A801B4B4A1C9A5C83
:10A5B0001A4B1B88D218194B1A80491C154A12785D
:10A5C0009142ECDB0322D243154B1A750022104B4B
:10A5D0001A701AE02D2803D101210F4A117014E0DE
:10A5E0000C49097803290DDA01463039CAB2094904
:10A5F0000978491C084B5A5406490978491C054AF0
:10A60000117002E00021024A117000BF00BF10BDAE
:10A610003007002039070020683400204C07002054
:10A62000333400202A4909780A2906D00B290AD098
:10A630000C291ED00D2945D125E04F2802D10B2130
:10A64000234A117042E04B2806D10121214A1170A2
:10A650000C211F4A11700BE0522806D100211D4A1F
:10A6600011700C211A4A117002E00A21184A117067
:10A670002CE00D2803D10D21154A117002E00A21AA
:10A68000134A117022E00A2818D1124909780029CA
:10A6900004D00321C943104A117503E00221C943C4
:10A6A0000D4A11750D49097A0B2903D10A21084A6F
:10A6B000117006E00021064A117002E00A21044AE6
:10A6C000117003E00A21024A117000BF00BF7047F9
:10A6D000300700206D07002033340020332E002087
:10A6E00000B5224909780A390B0019F04EFF080518
:10A6F0000B11171D23292F392B2802D10B211B4A9F
:10A70000117031E0512802D10C21184A11702BE050
:10A71000492802D10D21154A117025E04F2802D198
:10A720000E21124A11701FE0502802D10F210F4A4A
:10A73000117019E0452802D110210C4A117013E064
:10A740004E2802D11121094A11700DE03A2803D197
:10A750000321C943064A11750A21044A117003E016
:10A760000A21024A117000BF00BF00BD300700205F
:10A770003334002000B5694909780A390B0019F013
:10A7800004FF0C07111B252F39434D57737D9EC6BF
:10A790002B2803D10B21614A117002E00A215F4A84
:10A7A0001170B8E04E2803D10C215C4A117002E010
:10A7B0000A215A4A1170AEE0532803D10D21574A9D
:10A7C000117002E00A21554A1170A4E04F2803D10C
:10A7D0000E21524A117002E00A21504A11709AE08B
:10A7E0004E2803D10F214D4A117002E00A214B4A35
:10A7F000117090E04D2803D11021484A117002E0F9
:10A800000A21464A117086E0492803D11121434AA2
:10A81000117002E00A21414A11707CE03A2803D10C
:10A8200012213E4A117002E00A213C4A117072E086
:10A8300000213B4A9172D1723A4A1180302806D1E8
:10A840000121394A51721321344A11700BE0312829
:10A8500006D10221344A51721321304A117002E0AC
:10A860000A212E4A117056E02C2803D114212B4ABC
:10A87000117002E00A21294A11704CE02C2810D0F6
:10A8800030281BDB392819DC264909880A22514364
:10A89000244A11800146303912888918214A1180D2
:10A8A0000CE02049098801229202914203DA152125
:10A8B0001A4A117002E00021184A11702BE0184A60
:10A8C000D17A927A09021143164A128852009142B3
:10A8D00012DA134AD17A937A0A021A43104BD97AC0
:10A8E0009B7A09021943491C8BB20D498B721B0AD2
:10A8F000CB720C31885409E00321C9430A4A203A3B
:10A900001175012191750A21044A117003E00A2191
:10A91000024A117000BF00BF00BD0000690700209F
:10A92000332E0020340700205334002010B5044695
:10A93000484800780A38030019F027FE0B07111B5E
:10A94000252F39434D57616E8600442C03D10B20CF
:10A950004049087002E00A203E49087078E0492C1E
:10A9600003D10C203B49087002E00A2039490870E5
:10A970006EE0532C03D10D203649087002E00A2006
:10A980003449087064E0432C03D10E20314908702B
:10A9900002E00A202F4908705AE04F2C03D10F2003
:10A9A0002C49087002E00A202A49087050E0562C11
:10A9B00003D110202749087002E00A2025490870B9
:10A9C00046E0452C03D111202249087002E00A20FC
:10A9D000204908703CE0522C03D112201D49087018
:10A9E00002E00A201B49087032E03A2C03D1132000
:10A9F0001849087002E00A201649087028E02C2C3B
:10AA000009D10020144908700A211448FDF73BFCC5
:10AA10001420104908701BE02C2C0CD00E48007834
:10AA20000A2810D20C4801780078401C0A4A10709D
:10AA30000A48445407E00320C04308492B390875ED
:10AA40000A200449087003E00A200249087000BF88
:10AA500000BF10BD81070020820700205E34002067
:10AA6000014800787047000041000020034800784A
:10AA7000002801D1012070470020FCE740000020A1
:10AA8000002004490978002901D1012000E00020BC
:10AA9000704700004000002070B555480078030062
:10AAA00019F073FD050405102593A3009EE0012015
:10AAB00000F0CEFD002804D10EF0C7FE02204C4964
:10AAC000087093E04B48007800F008F9012000F08E
:10AAD00017F900F079F915F0BBFD4749086015F04A
:10AAE000B7FD464908600320414908707EE0012017
:10AAF00000F022F9012855D115F0AAFD3F49086060
:10AB000015F0A6FD3C490968401A3D49096888428C
:10AB10005AD3002400F01CF904463A484068001952
:10AB20003849486038480078002803D108468460D6
:10AB3000046013E033488068A04201D2204601E05F
:10AB4000304880682F49886008460068A04201D9D3
:10AB5000204601E02B4800682A4908602A4800780E
:10AB6000401CC0B22849087028490978884215DB82
:10AB700000252448406823490968401A214989680A
:10AB8000451A22480078811E2846FDF7C3FA20495D
:10AB90000968086004201649087002E00220144980
:10ABA000087011E015F054FD14490968401A642832
:10ABB0000AD900F00FF91748007802210843154917
:10ABC000087004200A49087010E000F0A1F800F0B5
:10ABD0004BFC0021102015F0C7F901200E4909682F
:10ABE000087000200249087000E000BF00BF70BD7F
:10ABF0004000002051000020540000205800002098
:10AC0000480000208813002050000020520000203F
:10AC100044000020410000204C00002010B500F04E
:10AC200077F800F021FC0021102015F09DF910BDEF
:10AC3000F8B505460C4616461F46032C00D20324E1
:10AC4000502C00D950241B4906980860192D0ADDA4
:10AC50001948007801210843174908700120154957
:10AC600009680870F8BD1548076000201149096897
:10AC700008701349087013494860086088600E49DD
:10AC800008701148057011490C70114806600EF0EB
:10AC9000F6FD0121102015F067F900F0EFFB00F040
:10ACA00041F80121084614F087F90120094908708C
:10ACB00000BFD7E74C0000204100002044000020E6
:10ACC0005000002088130020510000205200002076
:10ACD000480000204000002070470000014607485F
:10ACE0004068FF22F13290430A01FF23F1331A40FA
:10ACF0001043024A506000207047000000240040CA
:10AD00000249496B8143014A5163704780240040E6
:10AD1000034840684008400001494860704700000F
:10AD2000002400400348406840084000401C01499E
:10AD3000486070470024004001460448006B08400A
:10AD4000002801D0012070470020FCE7802400404B
:10AD50000148006A704700008024004010B5044696
:10AD6000002C01D1042010BD0120164948600220AA
:10AD70001AF078FA6078A1880843E188084361886E
:10AD80000843218908430F49496808430D49486031
:10AD900008468068091588432178890201229202B9
:10ADA00011400843074988600846806804218843A9
:10ADB000A17A8900042211400843024988600020DA
:10ADC000D1E70000002400400120014908607047DD
:10ADD000C02400400020014908607047C0240040A2
:10ADE00030B50A4600210EE0D400A41A074D6419BC
:10ADF000635C04785C4004700478AA256C4004709D
:10AE0000401C4C1CE1B20729EEDB30BD8CC10200B6
:10AE1000F0B589B012F082FF10210840002810D050
:10AE2000042012F0A3FFFC480088401CFA49088067
:10AE3000E1210901F8480088FDF782F988B2F64956
:10AE4000088012F06BFF20210840002822D0052046
:10AE500012F08CFFF1480078401CF0490870084659
:10AE600000783C2816DB00200870ED48FDF732FA28
:10AE7000E12109014418EA492046FDF743FAE84870
:10AE8000001DFDF727FA0446233CE549091D20462D
:10AE9000FDF738FAE3480078002804D001280ED0E6
:10AEA00002287DD1A9E103F005F8002806D1DA488F
:10AEB0000088DD4908600120DA490870D0E102F01D
:10AEC000F9FF01286DD1002107910691D248008831
:10AED000D5490968884207D3CF480088D2490988F4
:10AEE000401AD249088009E0CB480088E1210901D5
:10AEF0004018CD490988401ACC49088008201EF026
:10AF0000B9FC772807D1C94800884B21C9004018EF
:10AF1000C64908800BE008201EF0ACFC552806D17D
:10AF2000C2480088E121C9004018C04908800021BA
:10AF300008201FF0A1FFBA480C30FDF7CBF9BB4940
:10AF400009884418B6490C312046FDF7DBF9B448AE
:10AF5000417C027C08021043401C81B2B04801745D
:10AF6000090A417407A80FF0F7F806A80FF0E6F8F1
:10AF70000A216A461C20105EFDF7E2F800B2079035
:10AF80000A216A461820105EFDF7DAF800B2069032
:10AF900004201EF06FFC01283ED1A448008801E087
:10AFA0005AE129E1FDF752FCA14AA24B0191009020
:10AFB000FDF746FB059104909948001DFDF78AF9BD
:10AFC0000746FDF743FC03910290059B049AFDF7A9
:10AFD00029FB0546FDF774FC04469149091DFDF760
:10AFE00091F904F0A7FD002815D193480078401C82
:10AFF00091490870072190480078FDF7A1F8C8B280
:10B000008D4908700846017802201FF035FF0121A4
:10B010000A201FF031FFEBE069461C20085E002883
:10B0200022DA82480088FDF711FC0646804A524227
:10B03000824BFDF705FB04460D467948001DFDF7E0
:10B0400049F90646FDF702FC22462B460191009085
:10B05000FDF7E8FA03910290FDF732FC7049091DF3
:10B060000590FDF74FF9C3E069461820085E772187
:10B07000C943884221DA6D480088FDF7E7FB0646A0
:10B080006B4A52426D4BFDF7DBFA03910290644824
:10B09000001DFDF71FF90646FDF7D8FB0191009052
:10B0A000039B029AFDF7BEFA0446FDF709FC5C49D2
:10B0B000091D0590FDF726F99AE069461820085EFB
:10B0C0007221C943884221DA58480088FDF7BEFB47
:10B0D0005B4A5C4B01910090FDF7B2FA04460D46C5
:10B0E0004F48001DFDF7F6F80190FDF7AFFB06464F
:10B0F00022462B46FDF796FA03910290FDF7E0FBFE
:10B100004749091D0590FDF7FDF871E069461820D3
:10B11000085E6821C943884220DA44480088FDF768
:10B1200095FB0646424A484BFDF78AFA019100908A
:10B130003B48001DFDF7CEF80646FDF787FB0446A9
:10B14000019B009AFDF76EFA03910290FDF7B8FBA0
:10B150003349091D0590FDF7D5F849E069461820E7
:10B16000085E5921C943884221DA30480088FDF73A
:10B170006DFB2F4A354B01910090FDF761FA0646B1
:10B180000F462748001DFDF7A5F80190FDF75EFB6F
:10B19000044632463B46FDF745FA03910290FDF71F
:10B1A0008FFB1F49091D0590FDF7ACF820E01F48F3
:10B1B0000088FDF74BFB0646214A5242244BFDF71F
:10B1C0003FFA019100901648001DFDF783F80646EE
:10B1D000FDF73CFB0446019B009AFDF723FA03911F
:10B1E0000290FDF76DFB0E49091D0590FDF78AF8E9
:10B1F00002200C49087000BF32E001F067FA012814
:10B2000008D1144B1822D021054801F0C3FC0020BE
:10B210000449087024E00000700500207205002039
:10B22000F42600206105002064050020740500203C
:10B23000CDCCCCCCCCCC1A408405002033333B4061
:10B240009A99999999993940CCCC2140CCCC1C4001
:10B25000666618406005002000205A49087000BF4B
:10B2600000BF59480078002802D001284FD10BE0D8
:10B270000AF042FD002806D154480088544908606D
:10B2800001205149087046E00AF036FD01283DD101
:10B290004E4800884E490968884207D34B480088C9
:10B2A0004B490988401A4B49088009E04748008803
:10B2B000E1210901401846490988401A454908809A
:10B2C00045480068434909884018434908600846D2
:10B2D00000683C2817D9084600683C3808603F4899
:10B2E000FCF7F8FF04463C343C492046FDF70AF8D9
:10B2F0003A48001FFCF7EEFF0446153C3749091F8A
:10B300002046FCF7FFFF00202F49087003E00020D3
:10B310002D49087000BF00BF31480078002802D0D6
:10B32000012848D10BE018F09DFA002806D12748E3
:10B3300000882C4908600120294908703FE018F076
:10B3400091FA012836D121480088264909688842A7
:10B3500007D31E48008823490988401A1D490880E0
:10B3600009E01A480088E121090140181D490988AF
:10B37000401A1849088019480838C17C827C0802A4
:10B38000104314490988401881B214480838817460
:10B39000090AC174001DFCF79DFF0E4909882A2285
:10B3A0005143441A0D49091F2046FCF7ABFF00200A
:10B3B0000B49087003E000200949087000BF00BF76
:10B3C00009B0F0BD61050020620500207005002075
:10B3D00068050020740500206C050020FC26002074
:10B3E000850500208805002007480078002809D13D
:10B3F00006480078002805D105480078002801D1CA
:10B40000012070470020FCE7610500206205002054
:10B4100085050020014680200840002801D008460C
:10B420007047302905DB392903DC08463038C0B2C3
:10B43000F6E7612905DB662903DC08465738C0B208
:10B44000EEE7412905DB462903DC08463738C0B260
:10B45000E6E70846E4E701460A110A235A430B07C8
:10B460001B0FD218D0B27047034800680221084071
:10B4700001490860704700000024004010B50548ED
:10B4800000680121084303490860022019F0EAFE20
:10B4900010BD00000024004030B502460020140218
:10B4A000044D63191C68240C24048DB22C431C60C9
:10B4B00030BD0000000C004030B5024600201402F0
:10B4C000044D63195C68240C24048DB22C435C6029
:10B4D00030BD0000000C004010B5014600200B02FA
:10B4E000014C1A19906810BD000C004030B502469E
:10B4F00000201402024D63199C68996030BD000061
:10B50000000C004070B5024600201402054D63197E
:10B510001C6BAD14AC430D030126360335402C43A0
:10B520001C6370BD000C004010B5014600200B02EA
:10B53000034C1A19D3685B085B005B1CD36010BD19
:10B54000000C004010B5014600200B02034C1A19F4
:10B55000D3685B085B00D36010BD0000000C0040A6
:10B5600070B503460A4600201C02224D6119CC68C2
:10B57000AD00AC4315782D030326360335402C432C
:10B58000CC60CC6801256D02AC4355786D02012674
:10B59000760235402C43CC60CC687510AC4395786E
:10B5A0002D02761035402C43CC60CC687025AC431E
:10B5B000D5782D01702635402C43CC60CC68082509
:10B5C000AC431579ED00082635402C43CC60CC689F
:10B5D0000425AC435579AD00042635402C43CC609E
:10B5E000CC680225AC4395796D00022635402C438A
:10B5F000CC6070BD000C004010B500F009F910BD22
:10B6000070B5044600252C2C1BDA15F021F80546F0
:10B61000A0000D490858A84203D8A00008582D1AC8
:10B6200006E0A000084908580021C943081A451936
:10B63000A00006490858A84201D8002070BD01208A
:10B64000FCE70020FAE70000E40C0020940D002045
:10B6500070B504460025182C1BDA14F0F9FF0546D6
:10B66000A0000D490858A84203D8A00008582D1A78
:10B6700006E0A000084908580021C943081A4519E6
:10B68000A00006490858A84201D8002070BD01203A
:10B69000FCE70020FAE70000240C0020840C0020C6
:10B6A0000148007870470000C803002010B5064824
:10B6B000FCF71AFE054B064A43404A40134301D1AA
:10B6C000012010BD0020FCE7421A0020B8A7F6E5D3
:10B6D000D4C3B2A101480078704700009C0200204A
:10B6E00070B504460025002614F0B2FF064609484E
:10B6F0000068351A0848844203D1A54201D30120CD
:10B7000070BD0648844203D1A54201D30120F7E76A
:10B710000020F5E71800002050C30000C0270900F2
:10B720000148007870470000C9030020FFB583B0CE
:10B7300006460F461C4638461EF0D2F80290059881
:10B740001EF0CEF8019060782178000208430028AE
:10B7500006DD6078217800020843164988420FDB35
:10B7600060782178000208431249083188421EDDC2
:10B7700060782178000208430E490931884216DAC0
:10B780006078217800020843B04203D009480F30A6
:10B7900086420CD1A01C1EF0A3F8054602988542F3
:10B7A00005D30198854202D8012007B0F0BD0020E2
:10B7B000FBE70000F0FF0000014800787047000040
:10B7C0005203002001480068704700005403002025
:10B7D000002002498872C872704700004B2900207F
:10B7E0000020014908707047F6020020002001493E
:10B7F000C875704733340020002001490870704735
:10B800009C0200200020014908707047520300206C
:10B8100010B5012015F034F801280DD115F02AF8E3
:10B8200057490860084600685649884205D115F016
:10B830003DF8FF205449087096E05148006851498E
:10B84000884246D215F032F850480078002803D0DC
:10B850004E48007801281ED101204C490870484903
:10B860000968484A501A4949491CFCF74BFD4849A8
:10B87000C968491C4805400D4549C968C90AC9023B
:10B880000143434AD16015F007F842480078401C54
:10B890004049087068E03D48401CFCF71BFD3849F2
:10B8A0000968384A511A88420FD23949C968491C77
:10B8B0004805400D3649C968C90AC9020143344ADE
:10B8C000D160FF20304908704EE0FF202E490870FB
:10B8D0004AE02B4800682B49884245D914F0E6FF1E
:10B8E0002A480078002803D02848007802281ED172
:10B8F00002202649087022490968224A881A2349E9
:10B90000491CFCF7FFFC2249C968491E4805400D47
:10B910001F49C968C90AC90201431D4AD16014F010
:10B92000BBFF1C480078401C1A4908701CE01748EF
:10B93000401CFCF7CFFC12490968124A891A884258
:10B940000FD21349C968491E4805400D1049C968FE
:10B95000C90AC90201430E4AD160FF200A49087092
:10B9600002E0FF2008490870022014F089FF012836
:10B9700004D114F09BFFEE200349087010BD0000B5
:10B980000403002000093D00FA020020FC02002010
:10B9900000200040FB02002010B5002014F0BCFA8B
:10B9A000002014F0CDFA112014F02CFB022014F02A
:10B9B00017FB0121022014F049F9022014F046FB84
:10B9C000042014F0F9FA0121002014F03FF90020BE
:10B9D00014F03CFB0121062002F0F8FE002002F0EA
:10B9E00059FF01211C2014F0BFFA10BD00200149AD
:10B9F00008707047C404002010B500F001F810BDB5
:10BA0000F8B5C0480078030018F0BFFD050422E631
:10BA1000FBFAF9000020BC490870FF202D301FF010
:10BA200039FA1DF00DFF01280ED10020B64908702B
:10BA3000B648FCF74FFCA32101700020B149087003
:10BA4000A920B349087002E00120AE49087057E10F
:10BA500019F0AEF800287DD10824AE480688AE481B
:10BA60000568002751E0E85D0A2808DAE85D303013
:10BA7000C2B22046611C8CB2A8490A543EE0E85D7F
:10BA8000642816DAE85D0A21FCF75AFB3030C2B2AE
:10BA90002046611C8CB2A1490A54E85D0A21FCF7DA
:10BAA0004FFB3031CAB22046611C8CB29B490A540C
:10BAB00024E0E85D6421FCF743FB3030C2B220464D
:10BAC000611C8CB295490A54E85D0A21FCF738FBE9
:10BAD0000A210090FCF734FB3031CAB22046611CC9
:10BAE0008CB28E490A54E85D0A21FCF729FB3031FB
:10BAF000CAB22046611C8CB288490A542E222046C4
:10BB0000611C8CB285490A547F1C042FABDB601E7C
:10BB100084B22C222046611C8CB280490A54804990
:10BB20003046FCF70DFB3030C2B22146601C84B2B7
:10BB30007A4842547A493046FCF702FB0F467D2191
:10BB4000C9003846FCF7FCFA3030C2B22046611C0E
:10BB50008CB200E03FE071490A547D21C9003046B3
:10BB6000FCF7EEFA0F4664213846FCF7E9FA30306C
:10BB7000C2B22046611C8CB268490A546421304626
:10BB8000FCF7DEFA0F460A213846FCF7D9FA3030C6
:10BB9000C2B22046611C8CB260490A540A21304668
:10BBA000FCF7CEFA3031CAB22046611C8CB25B4938
:10BBB0000A540D222046611C8CB258490A541222A4
:10BBC000214656480FF05EFF02201FF06FF9022059
:10BBD0004C49087000BF93E01DF032FE012811D1DE
:10BBE0000020494908704948FCF774FBA321017003
:10BBF000002044490870A920454908702FE07BE0E7
:10BC000044E02DE00EF0D0F9001D002809D13E4996
:10BC1000087003203B490870FF202D301FF03AF9CF
:10BC20001DE018F0CAFF002804D00EF0BDF9C01CBA
:10BC3000002814D134480078401C33490870084665
:10BC40000078012808DB0020087003202D490870C7
:10BC500002201FF02BF902E001202A4908704FE072
:10BC600018F0A6FF002810D12E480068FCF722FB30
:10BC700084B21B2221462B4800680FF003FF2320CB
:10BC80001FF014F904201F49087039E01DF0D8FD99
:10BC900001280ED100201C4908701C48FCF71AFB33
:10BCA000A3210170002017490870A92018490870C5
:10BCB00021E018F082FF00281DD113480078401CB5
:10BCC000114908700846007801280DDB0020087033
:10BCD0000E48FCF7FFFAA521017000200949087001
:10BCE000A8200B49087006E0032006490870FF20D1
:10BCF0002D301FF0CFF803E000200249087000BF8C
:10BD000000BFF8BD960500204E060020C529002082
:10BD10008E050020A8050020A40500204F06002065
:10BD2000102700008406002010B500F001F810BDB7
:10BD300070B5E3480078030018F027FC05041C33B5
:10BD40004FFDFC000320DE490870FF202D301FF05E
:10BD5000A1F8DC48807A552804D0DA48763080781B
:10BD6000552803D10120D649087002E00320D449A8
:10BD70000870A3E118F01CFF002811D1D248006818
:10BD8000FCF798FA84B200222146CF4800680FF0F1
:10BD900079FE0220CA4908707D20C0001FF07AF8A1
:10BDA0008CE10EF001F9001D002809D1C749087087
:10BDB0000320C3490870FF202D301FF06BF80BE003
:10BDC00018F0F6FE002804D00EF0EEF8C01C002893
:10BDD00002D10320BA49087070E118F0E9FE00288A
:10BDE00072D10824002504E0B948405DB94948559E
:10BDF0006D1C082DF8DBB84A517A127A09021143FA
:10BE00000846B649FCF79CF93030C2B22046611CA6
:10BE10008CB2B0490A54B04A517A127A09021143DD
:10BE20000846AE49FCF78CF90E467D21C900304624
:10BE3000FCF786F93030C2B22046611C8CB2A549AD
:10BE40000A54A54A517A127A0902114308467D2103
:10BE5000C900FCF775F90E4664213046FCF770F90D
:10BE60003030C2B22046611C8CB29A490A549A4AB8
:10BE7000517A127A0902114308466421FCF760F9ED
:10BE80000E460A213046FCF75BF93030C2B220463C
:10BE9000611C8CB28F490A548F4A517A127A090276
:10BEA000114308460A21FCF74BF93031CAB220464B
:10BEB000611C8CB287490A542C222046611C8CB22A
:10BEC00084490A54002549E0BCE08348001DFCF782
:10BED00001FA405D00110A280CDB7F48001DFCF7C9
:10BEE000F9F9405D001137302146621C94B2794A5D
:10BEF00050540BE07848001DFCF7ECF9405D001150
:10BF000030302146621C94B2724A50547248001D6F
:10BF1000FCF7E0F9405D0007000F0A2810DB6E48CF
:10BF2000001DFCF7D7F9405D0007000F37302146B0
:10BF3000621C01E0BEE086E094B2664A50540CE018
:10BF40006548001DFCF7C6F9405D0007000F303062
:10BF50002146621C94B25F4A50546D1C5E49487A77
:10BF6000097A00020843A842AFDC5648007B8021D2
:10BF70000840002829D05348007B8007800F002804
:10BF800023D02C222046611C8CB252490A54312203
:10BF90002046611C8CB24F490A5430222046611C55
:10BFA0008CB24C490A5431222046611C8CB249495A
:10BFB0000A540D222046611C8CB246490A5437228D
:10BFC000214644480FF05EFD35E03E48807A552812
:10BFD00004D03C4876308078552821D12C22204648
:10BFE000611C8CB23B490A5431222146601C84B248
:10BFF0003848425430222046611C8CB235490A54DC
:10C000002046611C8CB233490A540D222146601C23
:10C0100084B230484254372221460FF033FD0AE003
:10C020000D222046611C8CB22A490A541622214650
:10C0300028480FF027FD04201EF038FF0420204977
:10C04000087000BF3AE00DF0AFFF001D00280DD1D1
:10C050001E490870A920224908701F48FCF73AF9C8
:10C06000A421017000201649087022E00DF09CFF09
:10C07000C01C002803D018F0A0FD002819D11348D7
:10C080000078401C114908700846007801280DDB33
:10C09000002008701048FCF71DF9A5210170A820A8
:10C0A0000F49087000200649087002E00420044986
:10C0B000087003E000200249087000BF00BF70BD97
:10C0C00098050020B82600208C0600208806002055
:10C0D000D2C10200CF290020C5290020102700006E
:10C0E0008E05002000200149087070479605002049
:10C0F00070B546480078002806D0012805D00328EE
:10C1000074D006287CD123E07EE000F0DFFA01281D
:10C110001DD13F48007820280FD0DC223D493E4801
:10C12000FCF798F83D4BDC22012149023A4800F027
:10C1300031FD03203549087009E0384BDC223649CF
:10C140000120400200F0E0FC0620304908705BE06E
:10C1500000F0BCFA012846D1002500242EE0A10001
:10C160002D4A8818FCF7B6F80021C943884201D14E
:10C17000002525E0A100284A8818FCF7ABF8064600
:10C1800031462748FCF712FC09D3A100224A88183F
:10C19000FCF7A0F806462349FCF708FC01D200256D
:10C1A0000EE0A1001C4A8818FCF794F8064600210E
:10C1B000FCF7FCFB00D00125601CC4B2372CCEDBA1
:10C1C00000BF002D0BD1DC2212491348FCF742F8C6
:10C1D000124BDC22012149020F4800F0DBFC032056
:10C1E0000A49087000BF0FE000E009E000F06EFAB5
:10C1F000012804D10C49087000200449087003E0AC
:10C2000000200249087000BF00BF70BD1605002065
:10C21000242600205CC20200AB3C00201505002053
:10C2200000007A4400007AC4170500200146002966
:10C2300006D10D48407F012800D170470020FCE75F
:10C24000012906D10848807F012800D1F5E70020A8
:10C25000F3E7022906D10448C07F012800D1ECE7AA
:10C260000020EAE70020E8E77029002010B5C0466A
:10C27000C04610BD10B507480078002808D1064810
:10C280000078002804D110F065FF012800D110BD0E
:10C290000020FCE7110C00201C0C002010B510F051
:10C2A00063FF0B48C079202802DB00210848C171D8
:10C2B00007488079202802DB00210548817102208F
:10C2C00008F01EFA04460349FCF71CF810BD0000F4
:10C2D000E4260020120C002010B512F095FA12F09E
:10C2E0001DF810F0A9FF10BDF1B584B08F4800789B
:10C2F000002801D105B0F0BD8D48FBF7EBFF441CD1
:10C300008B492046FBF7FEFF8948FBF7E3FF044615
:10C310001421FBF7FFFE012908D186490498FBF799
:10C32000F1FF8449091D0498FBF7ECFF8148FBF7F6
:10C33000D1FF044621460498FCF742FB03D27D4915
:10C340000498FBF7DFFF7B48001DFBF7C3FF0446A3
:10C3500021460498FCF72AFB04D27649091D04986B
:10C36000FBF7D0FF72480830FBF7B4FF05462946BB
:10C370000498FBF7DFFF04466D490831FBF7C2FF65
:10C380006B48FBF7A7FF04461421FBF7C3FE032904
:10C3900008D26748FBF79EFF04461421FBF7BAFE5C
:10C3A000002936D16248FBF795FF07466048FBF746
:10C3B00091FF0646113614213046FBF7ABFE4000D4
:10C3C0003D1A2846FCF727FA04465948001DFBF79A
:10C3D00081FF02905748001DFBF77CFF0746554838
:10C3E000FBF778FF019052480830FBF773FF00908D
:10C3F0000199FBF7F0FF06463946FBF7ECFF0546CF
:10C400000299FBF797FF21460390FCF729F8049067
:10C4100022E04748FBF75EFF07464548FBF75AFF17
:10C4200014210390FBF776FE40003E1A3046FCF7DD
:10C43000F2F904463E480830FBF74CFF06463C48FC
:10C44000001DFBF747FF07463146FBF773FF054624
:10C450002146FCF705F804903548FBF73BFF0446FE
:10C460001421FBF757FE002927D13148001DFBF7A7
:10C4700031FF03902F48001DFBF72CFF02902D4841
:10C48000FBF728FF07462A480830FBF723FF394609
:10C490000190FBF7A0FF06460299FBF79CFF0546BB
:10C4A0000399FBF747FF04462149091DFBF72AFFC3
:10C4B0001F4908310020FBF725FF1D48FBF70AFF45
:10C4C000E121C900884217D919490020FBF71AFF5A
:10C4D0001749091D0020FBF715FF154908310020F9
:10C4E000FBF710FF12490C310020FBF70BFF10493E
:10C4F00010310020FBF706FF049802F0E5F904462E
:10C500000B492839FBF7FEFE09482838FBF7E2FE05
:10C51000044608493439FBF7F5FE05482838FBF78F
:10C52000D9FE044604F0A2FF00BFE3E67D0300202D
:10C53000B01900207419002010B500F0C7F80128C8
:10C5400007D105480078002801D1012010BD002046
:10C55000FCE70020FAE700001405002010B54C4865
:10C560000078030018F011F80A0607112131415133
:10C570006171868E8AE00020464908700120464994
:10C58000087002204249087080E013F009FA41481F
:10C590000078012808D100203E49087001203E495A
:10C5A000087003203A49087070E0FFF7A1FD394890
:10C5B0000078012808D1002036490870012036494A
:10C5C000087004203249087060E002F0ADF931488B
:10C5D0000078012808D100202E49087001202E493A
:10C5E000087005202A49087050E014F075F92948B0
:10C5F0000078012808D1002026490870012026492A
:10C60000087006202249087040E011F037FE2148EA
:10C610000078012808D100201E49087001201E4919
:10C62000087007201A49087030E011F0A7FC19487B
:10C630000078012808D10020164908700120164909
:10C64000087008201249087020E000F03FF8012827
:10C650000FD112480078202808D020200F490870F8
:10C660000F4B012200210D4800F094FA09200849DF
:10C6700008700BE000F02AF8012802D100200449DC
:10C68000087003E000200249087000BF00BF10BD21
:10C690001405002017050020160500202426002080
:10C6A0001505002010B5FFF759FF00F087F810BD01
:10C6B00010B5044609F056FA012805D100F006F835
:10C6C000002801D0012010BD0020FCE703480078BD
:10C6D000002801D1012070470020FCE70400002061
:10C6E00003480078002801D1012070470020FCE7B2
:10C6F0000400002000B585B0072103A818F0A2FDB2
:10C700000C21684618F09EFD002168464173817334
:10C71000C1730174417403AA03210120000308F0CE
:10C7200001FD002168464173012141740021C1735C
:10C73000017403AA0821402008F0F4FC03AA09218F
:10C74000402008F0EFFC01220821402008F038FDCD
:10C7500001220921402008F033FD0022032101209D
:10C76000000308F045FD1148114908600122042129
:10C77000104812F039FC102010F000FF13F0BCFB41
:10C7800000900D4801904021684601725521417288
:10C790000021817269460648006808F095FE012272
:10C7A00002210C2000F0B2FA05B000BD00040040E8
:10C7B0003800002020200040A086010010B5C548A8
:10C7C0000078030017F0E1FE0906071019C4E5FD23
:10C7D000FCFBFA007CE10320BE4908700FF05EFE0E
:10C7E000BD4812F047FC73E10320BA4908700FF00E
:10C7F00071FEB94812F03EFC6AE1B748FEF770FFDF
:10C80000002859D0B548006808F055FEB4480078B3
:10C8100000283FD109F0AEF901281DD1B0480078B9
:10C82000401CAF49087003F08DF900220621AD4885
:10C8300012F0DAFB002203210120000308F0D8FCEB
:10C8400000220421A84812F0CFFBA34812F012FCEA
:10C850000720A04908707AE0A1480078401CA04950
:10C86000087003F06FF9002206219E4812F0BCFB0D
:10C87000002203210120000308F0BAFC0022042159
:10C88000994812F0B1FB944812F0F4FB082091494A
:10C8900008705CE000209249087003F053F9002210
:10C8A00003210120000308F0A3FC8B4812F0E2FBF7
:10C8B0000420884908704AE009F054F901282FD172
:10C8C00009F058F901280BD103F03CF90020844904
:10C8D0000870864812F0CEFB06207E49087036E0CC
:10C8E00013F0B6FE82490968401AC8282FD903F010
:10C8F00029F900207A49087000220621794812F0AF
:10C9000073FB002203210120000308F071FC0022C8
:10C910000421754812F068FB00206E49087016E08B
:10C920007448008801280FD113F092FE72490968FB
:10C93000401A7249884207D900206E4908800521B3
:10C940006648006808F01CFE032062490870BFE0DA
:10C950006148FEF7C5FE002817D0FFF7CBFE012285
:10C960000321100308F044FC012206215D4812F067
:10C970003BFB05215948006808F002FE564812F0BA
:10C9800079FB05205349087002E0042051490870E2
:10C990009EE05148FEF7A4FE00283CD04F480068B6
:10C9A000406908281DD104214C48006808F0E8FDC2
:10C9B000002206214B4812F017FB03E084E067E0F9
:10C9C0004AE02CE0002203210120000308F010FCC3
:10C9D00000220421444812F007FB00203D49087062
:10C9E0001CE04748007840218843454908700022F0
:10C9F00006213C4812F0F8FA00220321012000032E
:10CA000008F0F6FB00220421374812F0EDFA00206E
:10CA10003049087002E005202E49087058E033487C
:10CA2000FEF75EFE002813D0002206212D4812F0EA
:10CA3000DBFA002203210120000308F0D9FB0022C9
:10CA40000421294812F0D0FA00202249087002E09F
:10CA50000620204908703BE017F00CFC1E48FEF74A
:10CA60003FFE002813D0FFF745FE012203211003EB
:10CA700008F0BEFB012206211A4812F0B5FA012285
:10CA80000421194812F0B0FA0220124908701FE080
:10CA900017F0F0FB1048FEF723FE002813D0FFF735
:10CAA00029FE01220321100308F0A2FB0122062126
:10CAB0000C4812F099FA012204210B4812F094FA62
:10CAC00001200449087003E000200249087000BFFB
:10CAD00000BF10BD04000020C0270900380000205E
:10CAE00005000020080400402020004050C3000042
:10CAF000200000202E0000201C00002088130000D1
:10CB00003600002070470000F8B505460F46144671
:10CB10001E46402016490870002030702819012157
:10CB2000C903884221DC002C1DDD881184421ADCF7
:10CB300010480580104807601048048010480660BF
:10CB4000012204210F4812F04FFA012203211003A1
:10CB500008F04EFB012206210B4812F045FA012095
:10CB60000A490870F8BD0020FCE70020FAE7000041
:10CB700036000020340000200C0000202600002099
:10CB80001400002020200040080400400400002081
:10CB900070470000F8B507460D4614461E46602053
:10CBA0004D4908700020307028190121C9038842BE
:10CBB0007EDC002C7DDD881184427ADC47480580CC
:10CBC000474807602846E917890E09188911890125
:10CBD000691A444A1180104600884021081A4249C7
:10CBE00008802046E117890E09188902090C3F4A7E
:10CBF0001180E117890E091889118901611A3C4ACF
:10CC000011803A480088002827D13648008800194A
:10CC100040281ADD01203749088033480088201A4F
:10CC200084B22046E117890E091889112F4A118014
:10CC3000E117890E091889118901611A2C4A11809E
:10CC4000294800882C49088029E0002029490880CB
:10CC5000274800882849088021E0012025490880CC
:10CC600020480088002803D140202349088016E08E
:10CC70001D480088201A84B22046E117890E091841
:10CC800089111A4A1180E117890E09188911890141
:10CC9000611A174A118014480088174908801748FC
:10CCA000066001220421164812F09EF9012201E0DB
:10CCB00010E00DE00321100308F09AFA012206218A
:10CCC000104812F091F902200F4908700120F8BDB8
:10CCD0000020FCE70020FAE73600002034000020A6
:10CCE0000C000020280000202A0000202C0000203A
:10CCF0003000002032000020260000201400002018
:10CD000020200040080400400400002070B50446C4
:10CD10000E4615462046002805DBC206D20E01212C
:10CD20009140144A116000BF3146204617F03CFC88
:10CD3000012D0ED12046002809DB00BF00BFC2062E
:10CD4000D20E012191400C4A116000BF00BF00BF0C
:10CD50000FE0204600280ADBC206D20E01219140D6
:10CD6000054A80321160BFF34F8FBFF36F8F00BF52
:10CD700000BF70BD80E200E000E100E0F7B588B0E0
:10CD8000154600247F20C00507900C20069000BFA8
:10CD900009E0A001694A11580898FBF707FE00D87E
:10CDA00005E0601CC4B20698401EA042F1DC00BF42
:10CDB00063492846FBF7FAFD3CD8A1015F4A891870
:10CDC00048690999FBF70FFB05900999FBF70BFBE5
:10CDD0000646A001594A801801690898FBF703FB31
:10CDE00003900999FBF7FFFAA101544A89180590AD
:10CDF000C8680999FBF7F7FA0390A0014F4A801819
:10CE000081680898FBF7EFFAA20101904B481018CF
:10CE100041680198FBF78EFA02900399FBF78AFAB2
:10CE200004900599FBF786FA07463146FBF782FA2C
:10CE300007907DE043492846FBF7B8FD3CD8A101A7
:10CE40003E4A8918886A0999FBF7CDFA0590099935
:10CE5000FBF7C9FA0646A001384A8018416A0898CB
:10CE6000FBF7C1FA03900999FBF7BDFAA101334A18
:10CE700089180590086A0999FBF7B5FA0390A00193
:10CE80002E4A8018C1690898FBF7ADFAA2010190FB
:10CE90002A48101881690198FBF74CFA029003990F
:10CEA000FBF748FA04900599FBF744FA0746314628
:10CEB000FBF740FA07903BE0A101204A8918C86BB4
:10CEC0000999FBF790FA07460999FBF78CFAA2013A
:10CED00005901A481018816B0898FBF784FA0390A4
:10CEE0000999FBF780FA0746A20114495118486BCB
:10CEF0000999FBF778FA0390A001104A8018016B9A
:10CF00000898FBF770FA0190A0010C4A8018C16ADA
:10CF10000198FBF70FFA02900399FBF70BFA3946D9
:10CF20000490FBF707FA06460599FBF703FA07900A
:10CF300028460799FBF757FA0BB0F0BD7808002098
:10CF40000000044200003C4210B5C046C046C04646
:10CF5000C04610BD10B52E2001F072FD01280AD187
:10CF6000092010F0EBFE002805D12E2001F07AFDFB
:10CF7000022002F009FC10BDF0B589B004460E464F
:10CF800000270020069005900490039002900190E5
:10CF90000A2E01DA09B0F0BD0025CEE1A9006058E3
:10CFA0000021FBF70DFD06D8A9006058FB49096870
:10CFB000FBF7FCFC0CD3A90060580021FBF7F6FC42
:10CFC0007ED2A9006058F6490968FBF7F9FCF7D250
:10CFD0000498401CC0B20490781CC7B2022F70D1D4
:10CFE000012D49D1ED49A0680968FBF7E9FC05D995
:10CFF000EB49A0680968FBF7D9FC7DD8E749E068F0
:10D000000968FBF7DDFC05D9E549E0680968FBF72D
:10D01000CDFC0BD8E14920690968FBF7D1FC27D981
:10D02000DF4920690968FBF7C1FC21D90021E068CC
:10D03000FBF7BCFC0BD1D94920690968FBF7C0FCA0
:10D0400016D9D74920690968FBF7B0FC10D9D34934
:10D05000E0680968FBF7B4FC05D9D149E0680968C4
:10D06000FBF7A4FCC9D800212069FBF79FFC43D142
:10D0700005950120069063E10F2DF8D1C749E06ABC
:10D080000968FBF79DFC05D9C549E06A0968FBF70B
:10D090008DFCB2D8C149206B0968FBF791FC05D91A
:10D0A000BF49206B0968FBF781FC0ED8BB49606B58
:10D0B0000968FBF785FC2CD9B949606B096801E068
:10D0C00038E12CE0FBF772FC23D90021206BFBF741
:10D0D0006DFC0BD1B149606B0968FBF771FC18D985
:10D0E000AF49606B0968FBF761FC12D9AB49206B53
:10D0F0000968FBF765FC00E0FAE005D9A849206B58
:10D100000968FBF753FCADD80021606BFBF74EFCC0
:10D11000ADD102200690681EC0B2059010E1032F29
:10D120007EDB0D2F7CDCF01EA84261DD691C8900CE
:10D1300060589A490968FBF743FC07D9691C8900C4
:10D14000605897490968FBF731FC51D8A91C890040
:10D15000605892490968FBF733FC07D9A91C89007C
:10D1600060588F490968FBF721FC0FD8E91C89003A
:10D1700060588A490968FBF723FC35D9E91C890006
:10D18000605887490968FBF711FC2DD9A91C890053
:10D1900060580021FBF70AFC0FD1E91C8900605898
:10D1A0007E490968FBF70CFC1ED9E91C8900605810
:10D1B0007B490968FBF7FAFB16D9A91C890060585E
:10D1C00076490968FBF7FCFB07D9A91C8900605860
:10D1D00073490968FBF7EAFB0AD8E91C8900605823
:10D1E0000021FBF7E3FB03D1059501200690A7E0A2
:10D1F000052D7DDBE91E8900605868490968FBF749
:10D20000DFFB07D9E91E8900605865490968FBF70B
:10D21000CDFB6DD8291F890060586049096800E07E
:10D220004EE0FBF7CDFB07D9291F890060585C4908
:10D230000968FBF7BBFB0FD8691F89006058574985
:10D240000968FBF7BDFB35D9691F8900605854494F
:10D250000968FBF7ABFB2DD9291F89006058002115
:10D26000FBF7A4FB0FD1691F890060584B4909687F
:10D27000FBF7A6FB1ED9691F890060584849096859
:10D28000FBF794FB16D9291F8900605843490968A8
:10D29000FBF796FB07D9291F8900605840490968A8
:10D2A000FBF784FB47D8691F890060580021FBF712
:10D2B0007DFB40D102200690A81EC0B205903FE041
:10D2C0000E2F38D13549A06B0968FBF779FB05D9DA
:10D2D0003349A06B0968FBF769FB10D82F49E06B55
:10D2E0000968FBF76DFB07D92D49E06B096800E081
:10D2F00021E0FBF75BFB02D80320069020E02749E2
:10D3000020680968FBF75CFB05D925492068096896
:10D31000FBF74CFB0FD8214960680968FBF750FB0D
:10D3200005D91F4960680968FBF740FB03D8042052
:10D33000069005E00027681CC5B2B54200DA2DE66C
:10D3400000BF0698002863D1089020E0002515E072
:10D350006A1C9200A158AA00A058FBF731FB0BD21F
:10D36000A80020580390681C80002058A900605035
:10D37000691C890003986050681CC5B2701E08992A
:10D38000401AA842E4DC0898401CC0B20890701E05
:10D3900008998842DADC022007900EE05C03002046
:10D3A000600300200798800021580298FAF7C2FF16
:10D3B00002900798401CC0B20790B01E079988429F
:10D3C000F0DC301FFBF71CFA014600900298FBF7D7
:10D3D00047F8029009F054FA0A2818D10498032853
:10D3E00015DB00210298FBF7EBFA04D2944902986E
:10D3F000FBF7DCFA09D300210298FBF7D7FA06D233
:10D4000090490298FBF7DCFAF9D20020029014E16F
:10D41000069801284DD10598401CC0B2059005988A
:10D42000301AC6B2002509E0059828188000215856
:10D430000298FAF77FFF0290681CC5B2B542F3DB91
:10D440003046FBF7E8F9014600900298FBF708F830
:10D45000019000210198FBF7B3FA04D27A490198B0
:10D46000FBF7A4FA09D300210198FBF79FFA19D220
:10D4700076490198FBF7A4FA14D27548FAF72AFF07
:10D48000962808D872480C30FAF724FF962802D85C
:10D4900000200290D1E08321C9050298FAF7E0FF4D
:10D4A0000290CAE08321C9050298FAF7D9FF0290D9
:10D4B000C3E00698022845D1002507E0A8002158BE
:10D4C0000298FAF737FF0290681CC5B205988542AA
:10D4D000F4DB0598FBF79FF9014600900298FAF7F4
:10D4E000BFFF019000210198FBF76AFA04D2564968
:10D4F0000198FBF75BFA09D300210198FBF756FA74
:10D5000019D252490198FBF75BFA14D25048FAF746
:10D51000E1FE962808D84E480C30FAF7DBFE962834
:10D5200002D80020029088E08321C9050298FAF70A
:10D5300097FF029081E08321C9050298FAF790FFD6
:10D5400002907AE0069803283AD1E16BA06BFAF7D3
:10D55000F1FE0290012189070298FAF781FF0190FC
:10D5600000210198FBF72CFA04D237490198FBF708
:10D570001DFA09D300210198FBF718FA19D2334993
:10D580000198FBF71DFA14D23148FAF7A3FE96284A
:10D5900008D82F480C30FAF79DFE962802D80020B4
:10D5A00002904AE08321C9050298FAF759FF0290D8
:10D5B00043E08321C9050298FAF752FF02903CE04C
:10D5C0000698042839D161682068FAF7B3FE029002
:10D5D000012189070298FAF743FF01900021019881
:10D5E000FBF7EEF904D218490198FBF7DFF909D3EC
:10D5F00000210198FBF7DAF919D214490198FBF7D9
:10D60000DFF914D21248FAF765FE962808D81048B8
:10D610000C30FAF75FFE962802D8002002900CE04A
:10D620008321C9050298FAF71BFF029005E08321C8
:10D63000C9050298FAF714FF02900298AAE40000C4
:10D640008FC2753D8FC275BD0AD7233D0AD723BD52
:10D6500094190020FEB504460E4600200290142EB8
:10D6600000DD1426276820680190002518E0A80036
:10D6700021580198FBF7A4F902D2A8002058019084
:10D68000A80021583846FBF791F901D2A800275885
:10D69000A80021580298FAF74DFE0290681CC5B206
:10D6A000B542E4DB39460298FAF795FE00900199FD
:10D6B000FAF791FE0290B01EFBF7A2F80146009027
:10D6C0000298FAF7CDFEFEBDF3B597B00E460020E6
:10D6D000169014901390002515E0AA001799895808
:10D6E0002846EA0F12185210920003AB9950691C99
:10D6F0008A0017998958EA0F1218521092000BAB42
:10D700009950A81CC5B2B542E7DB00253AE00024D9
:10D710002FE0621C920003AB9958A2009858FBF7C7
:10D720004FF90DD2A00003A908581590601C800085
:10D730000858A10003AA5050611C89001598505048
:10D74000621C92000BAB9958A2009858FBF738F96D
:10D750000DD2A0000BA908581590601C8000085835
:10D76000A1000BAA5050611C890015985050601CF4
:10D77000C4B2F10F89194910491E491BA142C8DCE6
:10D78000681CC5B2F10F89194910491EA942BEDCB7
:10D7900001270FE0B80003AA11581498FAF7CAFD40
:10D7A0001490B8000BAA11581398FAF7C3FD139000
:10D7B000781CC7B2F10F89194910491EB942E9DC3A
:10D7C000301FFBF71DF8029013991498FAF7B2FD79
:10D7D00001900299FAF744FE1690169819B0F0BD20
:10D7E000F3B589B000200890002500260790069028
:10D7F0000590049003900290019000274C48006827
:10D80000002804D14B48076838460BB0F0BD00240F
:10D8100007E0A00046490858002800D104E0601C39
:10D82000C4B20A988442F4DB00BF0894089C012C1F
:10D8300005D13F4807683F4807603846E5E73C4860
:10D84000006804903A4800680390002415E0A000A6
:10D85000374909580498814203D3A0003449085835
:10D860000490A000324909580398814203D8A000CF
:10D870002F4908580390601CC4B208988442E6DB24
:10D88000002425E0A0002A4909580498401A029073
:10D8900029490298884207D8681CC5B2A0002449CB
:10D8A0000958069808180690A000214909580398BD
:10D8B000081A019020490198884207D8701CC6B206
:10D8C000A0001B490958059808180590601CC4B2AF
:10D8D00008988442D6DBB5420ED103990498401AC9
:10D8E0001549884205D829460698FAF713FC0746D9
:10D8F00015E01048076812E0B54208DD0A95069861
:10D9000007900A990798FAF705FC074607E00A9678
:10D91000059807900A990798FAF7FCFB0746002F2D
:10D9200002D00448076001E00248076838466CE707
:10D93000DC1F00207804002047E10000F7B59EB00E
:10D9400005461746002600201D901C901B901A903B
:10D950001990189017901690159028210BA8FAF797
:10D9600092FC282101A8FAF78EFC286819902868F3
:10D970001890012F0BD1286815904B491598086015
:10D980001F98006849490860159821B0F0BD00242F
:10D9900011E0A00029581998814202D3A00028580C
:10D9A0001990A00029581898814202D8A000285840
:10D9B0001890601CC4B2BC42EBDB002430E0A00035
:10D9C00029581998401A17903949179888420CD845
:10D9D000A1001F984058B1000BAA5050701CC6B24D
:10D9E000A00029581B9808181B90A00029581898C7
:10D9F000081A16902E49169888420FD8A1001F9831
:10DA000041581D98800001AA11501D98401CC0B2B9
:10DA10001D90A00029581A9808181A90601CC4B2CA
:10DA2000BC42CCDB1D98864214D10A2E0AD1314665
:10DA30001B98FAF76FFB159028220BA91B48FAF7E1
:10DA400009FC25E018480068159028211748FAF7C6
:10DA50001AFC1DE01D9886420DDD37461B981C9070
:10DA600039461C98FAF756FB159028220BA90F4847
:10DA7000FAF7F0FB0CE01D9F1A981C9039461C9891
:10DA8000FAF748FB1590282201A90848FAF7E2FBAB
:10DA90001598002803D004491598086002E0024850
:10DAA00000681590159870E77C040020DC1F0020AA
:10DAB00047E10000F0B587B004460E46002700207D
:10DAC00006902068059020680490032E2FDD002525
:10DAD00019E0A90060580599FAF772FF02D8A8006A
:10DAE00020580590A90060580499FAF75FFF02D802
:10DAF000A80020580490A80021583846FAF71AFCCC
:10DB00000746681CC5B2B542E3DBB01EFAF778FEE3
:10DB1000039038460499FAF75EFC01900599FAF7EC
:10DB20005AFC02900399FAF79BFC069003E0701EE2
:10DB3000800020580690069807B0F0BD10B5002070
:10DB4000C7494870022088700021C548C17006216D
:10DB50000171002141718171DD20C149C871E52148
:10DB6000BF480172D6214172CA218172BD49C1727A
:10DB7000090A01730020BA4948730021B84881732B
:10DB8000C17301210174072141741921817400209E
:10DB9000B349C8740021B2480175417501218175EE
:10DBA0000721C175992101760F21417600218176E7
:10DBB0000020AB49C876012008770721A8484177A3
:10DBC000192181770021C17730211C300171012199
:10DBD0004171022181710721C17119210172014630
:10DBE0000931A148FAF78EFB01219D48203041728E
:10DBF000002109304170142181708C21C1700521F0
:10DC000008380173002141739849801C0173090A87
:10DC100041730121C01E4174042111304170632100
:10DC200081707421C1706E21017162214171512195
:10DC30000F3041714921401D41704E2181704721B3
:10DC4000C17044210171412141714F2181714A21EB
:10DC5000C1714921017243214172482181722D21F4
:10DC6000C1724E210173472141734E2181734221BC
:10DC7000C1730021401F4175153041708170C17022
:10DC8000017141718171153801771C3041708170CB
:10DC9000C1700171417181710121001DC1700021AC
:10DCA000C01C41708170C1700171332141717821B4
:10DCB00081710021C01E81720421C17218210B30B4
:10DCC000417000218170AA21C170002101710B38BF
:10DCD00001744174014612310020FAF713FB6049C8
:10DCE00076310020FAF70EFB5D497A3101200004FD
:10DCF000FAF708FB5A497E3101200004FAF702FBCB
:10DD00005749823101200004FAF7FCFA5449863160
:10DD100001200004FAF7F6FA51498A310120000483
:10DD2000FAF7F0FA4E498E3101200004FAF7EAFAC8
:10DD30005A214B4880308174C174002004E00022D5
:10DD4000474994310A54401C2028F8DB0F214448ED
:10DD500080300175AA211430017255218172112180
:10DD60004173232181737F21C17302210174322108
:10DD70004174002181740521C17401750021417530
:10DD8000072181751421C175B8210C30017500215E
:10DD900041753749801C0175090A41750821801EAB
:10DDA0000176102141760F2181760421C17605216B
:10DDB0001B30417001211B384177E1218901801C12
:10DDC0000177090A417728211E3001700021417036
:10DDD000811C0020FAF796FA00212148C030817199
:10DDE000C171014608310020FAF78CFA1C49D03184
:10DDF0000020FAF787FA1A49D4311E48FAF782FA56
:10DE00001749D8310020FAF77DFA1549DC31002096
:10DE1000FAF778FA00211248D03001824182014697
:10DE200014311548FAF76EFA0D489430017C7630BB
:10DE300001717638417C763041717638817C76305C
:10DE4000C1707638C17C763081717638017D733847
:10DE50000173090A41737330417D7630C17110BD81
:10DE60002426002033160000B80B000052030000E7
:10DE70001A2B0000E0D14D000000404010B514F016
:10DE8000B3FC0B480078002804D0012803D00228F6
:10DE900007D103E009E000F017F806E000F0A4F96C
:10DEA00003E000200249087000BF00BF10BD000061
:10DEB0002A05002003480078002801D1012070477E
:10DEC0000020FCE72B05002010B5BB48007808288F
:10DED0007CD007DC030016F058FB0812447C7C5B06
:10DEE0008EAAB07C162872D004DC092870D00A28CB
:10DEF0006FD1F7E017286DD01828F9D11DE101F096
:10DF00000DFE01282CD1AD48C07A401CAB49C87227
:10DF1000C87A0A21FAF714F9C8B2A849C872E121EF
:10DF20000901242011F030F8A5480088401CA449BC
:10DF300008800D2000F08EFD0002000EAA2801D1FD
:10DF40000EF08EFA55219F488170232000F08AFD43
:10DF5000482000F087FD0BF06DFE01209649087007
:10DF60001BE10CF019F9002803D004209249087035
:10DF70000DE00CF007F9002809D093480CF072FF6F
:10DF80009249252011F000F804208B49087004E123
:10DF90000CF002F900281ED001F0CCFD092806D1B2
:10DFA00002208B49087006208349087022E08948C6
:10DFB000027BC37A10021843014600228548C01D27
:10DFC0000BF02AFD05207C49087013E04FE0A2E029
:10DFD00060E0DEE0A9E07C480078A52804D0252098
:10DFE000FDF70EFB002805D1F120794908700620C5
:10DFF00071490870D1E00020FEF718F9002806D01A
:10E0000001207349087006206B4908700EE06E48C5
:10E010000078A52804D02520FDF7F2FA002805D1C4
:10E02000F1206B490870062063490870B5E002F0E2
:10E0300085FB072060490870AFE0674A674964487C
:10E04000007801F093FF01F0EBFD01280ED101F003
:10E0500001FE012803D108205749087006E032214B
:10E06000262010F091FF0A205349087095E00CF02B
:10E0700089F801280DD1544B002257480188574890
:10E080000DF0B8FC6421262010F07EFF09204A49DB
:10E09000087082E0232000F0D3FC012804D0262061
:10E0A000FDF7AEFA00280FD1232000F0DBFC0220A0
:10E0B0004749087000214348417001200BF03EFDA4
:10E0C00007203D4908700CE03F480078A52808D19A
:10E0D00032213C48417003203D49087007203649F1
:10E0E00008705AE0482000F0ABFC002806D0482019
:10E0F00000F0B8FC3221262010F046FF2620FDF764
:10E100007FFA002806D101F061FD012802D1162016
:10E110002949087041E00CF035F8002804D011F0CE
:10E1200023F817202449087037E00CF02BF800285A
:10E1300002D01820204908702FE0FEF7C7FA012806
:10E1400026D10D2000F086FC0002000EAA280FD177
:10E1500000211C48763881700020214908700B4648
:10E160000122962117487438FEF714FD00F0F0FEE6
:10E170000BF00CFD13F034FFFDF738FCFDF728FB26
:10E1800000211048817000200B4908701549087063
:10E1900003E000200849087000BF00BFFFF78AFEB7
:10E1A000002807D12420FDF72BFA002802D11820DF
:10E1B0000149087010BD00002B0500204B290020EC
:10E1C000320500202E27002022050020B80B000079
:10E1D0003405002024260020200500204B270020A5
:10E1E000380500202A05002010B5FD4800780300FE
:10E1F00016F0CBF9190E3D5EF175A0DBF2EFEEEDF6
:10E20000F1F1ECEBEAE9E8E7E6E5E4E3E2E1F1006D
:10E2100001F084FC012829D1F248C07A401CF14960
:10E22000C872C87A0A21F9F78BFFC8B2ED49C872E3
:10E23000E1210901242010F0A7FEEB480088401CD2
:10E24000E94908800D2000F005FC0002000EAA2814
:10E2500001D10EF005F9232000F004FC482000F065
:10E2600001FC0BF0E7FC0120DD49087090E20BF0A7
:10E2700093FF00280DD01BF0DDFA002805D00DF02B
:10E280007DF90220D649087011E00420D4490870B5
:10E290000DE00BF077FF002809D0D4480CF0E2FD28
:10E2A000D349252010F070FE0420CD4908706FE29C
:10E2B0000BF068FF012811D11BF0BCFA012803D133
:10E2C0000520C749087009E0C8480CF0CBFDC849D3
:10E2D000252010F059FE0420C149087058E20BF0C7
:10E2E0005BFF002812D0002104201CF0C5FDC148AE
:10E2F000027BC37A1002184301460022BD48C01DAC
:10E300000BF08AFB0520B649087012E0B748007888
:10E31000A52804D02520FDF773F9002809D1012193
:10E3200004201CF0A9FDF120B34908700620AC4977
:10E3300008702DE20020FDF779FF002825D01BF0A2
:10E3400079FA012805D1AC4908700620A449087063
:10E350002AE007201BF08EFA01280FD100210720A8
:10E360001CF08AFD01201BF085FA04462146262078
:10E3700010F00AFE0A209A49087015E001209E4913
:10E3800008700620964908700EE098480078A52885
:10E3900004D02520FDF734F9002805D1F120964955
:10E3A000087006208E490870F2E102F0C7F90720D4
:10E3B0008B490870ECE1BBE1B2E1A7E18BE180E1C0
:10E3C0005EE142E12EE1F8E0F1E0D8E0B4E059E0AE
:10E3D00033E01FE000E0D7E1884A894986480078A9
:10E3E00001F0BCFE01F026FC012812D101F038FC3E
:10E3F000012803D108207A4908700AE001201BF0A7
:10E4000039FA04462146262010F0BEFD0A20744940
:10E410000870BDE10BF0B6FE01280DD1734B002250
:10E420007648018876480DF0E5FA6421262010F040
:10E43000ABFD09206A490870AAE1232000F000FB27
:10E44000012804D02620FDF7DBF800280FD1232077
:10E4500000F008FB00206B49087002206649087034
:10E4600000216948417007205D49087009E05F4854
:10E470000078A52805D103205F4908700720584976
:10E48000087085E1482000F0DBFA00280BD0482016
:10E4900000F0E8FA01201BF0EDF9044621462620A1
:10E4A00010F072FD47E02620FDF7AAF8002842D1BF
:10E4B00001F08CFB01283ED101F030FB01280FD187
:10E4C0004848C07A401C4749C872C87A0A21F9F7FF
:10E4D00037FEC8B24349C8720520414908702AE096
:10E4E0001BF0A8F9012815D147487638007B802118
:10E4F000084000280AD044487638007B8007800F07
:10E50000002803D014203649087014E00D20344947
:10E51000087010E006201BF0ADF9012808D1042096
:10E520001BF0A8F9002803D10D202D49087002E046
:10E5300016202B4908702BE101F048FB01281DD162
:10E540000BF020FE002819D000202B4908702E481F
:10E550002238827E437E10021843014601222A4857
:10E560000D380BF059FA01201BF084F904462146BE
:10E57000262010F009FD0E201949087008E101203D
:10E58000FDF754FE002806D001201B4908700F201B
:10E59000134908700AE02620FDF732F8002805D15B
:10E5A000F120154908700F200D490870F0E002F0C5
:10E5B000B9F810200A490870EAE0104A10490E48DC
:10E5C000007801F053FB01F021FB012829D101F073
:10E5D0003BFB01281AD111200149087021E00000FD
:10E5E0002B0500204B2900203205002022050020A9
:10E5F000B80B000024260020340500202005002050
:10E600004B270020350500202E27002001201BF07D
:10E6100031F904462146262010F0B6FC1320634948
:10E620000870B5E00BF0AEFD01280DD1604B012262
:10E630006048018860480DF0DDF93221262010F095
:10E64000A3FC122059490870A2E0232000F0F8F939
:10E65000012809D1232000F005FA0220574908704B
:10E660001020524908700AE02620FCF7C9FF002854
:10E6700005D103205149087010204C49087087E0EB
:10E68000482000F0DDF9002803D113F0AFFC012889
:10E690000AD1482000F0E6F901201BF0EBF804460F
:10E6A0002146262010F070FC2620FCF7A9FF002848
:10E6B00006D101F08BFA012802D116203B490870DF
:10E6C00066E00BF05FFD012804D10CF043FF15203C
:10E6D000364908705CE00BF055FD012815D11BF0A0
:10E6E000A9F802280ED101213548017213F078FCF7
:10E6F000FDF77CF9FDF76CF800202C4908703149D2
:10E70000087002E016202949087041E00BF03AFD3C
:10E71000002804D010F028FD17202449087037E0A5
:10E720000BF030FD002802D01820204908702FE09F
:10E73000FDF7CCFF012826D10D2000F08BF9000257
:10E74000000EAA280FD100211D48763881700020C4
:10E750001D4908700B460122962119487438FEF7AE
:10E7600019FA00F0F5FB0BF011FA13F039FCFDF784
:10E770003DF9FDF72DF800211148017200200B49E9
:10E7800008701049087003E000200849087000BFB5
:10E7900000BFFFF78FFB002807D12420FCF730FFD4
:10E7A000002802D118200149087010BD2B05002057
:10E7B00022050020200500204B27002034050020E2
:10E7C0002E2700202A05002038050020F0B58BB048
:10E7D00005460E4600242A480A9000200990202170
:10E7E00001A8F9F750FD274F012D0ED0022D0CD0B6
:10E7F000042D0AD0062D08D0082D06D00C2D04D0EB
:10E800000420099009980BB0F0BD1E48006A012150
:10E8100049028843710201225202114008431949FA
:10E820000862002407E0A000174908586843A100C7
:10E8300001AA5050641C082CF5D300241CE0104899
:10E840000A9011E00A98411E0A9100280AD00F4848
:10E850000C49C8620E48C862A00001A90858A1006E
:10E86000785001E00720CEE7A0003858A10001AAA7
:10E8700051588842E6D1641C082CE0D30998C2E7BD
:10E88000FFFFFF0000000240A0BD02005A5A000036
:10E89000A5A5000010B501460020084A084BDA6221
:10E8A000084ADA621A46126A0C239A438B000C2437
:10E8B00023401A43024B1A6210BD00005A5A00004E
:10E8C00000000240A5A5000070B5044647210906D6
:10E8D0002046FAF775F801D2002070BD8F21C905D6
:10E8E0002046F9F780FD0546F9F7BEFFF5E7000081
:10E8F00010B5002407F0E0FE044609480088201AFD
:10E9000080B208490860064804800846006805216E
:10E910000902884203D3032000020249086010BDA7
:10E92000D8030020D403002070B53D4800780028AB
:10E9300006D0012805D0032862D006286AD123E03A
:10E940006CE0FDF7C3FE01281DD136480078202871
:10E950000FD0482234493548F9F77CFC344B482223
:10E960000D2189013148FEF715F903202C49087063
:10E9700009E02F4B48222D490D208001FEF7C4F8F5
:10E9800006202749087049E0FDF7A0FE012836D18E
:10E99000012500241EE0A100244A8818F9F79AFCFA
:10E9A0000021C943884201D1002515E0A1001F4A7A
:10E9B0008818F9F78FFC1F49884207D8A1001B4A25
:10E9C0008818F9F787FC1C49884201D2002503E02A
:10E9D000601CC4B2122CDEDB00BF002D0BD148221C
:10E9E00011491248F9F736FC114B48220D218901D3
:10E9F0000E48FEF7CFF803200949087000BF0DE06C
:10EA0000FDF764FE012804D10C4908700020044978
:10EA1000087003E000200249087000BF00BF70BD0D
:10EA2000160500202426002014C20200633C0020AA
:10EA3000150500209919010066E600001705002061
:10EA400001465B2902DA0248405C70470020FCE77F
:10EA5000E836002001468800014A1058704700003F
:10EA60008025002001465B2904DA0020024A505428
:10EA7000012070470020FCE7E836002070B506460C
:10EA8000002405F0B3FEC4B2E007C00F00280ED08A
:10EA9000B848007802218843801CB64908700846AF
:10EAA000C078402188434030B249C8700BE0B1487B
:10EAB000007802218843AF4908700846C078402199
:10EAC0008843AC49C8700220204002280ED1A948D2
:10EAD0000078202188432030A64908700846C07875
:10EAE000202188432030A349C8700BE0A14800785A
:10EAF000202188439F4908700846C0782021884318
:10EB00009C49C87004202040042807D199484078C7
:10EB100040084000401C9749487005E095484078FF
:10EB2000400840009349487008202040082807D139
:10EB30009048407804218843001D8E49487005E0C4
:10EB40008C484078042188438A494870202020401E
:10EB5000202807D18748407802218843801C8549B6
:10EB6000487005E083484078022188438149487015
:10EB70004020204040280ED17E48007840084000C8
:10EB8000401C7C4908700846C0788021884380304A
:10EB90007849C8700BE07748007840084000754914
:10EBA00008700846C078802188437249C870802068
:10EBB000204080280ED16F480078402188434030A3
:10EBC0006C4908700846C07804218843001D6949D3
:10EBD000C8700BE067480078402188436549087099
:10EBE0000846C078042188436249C870FCF798FD44
:10EBF000012807D15F4840781021884310305D49D3
:10EC0000487005E05B4840781021884359494870B6
:10EC10001020204010280ED1564800780821884343
:10EC20000830544908700846C078102188431030D5
:10EC30005049C8700BE04F480078082188434D497F
:10EC400008700846C078102188434A49C8700DF002
:10EC5000E3FC0A2807D14748407820218843203028
:10EC60004449487005E043484078202188434149A1
:10EC7000487040484078C02188433E49487014F0AD
:10EC8000E7FD0446032C03D0042C01D0052C07D14A
:10EC900038484078C021884340303649487009E000
:10ECA000012C01D0022C05D132484078C021884384
:10ECB0003049487030484078002806D02D484078C8
:10ECC000C0218843C0302B4948700FF0CFF901288C
:10ECD0000ED12848007804218843001D254908707A
:10ECE0000846C0780821884308302249C8700BE0E4
:10ECF00020480078042188431E4908700846C078DF
:10ED0000082188431B49C870FCF7D0FC012807D1B3
:10ED1000184840780821884308301649487005E0B3
:10ED20001448407808218843124948701148C07837
:10ED300040084000401C0F49C870084680784008D1
:10ED40004000401C887009201AF094FD0949897818
:10ED50000843084988700DF065FC0546C00F40194E
:10ED6000C005000E0349087105223046F9F772FA12
:10ED700070BD0000780B00204D260020034800786D
:10ED8000002801D1012070470020FCE788070020FF
:10ED900010B50CF031FC11F015FE10BD5B2802DA45
:10EDA0000121014A11547047E836002070B504462D
:10EDB0000E460025FE20207060706820A070102094
:10EDC000E0705E484078102809D100BF04E05C483C
:10EDD000415D281D21546D1C072DF8DB24E05948A6
:10EDE000407801280DD1002056494870002505E0E3
:10EDF0005448801C415D281D21546D1C072DF7DBF4
:10EE000009E0002505E04E480E30415D281D2154E3
:10EE10006D1C072DF7DB49484078112804D149487B
:10EE2000417A201DFBF7DCFF44484078492811D087
:10EE300006DC11280BD045280AD046284CD108E022
:10EE4000512808D0542807D0642845D105E000BFD8
:10EE500000BF00BF00BF00BF00BF38488078E0722D
:10EE600039480078001D20733448007960733348B6
:10EE70004079A07331488079E0733048007A20747B
:10EE8000002505E03148415D2846113021546D1CB4
:10EE90002D4800888542F5DB28484078912805D127
:10EEA0002648017A20461130FBF79AFF2348027A60
:10EEB000207B0B30C1B2A01C0FF0A8F922490988B1
:10EEC00011316054162120480088123021541E4808
:10EED0000088133030802FE018488078E0721A489C
:10EEE0000078C01C2073154800796073134840797E
:10EEF000A07312488079E073002505E01348415D56
:10EF00002846103021546D1C0F4800888542F5DBDF
:10EF1000207B0B30C1B2A01C15F0F8FD0A4909880E
:10EF200010316054162108480088113021540648D9
:10EF300000881230308000BF00BF70BD8F400020BD
:10EF40007926002085400020F00B00209C40002006
:10EF50001FB52020AB490860AB48F9F7BBF9A949B8
:10EF60004860A948001DF9F7B5F9A6498860A64888
:10EF70000830F9F7AFF9A349C860A3480C30F9F796
:10EF8000A9F9A0490861A0481030F9F7A3F99D49F3
:10EF900048619D481430F9F79DF99A4988619A486B
:10EFA0001C30F9F797F99749C86197487238007F84
:10EFB00095497239497F0902084393497239897F1B
:10EFC000090408438F4908628F485638007A8E49F1
:10EFD0005639C979090208438B4956398979090498
:10EFE0000843884948628948886287481238C0784F
:10EFF00085490F3949780902084383490F398978CF
:10F000000904084380490F39C978090608437D4936
:10F01000C8627D480F3800797B490F394979090268
:10F02000084379490F398979090408437549086308
:10F0300075480E30007D7449223149780902084331
:10F04000714922318978090408436F492231C9780E
:10F05000090608436B4948636B48223000796A49C6
:10F060002231497909020843674922318979090423
:10F07000084365492231C979090608436149886313
:10F0800061482230007A60492231497A09020843F6
:10F090005D492231897A090408435B492231C97AE2
:10F0A000090608435749C86357482230007B564930
:10F0B0002231497B0902084353492231897B0904E3
:10F0C000084351492231C97B090608434D49086468
:10F0D0004D487238C07F4C495639097909020843B6
:10F0E000494956394979090408434649486446481C
:10F0F0001830F9F7EFF8434988646846FFF7BEFC1B
:10F1000001990098039102906946487A897A090228
:10F1100008433C4948653C482E30807D3A4944319B
:10F120004978090208433749886537482E30417DC0
:10F13000027D080210433349C86533482E30007EF3
:10F14000086631482E30407E48662F4872388078F5
:10F150002D497239C978090208432B497239097956
:10F1600009040843284972394979090608432549A1
:10F17000886725480E30807CC86723480E30C17CE4
:10F180002048803001602048723841781D48803026
:10F1900041601D482E30817E1A48803081601A48B7
:10F1A0003030417F027F08021043164980314861A8
:10F1B00015484E30417802780802104311498031D9
:10F1C00088610AF0EFFA0F498031C8610E48223099
:10F1D000017C763001717638417C76304171763829
:10F1E000817C7630C1707638C17C7630817176381A
:10F1F000017D73380173090A41737330417D7630A4
:10F20000C1711FBD8025002096260020970028B7D9
:10F210000020014908707047B00B00200020014910
:10F2200008707047F30B00200020014908707047F8
:10F23000040C002030B589B004460D461148817891
:10F24000684681750F480179684601760D48417915
:10F25000684641760B48C17A6846C177094881798A
:10F26000684681760748C1796846C17606480088B5
:10F27000064901AA31C2009105A80FC800F008F89C
:10F2800009B030BD873F0020A20B0020873D002041
:10F29000FFB581B00D9F0B9E0C9C0025FE202070B9
:10F2A00060706820A0701020E07000BF04E0584833
:10F2B000415D281D21546D1C072DF8DB68468079BF
:10F2C000E0726846C07B2073FB2E45DC301D607306
:10F2D0006846007AA0736846407AE0736846807A90
:10F2E00020746846C07A60743246204612300A990B
:10F2F000F8F7B0FF6846C07BC007C00F00280FD0EA
:10F30000627B444B21460E310020F9F7FFFC607B05
:10F31000C117090F09180911491C0907090E617362
:10F320000021607B0E302154022509E0607B0E3005
:10F33000205C615D4018C1B2607B0E3021546D1CB1
:10F34000607B0E30A842F1DC1621607B0F30215427
:10F35000607B1030388058E0301D81B200916846E3
:10F360000078607368464078A0736846007AE0735E
:10F370006846407A20746846807A60746846C07A2D
:10F38000A0743246204613300A99F8F763FF6846A6
:10F39000C07BC007C00F002816D069460A881D4BE5
:10F3A00021460F310120F9F7B1FC69460888C117E1
:10F3B000090F09180911491C09050A0C0092694630
:10F3C000487860730878A0730021684600880F3081
:10F3D000215402250BE0684600880F30205C615DF7
:10F3E0004018C1B2684600880F3021546D1C684631
:10F3F00000880F30A842EEDC1621684600881030E5
:10F400002154684600881130388005B0F0BD0000F6
:10F41000872600208F0B002030B589B004460D46AA
:10F4200011488178684681750F48017968460176F0
:10F430000D484179684641760B48C17A6846C177E4
:10F4400009488179684681760748C1796846C1765E
:10F4500006480088064901AA31C2009105A80FC8D4
:10F46000FFF716FF09B030BD9C440020F60B0020CA
:10F470009C42002001480078704700008402002070
:10F480001CB50721684615F0DDFE01216846417074
:10F49000C1706A460221C02005F044FE0322022109
:10F4A000C02005F015FE012203210846FDF72EFCC1
:10F4B0001CBD000010B500F00FF91348F8F70AFF63
:10F4C0001249884205D1002203210A20FDF71EFCC3
:10F4D0000AE00D48F8F7FEFE0D49884204D10022EB
:10F4E00003210B20FDF712FC0748F8F7F3FE032178
:10F4F00001610548F8F7EEFE1421016000210720A4
:10F5000010F032FD10BD00009413002000080040F0
:10F510000048004010B500F025F81148F8F7DAFE71
:10F5200000694021884344180D48F8F7D3FE046170
:10F530000B48F8F7CFFE006920218843441808489B
:10F54000F8F7C8FE04610648F8F7C4FE0069042114
:10F550008843041D0248F8F7BDFE046110BD000099
:10F560009413002038B580200EF008F800F06AF8F7
:10F570000121072010F0F8FC2F493048F8F7C2FEAF
:10F580002D48F8F7A7FE00684021884304462A4822
:10F59000F8F7A0FE04602849091D0020F8F7B2FE24
:10F5A000254908310420F8F7ADFE23491031022027
:10F5B000F8F7A8FE1021684601701F481030F8F7D0
:10F5C00089FEC1B2684641701B480830F8F782FED8
:10F5D000C1B26846C1701848001DF8F77BFEC1B281
:10F5E000684681701448F8F775FE044669460FF0C6
:10F5F00065FD1148F8F76EFE1149884205D10122D8
:10F6000003210A20FDF782FB0AE00B48F8F762FEAF
:10F610000A49884204D1012203210B20FDF776FB21
:10F620000548F8F757FE006840218843441802480F
:10F63000F8F750FE046038BD9413002000480040E5
:10F64000000800401CB50721684615F0FBFD0021AD
:10F65000684641706A46C02005F064FD0222002120
:10F66000C02005F0ADFD01220021C02005F0C0FD45
:10F67000012118480FF03CFD6A460121C02005F029
:10F6800051FD02220121C02005F09AFD0022012136
:10F69000C02005F0ADFD6A460421C02005F042FD02
:10F6A00002220421C02005F08BFD00220421C0208D
:10F6B00005F09EFD01216846417001716A460321F3
:10F6C000C02005F02FFD02220321C02005F078FDA7
:10F6D0001CBD0000004800401CB50721684615F01D
:10F6E000B1FD0020694648706A460121C02005F03E
:10F6F00019FD00220121C02005F062FD0022012138
:10F70000C02005F075FD6A460421C02005F00AFD01
:10F7100000220421C02005F053FD00220421C02056
:10F7200005F066FD6A460321C02005F0FBFC0022BF
:10F730000321C02005F044FD00220321C02005F074
:10F7400057FD6A460021C02005F0ECFC002211465E
:10F75000C02005F035FD01220021C02005F048FD44
:10F760001CBD00000148007870470000DA0300204B
:10F770000020014908707047DA0300200120014988
:10F7800008707047DA03002070B505460024002D8C
:10F7900004D0012D24D0022D7DD167E000203F4907
:10F7A00008703F4908703F4908603F4908603F4979
:10F7B000F8F7A8FD3D49091D0020F8F7A3FD002436
:10F7C00008E00020A1003A4A5050A100394A5050A8
:10F7D000601CC4B2962CF4DB0120374908705BE052
:10F7E00035480078012840D100203349087010F0D6
:10F7F000EBFD2B480078002837D0294801782C48A9
:10F80000FEF758F927490860254801782948FEF78E
:10F8100051F9254908608121C90522480068F9F796
:10F82000CFF812D38121C9051F480068F9F7C8F83D
:10F830000BD322491B480068F9F7B8F805D31F49D4
:10F8400019480068F9F7B2F804D200201549086099
:10F8500015490860154913480068F8F753FD134926
:10F86000091D11480068F8F74DFD15E00020124908
:10F8700008701348F8F72EFD06460C49F8F742FDCC
:10F880000F48001DF8F726FD06460849091DF8F740
:10F8900039FD01E0FFE700BF00BF70BD6804002034
:10F8A000690400206C04002070040020601900200E
:10F8B000041B00205C1D002074040020000080C098
:10F8C0003A1A002070B504460025552C03D10EF0DD
:10F8D00095FA054613E0012C04D1012004F010FF35
:10F8E00005460CE0022C04D1022004F009FF054675
:10F8F00005E0032C03D1032004F002FF054628464F
:10F9000070BD000070B504460025112C12D13A4894
:10F910000EF056FA00280BD0374800780004054353
:10F92000354840780002054333488078054361E05C
:10F93000324D5FE0222C12D131480EF041FA0028FE
:10F940000BD02F480079000405432D484079000270
:10F9500005432B48807905434CE0284D4AE0012CB3
:10F9600004D10020FFF776F8054643E0022C04D1CD
:10F970000A20FFF76FF805463CE0042C04D10B2069
:10F98000FFF768F8054635E0032C04D10C20FFF79B
:10F9900061F805462EE0052C04D106200DF0B2FDDD
:10F9A000054627E0062C04D107200DF0ABFD0546E7
:10F9B00020E0072C04D108200DF0A4FD054619E035
:10F9C000082C04D109200DF09DFD054612E0092CFC
:10F9D00004D10A200DF096FD05460BE00A2C04D157
:10F9E0002720FFF737F8054604E00B2C02D11BF067
:10F9F000ABFA0546284670BD40040020EEEEEE004E
:10FA00004704002070B50646002428480578012EDA
:10FA100027D108202840082801D1044303E0082109
:10FA200020468843044604202840042801D104438A
:10FA300003E004212046884304460220284002288F
:10FA400001D1044303E002212046884304464020BC
:10FA50002840402802D10120044325E064086400C6
:10FA600022E0022E20D110202840102801D104438A
:10FA700003E0102120468843044601200AF02AF8BA
:10FA8000002802D08020044303E0802120468843E0
:10FA9000044607484078002802D04020044303E091
:10FAA0004021204688430446204670BD2B04002098
:10FAB0004D26002038B504460025022C03D104F061
:10FAC000C7FE054622E0012C04D10C2004F0C0FE44
:10FAD00005461BE00A2C04D10A2004F0B9FE0546B5
:10FAE00014E0042C04D1042004F0B2FE05460DE01D
:10FAF000072C04D1072004F0ABFE054606E00E2CCF
:10FB000004D110F013FC0090009838BD2846FCE7A3
:10FB100002461068C840C007C00F70470448807A8A
:10FB20000349C97A884201D0012070470020FCE7D0
:10FB30004B2900200248C07A0149085C7047000048
:10FB40004B29002002480078024909680870704774
:10FB500036000020140000200148007870470000A3
:10FB6000F602002010B580200DF0FCFC0446600673
:10FB7000040E40200DF0F6FC04436006040E202025
:10FB80000DF0F0FC04436006040E10200DF0EAFCBA
:10FB900004436006040E08200DF0E4FC04436006F4
:10FBA000040E04200DF0DEFC04436006040E022067
:10FBB0000DF0D8FC04436006040E01200DF0D2FCC9
:10FBC00004436006040E204610BD00000148007882
:10FBD000704700008D070020014800787047000042
:10FBE000C40400200148407A7047000053340020CC
:10FBF00010B50446042C05DAA100034A8818F8F76A
:10FC000069FB10BD0020FCE7A41A0020034800781F
:10FC1000002801D1012070470020FCE7B10B002033
:10FC200003480078002801D1012070470020FCE73C
:10FC3000B30B002003480078002801D10120704751
:10FC40000020FCE7080C0020014800787047000005
:10FC5000B20B00200148007870470000B40B002070
:10FC60000148007870470000090C0020F0B591B001
:10FC700005460E461746012D7ED10020069006202F
:10FC800004F0E6FD81B2B2480170090A4170092012
:10FC900004F0DEFD80B2AE498870000AC87010F032
:10FCA00045FB059000210598F8F780FE1BD2E90777
:10FCB000059848400590A7490598F8F794FB044635
:10FCC000F8F7D2FD81B2A2480171090A41710146DB
:10FCD0004879097900020843E90308439C490871FF
:10FCE000000A487115E09B490598F8F77CFB04462B
:10FCF000F8F7BAFD80B296490871000A4871487950
:10FD00000979000208434104490C91480171090A2C
:10FD100041718F4948790979000208438C498871FB
:10FD2000000AC8710A2004F093FD0446884908318E
:10FD3000F8F7E8FA86490C318748F8F7E3FA87487C
:10FD4000F8F7C8FA86490390F8F74DFB0490F8F7E6
:10FD50008BFD04467E491031F8F7D4FA7F491439F7
:10FD60004A7C0B7C11021943084679491431F8F793
:10FD7000C9FA7749183100E0E2E00020F8F7C2FA4A
:10FD800009F018FD00127249087709F013FDC1B29D
:10FD90006F484177090A81770CF044FC6C49C91C13
:10FDA0000877000A487706A80AF0C8F96846008B69
:10FDB000404281B2664821300170090A417006A8AC
:10FDC0000AF0CAF968461821415E00290EDA008B54
:10FDD0004042C1B25E482030C170C0780121C903E1
:10FDE0004018C1B25A482030C17005E06846008B07
:10FDF000C1B257482030C1700AA80AF0FBF8544934
:10FE000025310020F8F77EFA00244BE00AA8005DB7
:10FE1000002846D04E482530F8F75CFA00014C49DE
:10FE200025310490F8F76EFA0AA8005D39280DDC38
:10FE300047482530F8F74EFA0AA9095D30390843DA
:10FE4000434925310490F8F75DFA2AE00AA8005DDD
:10FE5000662811DC0AA8005D61280DDB3C482530CE
:10FE6000F8F738FA0AA9095D5739084338492531A6
:10FE70000490F8F747FA14E00AA8005D462810DC61
:10FE80000AA8005D41280CDB31482530F8F722FA3A
:10FE90000AA9095D373908432D4925310490F8F73F
:10FEA00031FA641C0A2CB1DB0AF03CF928492031F4
:10FEB000487203A8FEF7E2FD04990398099108909F
:10FEC00008A8017822482030817408A84178204889
:10FED0002030C17408A881781D48203001750221A6
:10FEE0004175022004F00CFC07901D490798F8F7B3
:10FEF0007AFA0490F8F7B8FC044615493631F8F759
:10FF000001FA13493A310020F8F7FCF9672108A8F3
:10FF1000817531210176A12141760321C17712211A
:10FF200081763421C1763E20094901AAC1C20091DF
:10FF30000DA80FC8FFF7ACF901200A49087002E0CC
:10FF400002200849087000200749087011B0F0BD70
:10FF5000144000200000C84228B7000008270020F5
:10FF600000002041B20B0020B10B0020F0B591B091
:10FF700004460D461646012C7ED1002071490870BA
:10FF8000022004F0BDFB0C906F490020F8F7BAF98D
:10FF90006E490C98F8F727FA0490F8F765FC0746C5
:10FFA0006949091FF8F7AEF902A812F091FD02A8FD
:10FFB00007C809AB07C36946888C0A21F8F7C0F85F
:10FFC0006149091F08720CF02DFB5F49091F487237
:10FFD000000A88726846018D5B48001FC172090AD9
:10FFE00001736846408D5849091F48730FA80DF0EA
:10FFF000E7FE10A840785449091F887310A80178BB
:020000040001F9
:100000005148001FC17308A8817F4F48001F017429
:1000100008A8417F4C48001F417408A8017F4A4846
:10002000001F817403A8FEF729FD049903980E911F
:100030000D9008A8007D4449091FC87408A8417D97
:100040004148001F017508A8817D3F48001F417588
:1000500002218175092019F00DFC3B49091F897D9A
:1000600008433949091F88750A20FEF7F3FC00028E
:10007000010E3548001F00E02DE001760A20FEF752
:10008000E9FC000E3049091FC87510F04FF907460A
:10009000F8F7EAFB81B22C48001F4176090A817605
:1000A0009A2168468175022101761021417603214B
:1000B000C177562181767821C1761B202249091FFC
:1000C00001AA61C2009105A80FC8FFF7E1F801205D
:1000D0001F49087030E0032C10D11A48007801281D
:1000E00008DA18480078401C1649087001201849A1
:1000F000087021E00220164908701DE0F12C14D18F
:100100001448007D002808DD0AF046F8002804D0D5
:100110000021012009F012FD03E032210D488A3050
:10012000417002200A49087006E00021012009F010
:1001300005FD02200649087000200749087011B02B
:10014000F0BD0000B50B002056400020000020410B
:10015000B40B0020A4260020B30B0020F0B589B01A
:1001600004460D461646FB480078152877D00CDC6F
:10017000022875D004DC002810D0012871D1C9E014
:100180000A286FD01428F9D183E11E286BD01F28CC
:100190006AD0202869D02128F0D18EE2012C21D10B
:1001A0000020ED490870ED490870ED48C07920281D
:1001B00002DB0021EA48C171E948C079002803D177
:1001C0001F21E748817105E0E548C079401EC1B2B2
:1001D000E3488171012104201AF03AFE0120DD4933
:1001E000087096E0022C4CD1DB480078012827D11A
:1001F0000FF074FF012102201AF02AFE0020D749D7
:100200000870D7482C38C07955280ED10F20FEF73A
:1002100021FC0004000EAA2803D11E20CD4908703D
:1002200077E00A20CB49087073E00021012009F033
:1002300085FC0220CB4908700020C649087068E0A0
:10024000C54800780A2811D1012102201AF000FEC9
:100250000020C24908700A20BE49087059E095E1A3
:1002600074E03DE2BAE0CFE1DBE1EFE1BA480078CB
:100270001E284ED10020B94908702120B5490870C8
:1002800047E0032C03D11520B249087041E0F12C5E
:1002900039D1B348C079202802DB0021B048C171B0
:1002A000AF48C079002803D11F21AD48817105E016
:1002B000AB48C079401EC1B2A9488171FFF73AFC32
:1002C000072803D0FFF736FC012804D10121084696
:1002D0001AF0BEFD10E0FFF72DFC002806D1012129
:1002E00008461AF0B5FD0FF0E1FE05E0FFF722FC2D
:1002F000032801D10FF0DAFE02209A49087000208D
:100300009449087005E00220964908700020914940
:100310000870ECE194480078002816D1FCF7D6F973
:10032000002812D08E4989799B2251430122520321
:10033000891888B28D4B9B228D49FCF7E5FB012083
:1003400085490870022083490870D0E1FCF7BEF9A6
:10035000002842D001200DF0E7FC002836D080486C
:10036000A43881798348C1767D48A438C179814811
:100370001B3041707A48A438017A7E481B30817066
:1003800008A881787B481B30C17008A8417879485B
:100390001B30017108A8017876481B30417120217B
:1003A000817108A80DF0FAFC07A804F04BFA0020B0
:1003B00005E007990A5C6E499B310A54401CC0282D
:1003C000F7DBFF2063306C49088002E09B206A491C
:1003D000088014205F49087000BF88E167480078F2
:1003E000002855D1FCF772F9002851D000205F4950
:1003F0000870FF215A488171C7790CE05848801C69
:10040000F7F768FF0121B9400840002802D054489E
:10041000877102E07F1E002FF0DA00BF504880791C
:10042000FF2814D11F270CE04D48801CF7F752FF1E
:100430000121B9400840002802D04948877105E0F1
:100440007F1E4748C079401EB842EDDB00BF4448DC
:100450008079FF2806D102204249087000203D49DA
:10046000087015E03E4989799B22514301225203CD
:10047000891888B23D4B9B223D49FCF745FB9B20E8
:100480003D4908800A203449087014203149087019
:100490002DE1FCF71BF900285BD00F20FEF7DAFAFC
:1004A000C0B2AA282AD19A20354988700220087142
:1004B000102048710320C87232480088401C31491E
:1004C0000880084600782E4988712E48008800125E
:1004D000C8711B202849088012F04AFD2648008870
:1004E00029490D2201AB61C30091254905A8F7F701
:1004F000B1FE05A80FC8FEF7CBFE24E06720204917
:10050000887043200871A12048710320C8721D48DB
:100510000088401C1B4908800846007818498871EB
:10052000184800880012C8711348008810490D222D
:1005300001AB61C30091124905A8F7F78BFE05A82E
:100540000FC8FEF7A5FE01200649087000200149EA
:100550000870CCE0080C00200D0C00200C0C0020D2
:10056000E4260020090C0020110C0020F40B0020D0
:10057000C5440020054600200A0C00201C0C002069
:10058000A9440020060C0020894700205948007823
:10059000012810DA57480078401C56490870564820
:1005A00000781E2803D12020544908702BE0142025
:1005B0005249087027E05048007801281DD1FFF704
:1005C000B9FA072803D0FFF7B5FA012804D10121B1
:1005D00008461AF03DFC10E0FFF7ACFA002806D1FF
:1005E000012108461AF034FC0FF060FD05E0FFF72A
:1005F000A1FA032801D10FF059FD022040490870EB
:1006000000203E49087072E0FCF760F8002807D02F
:100610001E20394908700EF0B7FD1F2037490870B9
:1006200065E00EF023FF0FF019F801280DD13548D1
:100630000078002803D020203049087005E002200F
:100640002F49087000202D49087050E0FCF73EF853
:10065000002831D09B202C4988700120087110207F
:1006600048710320C87229480088401C2749088027
:100670000846007824498871244800880012C8710F
:10068000204800780C214843401C21490880084636
:10069000008820490D2201AB61C300911A4905A8C9
:1006A000F7F7D8FD05A80FC8FEF7F2FD01201449A1
:1006B000087000201149087019E0FCF707F80028BD
:1006C0000DD0154915480068F7F71CFE144B06229B
:1006D000C2211148FCF75EFA1E200849087006E0A6
:1006E00002200749087000200449087000BF00BFBD
:1006F00009B0F0BD0C0C00200D0C0020080C0020EF
:10070000090C0020100C0020A9440020060C002039
:100710000A0C0020A4470020E6260020200C002020
:10072000F40B0020012003490870002002490870E2
:1007300070470000B10B0020B20B002000200249DE
:100740000870024908707047080C0020090C00204E
:10075000014800687047000098070020FEB500249B
:100760000026FE480078002802D001287ED10BE048
:1007700000F010FEFA49086008460068042802D01C
:100780000120F6490870C6E2F5480078C007C00F9E
:1007900000286CD00020F349087100F015FE0020FD
:1007A000F14908700B2019F0BDF802A800F018FEFE
:1007B00001A803F06FFF684603F088FF002432E2CF
:1007C000A00002990858A100E84A5050A0000199E1
:1007D0000858A100E64A5050A000009A115820463F
:1007E0000FF070FFA000E149085C0006A100DF4A9D
:1007F0005158FF221202114009020843A100DB4AAE
:100800005158FF2212041140090A0843A100D74A97
:100810005158090E0843A1005050FAF747FF01282C
:1008200008D1D448F7F756FDA100D04A51584018D6
:10083000A1005050A000CE490858012109060840E7
:1008400088427DD1A000C9490858C00FC0070121C6
:10085000C907884215D1A000C44908584000400883
:10086000A100C24A5050A000114601E052E204E249
:100870000858C043401CA10050500A2019F052F8FB
:1008800002E0172019F04EF8A000B84908580028D7
:1008900004D0A0000858B84988420CD9A000B34938
:1008A00008580121C907884209D3A000AF49085858
:1008B000B249884203D84D2019F034F836E0A00040
:1008C000AA490858AD49884209D9A000A749085843
:1008D000AB49884203D8072019F024F826E0A0008D
:1008E000A2490858A649884211D9A0009F49085832
:1008F000A44988420BD8A0009C49085840004008F1
:1009000001218904081AA100984A50500EE0002CD9
:1009100005D19648C06BA100944A505006E0601E75
:10092000800092490858A100904A5050A1008F4A77
:1009300050580EF035FC212018F0F4FF162000E08E
:1009400010E018F0EFFF582018F0ECFF0020854968
:10095000487088700870C87000F028FD012000F011
:1009600025FDF7E0A000824908580121C90608408A
:10097000884238D17B484078102804DB0020A10051
:100980007A4A505013E077484078401C75494870C7
:10099000002C05D17548C06BA100744A505006E088
:1009A000601E800071490858A100704A5050A10093
:1009B0006E4A50580EF0F4FB022018F0B3FF1720D7
:1009C00018F0B0FF4D2018F0ADFF00206549087009
:1009D000C870212018F0A6FF002000F0E7FC0120DD
:1009E00000F0E4FCB6E0A000614908580121490686
:1009F000084088423AD15B488078102804DB002008
:100A0000A1005A4A505013E056488078401C55497E
:100A10008870002C05D15548C06BA100534A505036
:100A200006E0601E800051490858A1004F4A50500E
:100A3000A1004E4A50580EF0B3FB082018F072FF88
:100A4000212018F06FFF022018F06CFF172018F01B
:100A500069FF4D2018F066FF002042490870C870F9
:100A600000F0A4FC012000F0A1FC73E0A0004049CC
:100A7000085801218906084088421DD1394800786C
:100A8000401C384908700846007803280EDC002C0A
:100A900005D13648C06BA100344A505006E0601EB4
:100AA000800032490858A100304A5050A1002F4A16
:100AB00050580EF075FB4DE0A0002D49085801215B
:100AC00049070840884204D0A00029490858002856
:100AD00029D1032018F026FF2248C078401C214964
:100AE000C870002C05D12148C06BA1001F4A50508E
:100AF00006E0601E80001D490858A1001B4A5050A6
:100B00001848C078102808DB00201649C870FDF787
:100B1000D1F9012801D100F069FCA100134A505815
:100B20000EF03EFB16E0212018F0FCFE002C05D153
:100B30000E48C06BA1000D4A505006E0601E8000B8
:100B40000A490858A100094A5050A100074A5058C4
:100B50000EF026FBA0000649085815E039030020D6
:100B60003003002071030020CA03002084170020F6
:100B7000C41700204A1A0020333303000701008005
:100B8000CCCC008000000480012109070840884285
:100B900044D1092018F0C6FE701CC6B2102E09D12F
:100BA000002405E00120A1005C4A5050601CC4B242
:100BB000102CF7DB002C15D15848C06B0121C90758
:100BC00088420AD85548C06B5549884205D35348D6
:100BD000C06BA100514A505023E00120A1004F4AB0
:100BE00050501EE0601E80004C4908580121C90782
:100BF00088420ED8601E80004849085848498842FB
:100C000007D3601E800045490858A100434A505050
:100C100007E00120A100414A505002E0632018F093
:100C200081FE601CC4B2102C00DAC9E504F0D6F9CC
:100C30000220FEF7DDFF07463A49F7F763FB032082
:100C4000FEF7D6FF074637490C31F7F75BFBFEF797
:100C500095FD3448F7F73EFB07463349F7F752FB5B
:100C600030480C30F7F736FB07462F490C31F7F7C1
:100C700049FB00202D4908704BE02D4800680221F7
:100C80000840022845D12B480079401C29490871A9
:100C900000F09AFB00F078FB05462648007905280D
:100CA0000BDB05202349087140211C48F7F7EBFABC
:100CB00040212148F7F7E7FA19E0002410E0002C62
:100CC00005D11648C06BA100144A505006E0601EC2
:100CD000800012490858A100104A5050601CC4B24C
:100CE000102CECDBA1000D4A50580EF059FAE80721
:100CF000C00F002803D0012018F014FE06E00220E7
:100D00002840022802D1012018F00CFE00200749DB
:100D1000087000E000BF00BFFEBD00008417002087
:100D200066660000941900204C1900203903002049
:100D30003003002071030020C417002010B5344890
:100D40000078002802D001285FD14CE00120FDF797
:100D500077FE012846D1FDF785FE002405E000203E
:100D6000A1002C4A5050601CC4B2102CF7DB2A4A58
:100D700000200146F7F7CFFA28490020F7F7C2FA1A
:100D80002649091D0020F7F7BDFA25490020F7F78D
:100D9000B9FA2349091D0020F7F7B4FA21490020C8
:100DA000F7F7B0FA00202049086020490860204980
:100DB00008602049086000F043F8FBF787FC002832
:100DC0000DD01D4B1622FF2101311C48FBF7E2FE1E
:100DD00000200F490870FF2018F0A4FD02E0012058
:100DE0000B49087012E0FBF771FC00280CD0124B85
:100DF0001622FF2101311148FBF7CCFE00200449E7
:100E00000870FF2018F08EFD00E000BF00BF10BD8D
:100E1000B1030020841700209D0300203819002012
:100E2000801900207E030020007F0020047F002026
:100E3000087F00200C7F0020F80300202C1A0020DF
:100E400010B577201D490870882048701C480CF0A8
:100E5000B7FF1B480078194988701948417817482E
:100E6000C1701748817815480171154801791348F8
:100E700041711448F7F72EFA04461049891DF7F717
:100E800041FA1048001DF7F725FA04460B490A31CC
:100E9000F7F738FA0B482830F7F71CFA04460749E9
:100EA0000E31F7F72FFA07482C30F7F713FA0446FC
:100EB00002491231F7F726FA10BD00002C1A002063
:100EC000DB03002038190020F8B5B2480078030091
:100ED00013F05BFB090627F9F3F2F1F0EFEEF200F5
:100EE000FBF7F4FB00281BD000240DE0A000AA4A69
:100EF00081180020F7F706FAA000A84A8118002000
:100F0000F7F700FA601CC4B2122CEFDBA44B1622D8
:100F1000A449FF200130FBF7F7FD01209D4908702F
:100F200035E19F480078FBF7C3FB01287ED1FBF732
:100F3000CDFB0128FAD19B480078772877D19948D2
:100F400040788828FAD1984800689849884229D181
:100F5000042197480CF02CFA012806D19148801DF5
:100F6000F7F7B8F99249086005E08E49891D904865
:100F70000068F7F7C7F904218E480CF019FA012828
:100F800006D188480A30F7F7A5F98A49086005E0D4
:100F900084490A3187480068F7F7B4F905207D498C
:100FA000087002E007207B4908707E480E30F7F792
:100FB00091F905468121C905F7F702FD1BD3794850
:100FC0001230F7F787F905468121C905F7F7F8FCD4
:100FD00011D374480E30F7F77DF905467649F7F7D7
:100FE000E5FC08D36F481230F7F774F905467249EB
:100FF000F7F7DCFC0CD26B490E310020F7F782F9D1
:10100000684912310020F7F77DF905206149087021
:101010006448801DF7F75EF905465F49091DF7F73B
:1010200071F960480A30F7F755F901E04AE02AE023
:10103000054659490831F7F765F95A48801DF7F711
:1010400049F905465D49F7F75DF956480E30F7F75F
:1010500041F9054650492C31F7F754F951481230FF
:10106000F7F738F905464C493031F7F74BF94A485C
:10107000001DF7F72FF90746F7F740FC0546504AE1
:10108000F7F749F91EE04D490020F7F73BF9FBF768
:101090001DFB002813D0FFF7D3FE414B1622FF2182
:1010A00001314048FBF776FD03203A49087009E01A
:1010B00056E040E036E025E068E015E003E002207D
:1010C0003449087063E0FBF701FB00280BD0FFF701
:1010D000B7FE334B1622FF2101313248FBF75AFD90
:1010E00003202C49087052E02D480078FBF7E0FA05
:1010F000012806D1FBF7EAFA012802D10720254989
:10110000087044E0FBF7E2FA00280AD0244B1022D2
:10111000FF2107312348801DFBF73CFD03201D49BB
:10112000087034E01520FDF795FC26490860012081
:10113000254908702BE01A480078FBF7B9FA012816
:101140000DD1FBF7C3FA012809D1154B0C221F4919
:10115000FF205130FBF7D8FC08200E49087016E03C
:101160000F480078FBF7A4FA01280ED1FBF7AEFA7E
:1011700001280AD1FAF79AFA002803D11349083155
:10118000F7F7C0F806200349087000E000BF00BF71
:10119000F8BD0000C5030020341900207C19002090
:1011A000E20300202C1A0020147F00206D5C4B3AD3
:1011B000007F0020047F0020000080C03503002055
:1011C0009D03002090030020C6030020421A002047
:1011D00070B559480078002804D001280BD00628A3
:1011E00072D182E0E121090103200CF075FF01209A
:1011F000514908709DE003200CF0A0FD002819D093
:101200000BF0C4FA012815D00320FDF719FC0128C2
:1012100010D04A48007800280CD1FAF741FA01288A
:1012200008D012F0D6FD012804D000200FF0B6F847
:10123000012859D1FBF74AFA002855D000200FF0B9
:10124000B7F803200CF07AFD00282ED13C48F7F7C0
:1012500041F805463B48F7F73DF806462946F7F7BB
:10126000BAF804467F21C9052046F7F7A9FB04D345
:1012700035492046F7F79AFB13D23248F7F72AF898
:1012800005462F49F7F73EF8FFF7DAFD2F4B1622F8
:10129000FF2101312E48FBF77DFC0620264908700E
:1012A00022E00020244908701EE0FAF7F9F901282D
:1012B0000BD1002027490870274B0422FF21593108
:1012C0002648FBF767FC0FE032E000201B4908705E
:1012D000FFF7B6FD1D4B1622FF2101311C48FBF71D
:1012E00059FC06201449087023E0FBF7EFF90028A9
:1012F0001DD0FF2018F016FB0320FDF7A1FB0128ED
:1013000005D10320FDF7AEFB0120154908700BF055
:101310003DFA012803D012F05CFD012804D1012020
:1013200008F058FA13F07CF900200349087000E037
:1013300000BF00BF70BD0000C4030020B003002048
:101340006C03002038190020000080BFF903002042
:101350002C1A0020C80300209C0300204A1A0020F9
:10136000C703002010B5074800780A2807DA0548A7
:101370000078401C0349087000F038F801E003F0E1
:1013800033FD10BDCA0300200148007870470000FB
:101390008A0200200148007870470000890200207E
:1013A00001480078704700008C020020072800DD0B
:1013B000704701218140034A12788A4301490A702B
:1013C00000BFF5E78A020020042001490870704739
:1013D0008902002000200149087070478C0200201B
:1013E0000149016070470000C813002010B5FEF7E6
:1013F00047F8FEF7B7F800200F4908600F4908606A
:101400000F4908700F4908700F4908700F4908709C
:101410000F4908700F4908700F4908700F4908708C
:101420000F4908600F4908600F4908600FF010F974
:101430000B49086010BD00007C02002080020020E3
:1014400084020020850200208602002087020020FE
:10145000880200208D0200208B0200208C020020D8
:10146000980200209002002094020020F8B5044663
:10147000002C0AD00120C004844202D317488442C1
:1014800003D9062018F04EFA02E0422018F04AFA7A
:10149000002C07D001208004844203D2042018F0DD
:1014A00041FA02E02C2018F03DFA0EF03FFF07460B
:1014B0000B493846F7F784FA08D33846F7F71EFA8F
:1014C00005460022074BF7F72DFA03D2052018F046
:1014D00029FA02E0372018F025FAF8BD00000514BB
:1014E00000005C420000E0BFF0B589B00025002795
:1014F00000261720FDF7AEFAFE490860084600688E
:1015000003F019FAFC490860084601680020F6F764
:1015100062FFFA49086000242DE0A000F84908584D
:101520000121C90788421CD3A000F5490858400092
:101530004008A100F24A5050A100505803F0FBF9B6
:1015400000210790F6F74BFFA100EE4A5050A00093
:10155000EB4908580121C9070843A100E84A505047
:1015600007E0A100E64A505803F0E5F9A100E54A7A
:101570005050601CC4B2102CCFDB05F081F90A2852
:1015800073D10020E04908701021DE48FBF7F4FC1D
:101590000646DE48066000213046F7F707FA08D213
:1015A0000A20DB49087031460020F6F714FF064692
:1015B00002E00120D64908703046FDF785F9089011
:1015C000089800F0B3FA07463846FDF77DF9D1498F
:1015D0000690F6F797FECF48F6F77CFECE490690C8
:1015E000F6F790FECB48F6F775FE0690FFF73EFF44
:1015F000CA48407901280BD1C9480078401CC84925
:10160000087008460078F02805DB0020087002E02A
:101610000020C3490870C048F6F75CFE002805D0DA
:10162000162018F07FF9582018F07CF9384608F099
:1016300005F90746384601F0D7FB39460020F7F791
:10164000B5F97DD0B748007800280FD1B6480068BA
:10165000F7F7E1F8432109060590F6F701FF39464F
:101660000690F6F7C0FE054612E08EE1AF49384617
:10167000F6F7B9FE0746AC480068F7F7CCF83946EC
:101680000590F6F7B0FEAA490690F6F7E9FE054682
:10169000A8492846F6F7A7FEA7490690F6F7E0FE08
:1016A0000546A6492846F6F7DBFE05469848007829
:1016B000012813D1A248F6F717FE0391029028469D
:1016C000F7F71CF901910090039B029AF6F706FFC9
:1016D0009B4A05910490F6F71EFEE0E01620FDF708
:1016E000B9F9984988423BD19548F6F7FDFD059137
:1016F00004902846F7F702F903910290059B049A9B
:10170000F7F724F905D88E4A00200146F6F703FEC4
:1017100012E08B48F6F7E8FD039102902846F7F7B0
:10172000EDF801910090039B029AF6F781FF844A3D
:1017300005910490F6F7EFFD8148F6F7D5FD00E03E
:10174000A7E005910490F7F715F973490839069059
:10175000F6F7D8FD70480838F6F7BCFD7A490860FE
:101760006D48001FF6F7B6FD78490690F7F728F99F
:1017700021D2294676480068F6F7DCFD74490860F6
:101780006C4973480068F7F71BF97BD269497048C8
:101790000068F6F720FE6E4908605F48001FF6F704
:1017A00099FD64490590F6F7C5FD5B49091F069050
:1017B000F6F7A8FD66E05848001FF6F78BFD65496F
:1017C0000690F7F7FDF821D2294661480068F6F740
:1017D000B1FD5F49086060495D480068F7F7F0F8BF
:1017E00050D25D495A480068F6F7F5FD584908603F
:1017F0004948001FF6F76EFD57490590F6F79AFD28
:101800004549091F0690F6F77DFD3BE04248001F61
:10181000F6F760FD4649A0390690F7F7D1F824D2D3
:1018200029464B480068F6F785FD494908607F2145
:10183000C90547480068F7F7C3F823D27F21C905D7
:1018400043480068F6F7C7FD414908603248001F69
:10185000F6F740FD7F21C9050590F6F76BFD2E498F
:10186000091F0690F6F74EFD0CE02B48001FF6F717
:1018700031FD29460590F6F75DFD2749091F0690C1
:10188000F6F740FD2448001FF6F724FD33490860B1
:1018900005E02148001FF6F71DFD304908603A4673
:1018A0001B480178284612F017FD0790012189078F
:1018B0000798F7F785F805D3032189070798F7F705
:1018C00075F801D2002007901D48F6F70DFD039131
:1018D00002900798F7F712F801910090039B029A83
:1018E000F6F7FCFD164A05910490F6F714FD14482E
:1018F00036E00000580300205C0300206003002055
:1019000084170020EC19002070030020B40300208D
:10191000A50300208819002040190020D8190020B4
:10192000CB030020C0030020D4030020643B7F3F92
:10193000002474490000C8420000614500007A4458
:101940009D0300203C4D0000007F0020A3BBBE4C47
:10195000A80300207696184B00002041047F002049
:10196000F6F7C2FC05910490F7F704F85C4906907D
:10197000F6F7C8FC5A48F6F7ADFC5A4908605A48D1
:1019800005605A485A490860A7E05A48007801287B
:1019900004D100205749087019F092FA10215648D6
:1019A000FBF7EAFA06465548066000213046F6F78E
:1019B000FDFF00D200263046FCF786FF089008980D
:1019C00000F0B4F807463846FCF77EFF4C49086043
:1019D0004C48407901280BD14B480078401C4A49BB
:1019E0000870084600780F2805DB0020087002E028
:1019F000002045490870384607F020FF0746384662
:101A0000FAF772FC384601F0EFF939460020F6F794
:101A1000CDFF51D0162017F085FF582017F082FF18
:101A20003A480068F6F7F7FE432109060590F6F7F5
:101A300017FD39460690F6F7D6FC35490790F6F7BC
:101A40000FFD05463348F6F745FC29460690F6F7A4
:101A500071FC30490790F6F755FC2F48F6F744FC27
:101A6000059104902D492846F6F7FAFC0190F6F707
:101A700045FF03910290059B049AF6F72FFD264A35
:101A800007910690F6F747FC2348F6F72DFC0591E1
:101A90000490F6F76FFF12490790F6F733FC1D48E4
:101AA000F6F718FC1E4908601E4805600C48F6F75A
:101AB00011FC0C4908600DE00948F6F70BFC0949D8
:101AC00008600748001DF6F705FC1749086000206C
:101AD0001449086005480649086009B0F0BD0000D7
:101AE00038190020007F0020187F00206D5C4B3AE1
:101AF000147F002045030020EC190020B4030020CF
:101B00003C030020D8190020CB030020D403002080
:101B100000001042801900209D03002000007A443C
:101B2000087F00200C7F0020047F002001B59CB0BE
:101B300000201B901A9019901C9812F031FA052081
:101B40000CF0F2F8002811D005200CF01DF9FD482A
:101B50000068FD49884203D90120FC49087002E071
:101B60000020FA4908700020F6490860F8491C98DE
:101B70000968884204D3012189041C98884202D351
:101B800000201B90F5E3EF480068401CED49086019
:101B90001C9802F0D0FE1A90EE491A98F6F723FC32
:101BA0001A90F9F783FD01281AD1EB480068401C10
:101BB000E949086004200CF0B7F8002813D004208D
:101BC0000CF0E2F8E4480068DF49884204D902F0EA
:101BD000BDFE0120E14908700020DF49086002E0F5
:101BE0000020DD490860DE480078002803D0DD4889
:101BF0000068199002E00EF099FB19901998F6F719
:101C00007DFE0022D84B17911690F6F78BFE0CD272
:101C1000D648F6F75FFB5F2807D9D4480C30F6F7B3
:101C200059FB5F2801D9D24819900BF063FCD149C8
:101C30000860D1481A99F6F7D6FB15901A99F6F76D
:101C4000D2FB1790CD481999F6F7CDFB13901A994E
:101C5000F6F7C9FB1590CA481999F6F7C4FB11901D
:101C60001999F6F7C0FB1390C6481A99F6F7BBFB13
:101C70001190C5481999F6F7B6FBC4490F90F6F7CD
:101C800059FB10901199F6F755FB12901399F6F73E
:101C9000A2FB14901599F6F74DFB16901799F6F7DD
:101CA00049FB1890BA491898F6F780FE7ED80021B3
:101CB0001998F6F77BFE04D3B6491998F6F780FE1B
:101CC00003D2B548006D179028E01998F6F7CCFDBF
:101CD000C0B215901598F6F79EFD0D901999F6F77C
:101CE0007EFB149015988000AB4908580B9015980E
:101CF000401C800008580A900B99F6F76CFB0C907A
:101D00001499F6F770FB0D9015988000A2490858B9
:101D100001460C900D98F6F70DFB179017990846A1
:101D2000F6F761FB0C901A99F6F75DFB9B490D9055
:101D3000F6F759FB13901998129000211998F6F7AD
:101D400035FE02D20020129006E095491998F6F768
:101D500037FE01D29248129092481299F6F743FB4F
:101D60000C9091481299F6F73EFB08901299F6F7FD
:101D70003AFB0A908D481299F6F735FB07901299B5
:101D8000F6F731FB08901299F6F72DFB09900A99A6
:101D9000F6F7D0FA0B900C99F6F71DFB84490D90DD
:101DA000F6F7C8FA11908348129900E0EAE1F6F7D5
:101DB0001AFB0B9080481299F6F715FB09901299BF
:101DC000F6F711FB0A900B99F6F7B4FA7B490C90E1
:101DD000F6F7B0FA7A490D90F6F705FB10907848BF
:101DE0001099F6F700FB0B901399F6F7FCFA75497A
:101DF0000C90F6F7F8FA0D901199F6F731FB0F9069
:101E000071491398F6F7EFFA1B906D490F98F6F7A2
:101E100027FB0E906D490E98F6F7C8FD55D26C4819
:101E20000E99F6F7E0FA0C906A480E99F6F7DBFA8D
:101E300008900E99F6F7D7FA0A9067480E99F6F7C8
:101E4000D2FA05900E99F6F7CEFA06900E99F6F7AB
:101E5000CAFA089061480E99F6F7C5FA02900E99F1
:101E6000F6F7C1FA03900E99F6F7BDFA04900E99B1
:101E7000F6F7B9FA06905A480E99F6F7B4FA0190B7
:101E80000E99F6F7B0FA02900E99F6F7ACFA0390B5
:101E90000E99F6F7A8FA04900E99F6F7A4FA0590B1
:101EA0000699F6F798FA07900899F6F743FA099019
:101EB0000A99F6F790FA0B900C99F6F73BFA494914
:101EC0000D90F6F737FA169051E147490E98F6F75C
:101ED0006DFD36D245480E99F6F785FA0C904448C8
:101EE0000E99F6F780FA08900E99F6F77CFA0A90A8
:101EF00040480E99F6F777FA05900E99F6F773FABF
:101F000006900E99F6F76FFA08903B480E99F6F78F
:101F10006AFA02900E99F6F766FA03900E99F6F7B0
:101F200062FA04900E99F6F75EFA069033480E991D
:101F3000F6F759FA01900E99F6F755FA02900E99B4
:101F40005EE07DE0F0030020B8A10000C90300209E
:101F50005803002000007A43EC030020C80300204F
:101F600052030020540300200000E0BF4C19002061
:101F70000000A041CC0300208109DC3C6EDD4D3D1A
:101F800028EF633BC3F504412506413EB29D8BC05B
:101F9000000002430000C842F8BF0200228C0A324F
:101FA00000005C4223DB5C421A516A3FA69BC4BB23
:101FB0006606DF443B4A5B372684B3B64703803F5F
:101FC00000007A4400006041688B0A44CDCCAC40EC
:101FD0004B75013D61E28F3C1A53B03B3EF4553ADC
:101FE000E93A4938C009653F00004842643B043B78
:101FF0005762D838451E4D3632CE46330689982F63
:10200000F6F7F1F903900E99F6F7EDF904900E99B1
:10201000F6F7E9F905900699F6F7DDF907900899C2
:10202000F6F788F909900A99F6F7D5F90B900C990B
:10203000F6F780F9FE490D90F6F77CF9169096E0D8
:10204000FC490E98F6F7B2FC55D2FB480E99F6F70C
:10205000CAF90C90F9480E99F6F7C5F908900E994F
:10206000F6F7C1F90A90F6480E99F6F7BCF9059013
:102070000E99F6F7B8F906900E99F6F7B4F90890AC
:10208000F0480E99F6F7AFF902900E99F6F7ABF912
:1020900003900E99F6F7A7F904900E99F6F7A3F9B5
:1020A0000690E9480E99F6F79EF901900E99F6F719
:1020B0009AF902900E99F6F796F903900E99F6F7B1
:1020C00092F904900E99F6F78EF905900699F6F7B5
:1020D00082F907900899F6F72DF909900A99F6F711
:1020E0007AF90B900C99F6F725F9D8490D90F6F787
:1020F00021F916903BE0D6480E99F6F774F90C904A
:10210000D4480E99F6F76FF908900E99F6F76BF927
:102110000A90D1480E99F6F766F905900E99F6F7F0
:1021200062F906900E99F6F75EF90890CB480E9981
:10213000F6F759F904900E99F6F755F905900E99AE
:10214000F6F751F906900E99F6F74DF907900899B0
:10215000F6F7F0F809900A99F6F73DF90B900C990B
:10216000F6F7E8F8BE490D90F6F7E4F816901699E0
:102170001B98F6F738F91B9019A807C8FAF7FEFD67
:102180001B90EEE3B7491998F6F71AFC7ED2B649D0
:102190001898F6F70BFC7AD2B44800680146139001
:1021A0001A98F6F7C7F81590B048006801461190E4
:1021B0001A98F6F7BFF81390AC48006801461090E3
:1021C0001A98F6F7B7F81190A848806A014610905F
:1021D0001198F6F708F912901399F6F704F914908C
:1021E0001599F6F700F91790A0480068014610907D
:1021F0001A98F6F79FF812909C48006801460F90D5
:102200001A98F6F797F810909848406A01460F9090
:102210001098F6F7E8F811901299F6F7E4F8139091
:102220001999F6F7E0F815909048006801460E906D
:102230001A98F6F77FF80F908C48006A01460E90C6
:102240000F98F6F7D0F810901999F6F7CCF811908E
:102250001999F6F7C8F813908448C0690D90199938
:10226000F6F7C1F80E901999F6F7BDF80F90199985
:10227000F6F7B9F811907D48006801460B901A985E
:10228000F6F758F80D907948006801E07DE171E0BB
:1022900001460A901A98F6F74DF80B90734880693A
:1022A00001460A900B98F6F79EF80C900D99F6F7F8
:1022B0009AF80F906D480068014609901A98F6F751
:1022C00039F80A9069484069014609900A98F6F77A
:1022D0008AF80B901999F6F786F80D906348006913
:1022E00008901999F6F77FF809901999F6F77BF895
:1022F0000B905E480068014606901A98F6F71AF8A7
:1023000007905A48C068014606900798F6F76BF8A0
:1023100009905648806806901999F6F764F8079076
:1023200052484068014606900798F6F703F808906F
:102330000999F5F7FFFF0A900B99F5F7FBFF0C9051
:102340000D99F5F7F7FF0E900F99F5F7F3FF109041
:102350001199F5F7EFFF12901399F5F7EBFF149031
:102360001599F5F7E7FF16901799F5F7E3FF1B901E
:10237000F7E2F3E33D48C06A014613901A98F5F777
:10238000D9FF15903948C06A014611901A98F5F79F
:10239000D1FF13903548C06A014610901A98F5F79E
:1023A000C9FF11903148406D014610901198F6F721
:1023B0001AF812901399F6F716F814901599F6F783
:1023C00012F817902948C06A014610901A98F5F73C
:1023D000B1FF12902548C06A01460F901A98F5F790
:1023E000A9FF10902148006D01460F901098F5F755
:1023F000FAFF11901299F5F7F6FF13901999F5F776
:10240000F2FF15901948C06A01460E901A98F5F728
:1024100091FF0F901548C06C01460E900F98F5F78C
:10242000E2FF10901999F5F7DEFF119019991FE05E
:1024300070256B3F0000C843CB694B39C66FA73589
:102440000D4FA03168681D2DF82DF527CB106F3F7B
:10245000574FED37D96F1233D9FBC82D6F73E1A7F2
:102460004AA1713F00000C4200002A439C07002053
:10247000F5F7B9FF1390FE48806C0D901999F5F7A8
:10248000B2FF0E901999F5F7AEFF0F901999F5F775
:10249000AAFF1190F648C06A01460B901A98F5F70A
:1024A00049FF0D90F248C06A01460A901A98F5F764
:1024B00041FF0B90EE48406C01460A900B98F5F7EF
:1024C00092FF0C900D99F5F78EFF0F90E848C06AC7
:1024D000014609901A98F5F72DFF0A90E448006C20
:1024E000014609900A98F5F77EFF0B901999F5F7C8
:1024F0007AFF0D90DE48C06B08901999F5F773FFCD
:1025000009901999F5F76FFF0B90D948C06A0146F9
:1025100006901A98F5F70EFF0790D548806B014694
:1025200006900798F5F75FFF0990D148406B069039
:102530001999F5F758FF0790CD48006B01460690B2
:102540000798F5F7F7FE08900999F5F7F3FE0A905A
:102550000B99F5F7EFFE0C900D99F5F7EBFE0E9049
:102560000F99F5F7E7FE10901199F5F7E3FE129039
:102570001399F5F7DFFE14901599F5F7DBFE169029
:102580001799F5F7D7FE1B90EBE1BA491898F6F7C3
:102590000DFA7DD2B648806D014613901A98F5F772
:1025A000C9FE1590B248806D014611901A98F5F752
:1025B000C1FE1390AE48806D014610901A98F5F751
:1025C000B9FE1190AA488030006801461090119819
:1025D000F5F709FF12901399F5F705FF1490159977
:1025E000F5F701FF1790A248806D014610901A98E8
:1025F000F5F7A0FE12909E48806D01460F901A9844
:10260000F5F798FE10909A48C06F01460F90109809
:10261000F5F7E9FE11901299F5F7E5FE1390199977
:10262000F5F7E1FE15909248806D01460E901A98DC
:10263000F5F780FE0F908E48806F01460E900F9840
:10264000F5F7D1FE10901999F5F7CDFE1190199973
:10265000F5F7C9FE13908648406F0D901999F5F76C
:10266000C2FE0E901999F5F7BEFE0F901999F5F775
:10267000BAFE11907E48806D01460B901A98F5F7CE
:1026800059FE0D907A48806D01460A901A9800E034
:102690006DE0F5F74FFE0B907548006F01460A900C
:1026A0000B98F5F7A0FE0C900D99F5F79CFE0F9096
:1026B0006F48806D014609901A98F5F73BFE0A9025
:1026C0006B48C06E014609900A98F5F78CFE0B9096
:1026D0001999F5F788FE0D906548806E0890199954
:1026E000F5F781FE09901999F5F77DFE0B9060488A
:1026F000806D014606901A98F5F71CFE07905C481D
:10270000406E014606900798F5F76DFE099058480F
:10271000006E06901999F5F766FE07905448C06D53
:10272000014606900798F5F705FE08900999F5F718
:1027300001FE0A900B99F5F7FDFD0C900D99F5F748
:10274000F9FD0E900F99F5F7F5FD10901199F5F739
:10275000F1FD12901399F5F7EDFD14901599F5F729
:10276000E9FD16901799F5F7E5FD1B90F9E0404853
:1027700080304068014613901A98F5F7DBFD1590FC
:102780003B4880304068014611901A98F5F7D2FD19
:102790001390374880304068014610901A98F5F73A
:1027A000C9FD119032488030C06A014610901198DE
:1027B000F5F719FE12901399F5F715FE1490159977
:1027C000F5F711FE17902A488030406801461090B6
:1027D0001A98F5F7AFFD1290254880304068014601
:1027E0000F901A98F5F7A6FD109021488030806A66
:1027F00001460F901098F5F7F6FD11901299F5F734
:10280000F2FD13901999F5F7EEFD159018488030F8
:10281000406801460E901A98F5F78CFD0F90144809
:102820008030406A01460E900F98F5F7DCFD10905D
:102830001999F5F7D8FD11901999F5F7D4FD139072
:102840000B488030006A0D901999F5F7CCFD0E9079
:102850001999F5F7C8FD0F901999F5F7C4FD119076
:1028600003488030406801460B901A9804E000004D
:102870009C07002000002A43F5F75CFD0D90FC4802
:10288000406801460A901A98F5F754FD0B90F848F5
:10289000C06901460A900B98F5F7A5FD0C900D99BB
:1028A000F5F7A1FD0F90F2484068014609901A988B
:1028B000F5F740FD0A90EE488069014609900A98B4
:1028C000F5F791FD0B901999F5F78DFD0D90E848FE
:1028D000406908901999F5F786FD09901999F5F75F
:1028E00082FD0B90E2484068014606901A98F5F781
:1028F00021FD0790DE480069014606900798F5F72C
:1029000072FD0990DA48C06806901999F5F76BFDD9
:102910000790D7488068014606900798F5F70AFDAA
:1029200008900999F5F706FD0A900B99F5F702FD55
:102930000C900D99F5F7FEFC0E900F99F5F7FAFC47
:1029400010901199F5F7F6FC12901399F5F7F2FC37
:1029500014901599F5F7EEFC16901799F5F7EAFC27
:102960001B90C4491898F6F721F818D8C248006897
:102970008830F5F7AFFC1690BF4800689030F5F747
:10298000A9FC14901B99F5F72EFD15901699F5F7F3
:10299000D1FC17901B99F5F726FD1B9053E0B74922
:1029A0001898F6F703F818D8B34800685C30F5F7C4
:1029B00091FC1690B04800686430F5F78BFC1490D9
:1029C0001B99F5F710FD15901699F5F7B3FC1790C4
:1029D0001B99F5F708FD1B9035E0A9491898F5F704
:1029E000E5FF18D8A44800683030F5F773FC16905E
:1029F000A14800683830F5F76DFC14901B99F5F785
:102A0000F2FC15901699F5F795FC17901B99F5F7C0
:102A1000EAFC1B9017E098480068001DF5F75AFC87
:102A20001690954800680C30F5F754FC14901B99EB
:102A3000F5F7D9FC15901699F5F77CFC17901B99C2
:102A4000F5F7D1FC1B903F2109061998F5F7AEFF69
:102A500002D200201DB000BD8A491998F5F7A6FFE3
:102A60000CD28948F5F736FC5F2805D386480C3030
:102A7000F5F730FC5F2801D20020EBE78349199875
:102A8000F5F794FF06D200201999F5F78FFF01D0D2
:102A90000020DFE7F8F70AFE012806D17C491B98E1
:102AA000F5F784FF01D80020D4E77748F5F712FC4A
:102AB0001590F5F7CBFE0022764B17911690F5F79F
:102AC00031FF0DD370480C30F5F704FC1590F5F785
:102AD000BDFE00226F4B17911690F5F723FF06D22B
:102AE0006D491B98F5F762FF01D80020B2E700217D
:102AF0001B98F5F75BFF01D200201B905F491998E6
:102B0000F5F75EFF3BD865491B98F5F74FFF05D2F7
:102B100063491B98F5F767FC1B903CE15F491B98E4
:102B2000F5F74EFF0AD855491B98F5F73FFF05D238
:102B30005C491B98F5F757FC1B902CE14F491B98FB
:102B4000F5F73EFF0BD858491B98F5F72FFF06D233
:102B500056491B98F5F747FC1B901CE120E15449AE
:102B60001B98F5F72DFFD8D852491B98F5F71EFF93
:102B7000D3D251491B98F5F736FC1B900BE14F4916
:102B80001998F5F71DFF2FD83C491998F5F70EFF56
:102B90002AD245491B98F5F709FF05D248491B98E9
:102BA000F5F721FC1B90F6E041491B98F5F708FF6B
:102BB0000AD844491B98F5F7F9FE05D23E491B98FF
:102BC000F5F711FC1B90E6E03E491B98F5F7F8FE7F
:102BD00009D82B491B98F5F7E9FE04D23A491B980E
:102BE000F5F701FC1B90D6E038491998F5F7E8FE97
:102BF00024D832491998F5F7D9FE1FD227491B98D6
:102C0000F5F7DEFE0AD82A491B98F5F7CFFE05D264
:102C10002B491B98F5F7E7FB1B90BCE029491B9853
:102C2000F5F7CEFE09D816491B98F5F7BFFE04D27A
:102C300021491B98F5F7D7FB1B90ACE02449199864
:102C4000F5F7BEFE58D821491998F5F7AFFE53D2D3
:102C500012491B98F5F7B4FE3ED81E491B98F5F7AC
:102C6000A5FE39D216491B98F5F7BDFB1B9092E0E3
:102C70001C08002000007041CC030020000004422A
:102C8000000002430000A0404C190020CDCCCC3DF8
:102C90006666664100006340CDCC4C410000E041D7
:102CA0001283803F60E5803F000010428941803FF1
:102CB000000018420000BE42DBF97E3F3333EF4193
:102CC0004E62803F00008242643B7F3F0000C4416F
:102CD00014AE934100002C4236491B98F5F770FE64
:102CE00059D835491B98F5F761FE54D233491B98E2
:102CF000F5F779FB1B904EE031491998F5F756FE30
:102D000049D230491B98F5F751FE05D22E491B9840
:102D1000F5F769FB1B903EE02A491B98F5F750FE3A
:102D20000AD82A491B98F5F741FE05D228491B9875
:102D3000F5F759FB1B902EE024491B98F5F740FE50
:102D40000AD81C491B98F5F731FE05D221491B987A
:102D5000F5F749FB1B901EE01F491B98F5F730FE65
:102D60000AD815491B98F5F721FE05D213491B987F
:102D7000F5F739FB1B900EE00F491B98F5F720FE85
:102D800009D816491B98F5F711FE04D214491B986F
:102D9000F5F729FB1B901B9817F058FB1B9000BF01
:102DA00010491B98F5F70CFE01D20E481B901B989A
:102DB00050E600000000824200000243DBF97E3F43
:102DC00014AE93410000E041EE7C7F3F00004042A2
:102DD0004E62803FD7A3803F0000964200800944A6
:102DE000643B7F3F0060EA45F0B585B004460027AC
:102DF0000020039002900190FBF75CF8002802D1BC
:102E000001209749087097480078002806D00128CB
:102E100023D002282AD0032871D111E100212046B5
:102E2000F5F7C4FD18D003F02BFD0A2805D18E4814
:102E3000F5F750FA8D49086004E08D48F5F74AFA35
:102E40008A49086003210C200BF046F900208449D0
:102E50000870012083490870FFE00C200AF06EFF23
:102E6000002802D102207F490870F6E000212046A8
:102E7000F5F79CFD7ED103F003FD0A287BD17A484B
:102E8000F5F728FA0546794801682846F5F7A3FAC8
:102E900007463F2109063846F5F79DFA03907F2142
:102EA000C9053846F5F797FA029072493846F5F7A2
:102EB00092FA019070490298F5F782FD20D86F4987
:102EC0000298F5F773FD1BD86748F5F703FA064635
:102ED0006B490298F5F787FA31460090F5F77FFACB
:102EE00005466149F5F70EFA5F48F5F7F3F90090EA
:102EF000F5F704FD0546634AF5F70DFA9AE0A8E0F8
:102F000061490398F5F75CFD1FD860490398F5F710
:102F10004DFD1AD85448F5F7DDF90646584903988F
:102F2000F5F761FA31460090F5F759FA05464E4932
:102F3000F5F7E8F94C48F5F7CDF90090F5F7DEFC28
:102F40000546504AF5F7E7F974E051490198F5F75D
:102F500037FD6FD84F490198F5F728FD6AD84048EA
:102F60000078012866D14048F5F7B4F906464A4989
:102F7000019801E063E014E0F5F735FA314600907E
:102F8000F5F72DFA05463849F5F7BCF93648F5F757
:102F9000A1F90090F5F7B2FC05463A4AF5F7BBF9FE
:102FA00048E03348F5F796F9054630480168284669
:102FB000F5F711FA074639493846F5F70CFA039048
:102FC00037493846F5F707FA029036490298F5F77F
:102FD000F7FC15D834490298F5F7E8FC10D82448D6
:102FE000F5F778F9064626490298F5F7FCF93146D7
:102FF0000090F5F7F4F905461D49F5F783F919E056
:103000002A490398F5F7DCFC14D829490398F5F709
:10301000CDFC0FD81648F5F75DF906461849039818
:10302000F5F7E1F931460090F5F7D9F90546104971
:10303000F5F768F900200A4908700A4908700CE0A1
:1030400000212046F5F7B2FC02D1002005490870A6
:1030500003E000200349087000BF00BF05B0F0BDC9
:10306000E8030020E303002038190020E4030020D7
:103070008019002000002041295C0FBD295C0F3D14
:10308000CDCC4C3E9D030020295C8FBC295C8F3C3D
:10309000CDCC4CBFCDCC4C3F9A99593F0000FA4360
:1030A00000007A4400000CC200000C4200008CC1F9
:1030B00000008C4103480078012800D170470020AF
:1030C000FCE700008D02002010B5FCF7D9F9FCF7F1
:1030D00049FA00201549086015490860154908702B
:1030E0001549087015490870154908701549087088
:1030F000154908700420154908700020144908700B
:10310000144908701449087014490860144908608B
:10311000144908600DF09CFA104908601920FBF76B
:1031200099FCC1B21048C17010BD00007C020020A3
:1031300080020020840200208502002086020020F8
:1031400087020020880200208D02002089020020D2
:103150008A0200208B0200208C02002098020020AE
:1031600090020020940200209A000020F8B500266A
:103170000024FE480078232801D301F000F8430022
:103180007B449B885B009F4422005100A100F60015
:1031900012012F015603D803FA0341045E047E0492
:1031A000CB042706DF060607AF07FA07C407E207C6
:1031B0004E016A018A01DA01FA07DD00E70407051A
:1031C0005705B7050A06D4021D0375069506E8499A
:1031D00001200006F5F796F8E5481C38C07810285D
:1031E00003DD1021E2481C38C170E2480078012854
:1031F00002D10020DF4908700DF02AFADE4908608C
:103200000120DA490870DD4908700020DC490870A7
:10321000DC4908700120DC4908600020DB490860B7
:10322000DB48DC490860FCF775F9C4E34E20FBF786
:1032300007FC00282AD00DF00BFACF490968401A84
:10324000D549884241D94E20FBF70CFCCC48007888
:1032500001283AD10DF0FCF9C74908600020C8499F
:1032600008700220C14908700120C449087002207A
:10327000C54908600420C5490860C848C5490860B8
:10328000C748C8490860FCF745F91EE0BC4800780B
:1032900001281AD10DF0DCF9B74908600020B849BF
:1032A00008700220B14908700120B449087002205A
:1032B000B54908600420B5490860B848B5490860B8
:1032C000B748B8490860FCF725F9AEE7AD48007883
:1032D000012836D10020AB490870B148C078B24906
:1032E0004870084640780421084004280AD100208C
:1032F000AE4908600DF0ACF99F49086019209B4960
:1033000008701EE0A9480068401CA84908600846EB
:103310000068FF212D3188420ED90020A3490860A2
:103320000220A3490870A348007801210843A1495D
:103330000870FEF717F804E00120914908708B49E6
:10334000087072E700208E490870032087490870D2
:1033500001208A4908700DF07BF987490860062032
:1033600089490860002089490860934889490860B4
:10337000FCF7D0F859E782480078012816D10020E0
:103380007F4908700DF064F97B4908600420774993
:1033900008700120794908707B49086000207B494A
:1033A000086086487B490860FCF7B4F83DE774483C
:1033B0000078012817D10DF04BF96F490860002003
:1033C0006F49087005206949087001206B49087031
:1033D00006206D49086000206C49086078486D49F6
:1033E0000860FCF797F820E765480078012819D1B4
:1033F0000DF02EF960490860002061490870142022
:103400005A49087001205D49087006205E4908602D
:1034100000205E4908606B4908706B485D49086090
:10342000FCF778F801E756480078012816D100200B
:103430005349087015204D4908700DF009F94E499F
:10344000086001204D4908704F49086000204F492D
:1034500008605E484F490860FCF75CF8E5E64848BC
:10346000007801281AD10DF0F3F8434908600020D4
:103470004349087016203D49087001203F490870F3
:1034800002204149086004204049086043484149FE
:103490000860434843490860FCF73CF8C5E63948F2
:1034A000007801284AD10020364908703C48C0788D
:1034B0003D49C8700846C0780821084008281DD139
:1034C00000203A4908602E4908700DF0C1F82A49D9
:1034D000086017202549087001202849087002203B
:1034E00029490860042029490860394829490860A9
:1034F0002B482C490860FCF70DF81FE02B480068AA
:10350000401C2A49086008460068FF212D31884286
:103510000ED9002025490860022025490870254859
:1035200000780121084323490870FDF71BFF05E0DF
:1035300001201349087015200C49087075E61148E0
:10354000007801287DD100200E4908700C490870D0
:103550000DF07EF808490860114800781249C870DB
:103560000F48407888700E48807833E0850200204C
:10357000B60000208B020020980200208602002066
:103580008802002087020020800200207C020020A8
:1035900050B802006402002050C3000022B80200AC
:1035A0006C020020680200205C00002090020020D5
:1035B000890200208A0200200AB8020051B80200E5
:1035C00010B802007802002016B8020054B80200B9
:1035D0003EB802004870F848C078087000201AE031
:1035E000014609318900F54A525C014609318900DA
:1035F000F24BC91849785218014609318900C91897
:1036000089785218014609318900C918C9785118BA
:103610000C19411CC8B21028E2DB2106FF2212025D
:10362000224012021143FF2212042240120A1143C7
:10363000220E11430846E249F4F764FE00240020FC
:103640001BE075E001464F318900DC4A525C0146BF
:103650004F318900D94BC9184978521801464F316A
:103660008900C9188978521801464F318900C91854
:10367000C97851180C19411CC8B22E28E2DB21066A
:10368000FF221202224012021143FF2212042240A2
:10369000120A1143220E11430846C949091DF4F7C5
:1036A00031FE002004E0C749095C8E19411C88B234
:1036B000432109018842F6D33106FF22120232402B
:1036C00012021143FF2212043240120A1143320E39
:1036D00011430846BA490831F4F714FEBA48F4F722
:1036E000F9FDB04210D00620B84908700120B84951
:1036F0000870B84908600020B7490860B748B84961
:103700000860FBF707FF13E01F20B0490870012095
:10371000AF4908700220AF4908600420AE49086034
:10372000B048AF490860A448AF490860FBF7F2FE13
:103730007BE5AE480078012843D10020AB490870F2
:10374000AB4908700CF084FFAA4908609A480078D9
:103750009D490870984840784870974880788870EC
:103760009548C078C8709648F4F7B4FD0546964869
:10377000F4F7B0FD854210D007209449087001206D
:103780009349087093490860002093490860934862
:1037900093490860FBF7BEFE13E020208B490870B8
:1037A00001208B49087002208A49086004208A4958
:1037B000086091488A4908607F488B490860FBF798
:1037C000A9FE32E589480078012833D100208749D5
:1037D0000870874908700CF03BFF864908607648FE
:1037E0000078794908707448407848707248807849
:1037F00088707148C078C8707148001DF4F76AFD80
:1038000005467148F4F766FD854203D007206F49ED
:10381000087002E01E206D49087001206C49087094
:103820006C49086000206C4908606C486C4908606D
:10383000FBF770FEF9E46E48007801287CD1002582
:1038400000206B4908700CF003FF6A4908606B4860
:103850000068401E6A490978884235D95C20694968
:10386000087067490878C10F09184910654A5170F6
:1038700063490878C10F091849104900411AC9075E
:10388000090E917000BF09E05D480078C001401941
:103890004C49095CE81C5B4A11546D1C802DF3D324
:1038A00001204B49087083204A49086000204A499A
:1038B000086054484A490860FBF72CFE50480078DD
:1038C000401C4F49087036E05C204E4908704C4956
:1038D0000878C10F091849104A4A517048490878B8
:1038E000C10F091849104900411AC907090E917002
:1038F000002509E042480078C00140193149095CBF
:10390000E81C404A11546D1C3F4800688542F1D3C1
:1039100001202F4908703C480068C01C2D490860F0
:1039200000202D49086037482D490860FBF7F2FD5B
:1039300007202649087000BF77E42D480078012849
:103940001CD10CF085FE2B49086000202849087026
:1039500008201E49087001201D490870FF20FF3013
:103960001C49086000201C490860012018490870A3
:103970001248801C1A490860FBF7CCFD55E41C482E
:103980000078012816D10CF063FE1A490860002067
:103990001749087009200D49087001200C4908706A
:1039A0000C49086000200C4908600C480C4908606C
:1039B000FBF7B0FDE4E30EE26C02002062000020A1
:1039C0005602002055B802005C000020850200204D
:1039D00086020020800200207C02002052B80200F3
:1039E0006402002040B80200680200208702002024
:1039F000880200209802002042B8020070020020D5
:103A0000780200208814002074020020FE4800780C
:103A1000012817D10CF01CFEFC4908600020FA496F
:103A200008700A20FA4908700120FA490870062037
:103A3000F94908600020F9490860F948F949086027
:103A4000FBF768FD9CE3F048007801281AD10CF0E0
:103A5000FFFDEE4908600020EB4908700B20EC499F
:103A600008700120EB4908700220EB49086004202F
:103A7000EA490860EC48EB490860EC48EC4908600A
:103A8000FBF748FD7CE3EB480078012847D1002094
:103A9000E8490870E548C078E749C8700846C0782A
:103AA0000221084002281AD10020E44908600CF0E5
:103AB000CFFDD64908600020D34908700C20D449B6
:103AC00008700120D3490870D34908600020D34909
:103AD0000860DB48D3490860FBF71CFD1FE0D748AE
:103AE0000068401CD549086008460068FF212D3158
:103AF00088420ED90020D14908600220D1490870BF
:103B0000D148007801210843CF490870FDF72AFC0D
:103B100005E00120BC4908700A20BD4908702FE368
:103B2000B9480078012816D10CF092FDB749086019
:103B30000020B54908701A20B54908700120B54920
:103B40000870B54908600020B4490860BF48B5490D
:103B50000860FBF7DFFC13E3AB48007801281AD1BB
:103B60000CF076FDA94908600020A74908701B20C9
:103B7000A74908700120A74908700220A6490860DB
:103B80000420A6490860A848A6490860A748A84993
:103B90000860FBF7BFFCF3E2A648007801284AD191
:103BA0000020A4490870A148C078A349C8700846FD
:103BB000C0780821084008281DD100209F490860CE
:103BC000914908700CF044FD904908601C20904910
:103BD000087001208F49087002208F490860042076
:103BE0008E4908609A488F4908609048904908605B
:103BF000FBF790FC1FE091480068401C8F4908606B
:103C000008460068FF212D3188420ED900208B49DB
:103C1000086002208B4908708B4800780121084316
:103C200089490870FDF79EFB05E001207649087080
:103C30001A2077490870A3E27E48007801285AD1FB
:103C400000207C490870704908700CF001FD6F4934
:103C50000860764800787849087074484078487061
:103C60007248807888707148C078C8707948F4F7D5
:103C700031FB05467048F4F72DFB854227D0764886
:103C80000068401C744908600846006803280DD984
:103C90000020086002206B4908706B480078012101
:103CA000084369490870FDF75DFB24E00720584987
:103CB000087001205749087057490860002057498B
:103CC00008605F4857490860FBF724FC13E01D209B
:103CD0004F49087001204F49087002204E49086082
:103CE00004204E4908605D484E4908604F485049DD
:103CF0000860FBF70FFC43E24E48007801284DD1E5
:103D000000204C490870404908700CF0A1FC3F4964
:103D10000860464800784849087044484078487030
:103D20004248807888704148C078C8704948001D72
:103D3000F4F7D0FA05464048F4F7CCFA85421AD099
:103D400045480068401C444908600846006803284C
:103D50000DD90020086002203A4908703A480078DE
:103D60000121084338490870FDF7FCFA09E00720F3
:103D70002749087005E00020374908601E202449C3
:103D80000870012023490870234908600020234956
:103D900008602B4823490860FBF7BCFBF0E11A4898
:103DA0000078012817D10CF053FC18490860002056
:103DB000154908700D201649087001201549087032
:103DC0000620154908600020144908602448154958
:103DD0000860FBF79FFBD3E10B480078012848D12E
:103DE0000CF036FC094908600020074908700120E2
:103DF0000849087008490860002008490860194807
:103E00000849086030E00000880200209802002085
:103E10008502002086020020800200207C02002013
:103E200024B802006402002022B802006C020020C4
:103E300068020020870200205C0000209002002021
:103E400052B80200890200208A02002054B8020001
:103E500040B80200560200209402002042B802003E
:103E60002AB8020050B80200FBF754FB2120D549C4
:103E7000087085E1D448007801281AD10CF0E8FBDD
:103E8000D24908600020D04908702220CD4908702E
:103E90000120CF4908700220CE4908600420CE4995
:103EA0000860CE48CE490860CE48CF490860FBF78D
:103EB00031FB65E1CD480078012844D10020CB4991
:103EC0000870C848C078CA4948700846407804213C
:103ED0000840042817D10020C64908600CF0B8FB40
:103EE000BA4908600120BA490870BA490860002040
:103EF000B9490860C048BA490860FBF70BFB0E20BF
:103F0000B04908701FE0BB480068401CB949086010
:103F100008460068FF212D3188420ED90020B5499E
:103F200008600220B5490870B548007801210843AF
:103F3000B3490870FDF716FA05E00120A2490870A0
:103F40002120A04908701BE19F480078012821D159
:103F50000020AC4908709C4908700CF079FB9B4923
:103F60000860A948C078A8491431C97848437D2120
:103F70004843C117490E0918C8117D21C900F4F73B
:103F8000DFF8C01C87B2394608200AF0A5F80F20D8
:103F90008C490870F4E0082009F0D0FE00280BD10D
:103FA00002209649087096480078012108439449F8
:103FB0000870FDF7D7F996E09248007801283ED1C5
:103FC00092480088FF210131084390490880002071
:103FD0008F4908708B4908708B48C0788A49143122
:103FE000C97848437D214843C117490E0918C811B3
:103FF0007D21C900F4F7A4F8C01C87B23946082017
:104000000AF06AF80CF024FB7049086012206D4930
:10401000087001206E49087002206E4908607A48D5
:104020001430C0780C2148436B49086079486C49CA
:10403000086079486C490860FBF76CFA53E07748F0
:10404000007801280BD1F8F741FB012807D10020A7
:104050006F490870714908705A49087043E0FDF7CC
:104060009FF901281AD1FDF7B5F9002068490870B9
:104070000CF0EEFA554908601020524908700120F2
:1040800053490870062053490860002052490860CF
:10409000634853490860FBF73DFA24E0FDF780F9D7
:1040A00002281AD1FDF796F90020594908700CF042
:1040B000CFFA46490860102042490870012044495F
:1040C00008700620434908600020434908605548AD
:1040D00043490860FBF71EFA05E001204C490870CF
:1040E0000F20384908704BE03748007801280CD180
:1040F00000203E4908703449087036490860364946
:1041000008600F202F49087002E010202D49087028
:1041100036E036480078012815D100203349087070
:104120002949087013202749087001202849087080
:10413000284908600020284908602F48284908605D
:10414000FBF7E8F902E012201E49087018E01E484B
:10415000007801280FD10020244908701A490870FE
:104160001C4908601C4908600120244908700F2080
:104170001449087002E013201249087000E000BFE3
:1041800000BF104800780F281BD00E480078002888
:1041900017D00CF05DFA0D490968401A224988428F
:1041A0000FD31748007802210843154908700220F0
:1041B0001249087000200849086006490860FDF7A8
:1041C000D1F8F8BD85020020880200209802002066
:1041D00086020020800200207C02002022B802001B
:1041E000640200206C020020680200208702002088
:1041F0005C0000209002002052B8020089020020DA
:104200008A0200208402002086000020C0040020D2
:104210008D02002030B80200C81300208B0200205D
:104220004AB8020044B80200B0AD01007047000077
:1042300010B525480078002804D0012812D00228A3
:104240003ED12AE002F01CFB0A2805D107F03AFC17
:1042500002201D49087004E000F0B0F801201A495E
:1042600008702EE002F00CFB0A2815D1002002F0A5
:104270000BFA002015490870082000F08DF8002086
:10428000134908601349086013490860134814492A
:10429000086002200C49087013E002F0F1FA0128CE
:1042A0000DD100200F49088000F088F8102000F0A0
:1042B00073F80D480A49086001200349087000E0BE
:1042C00000BF00BF10BD00007C030020520300208F
:1042D000087F00200C7F0020187F00205A6B7C8D07
:1042E000107F00201C7F00208D7C6B5AF8B525487C
:1042F0000078002802D0012840D107E03C210520A9
:1043000009F0EAFE01201F49087038E0052009F095
:1043100015FD002831D1022000F0F2F900901220A2
:10432000FAF78EFB00281ED11748F3F7D3FF054696
:1043300029460098F4F74FF804461449F4F740FB77
:1043400011D21148F3F7C6FF04461149F3F7DAFF1B
:104350000F48F3F7BFFF0646F4F7D0FA04460D4ABC
:10436000F3F7D9FF06E01220FAF77CFB0649009824
:10437000F3F7C8FF00200349087000E000BF00BF4A
:10438000F8BD000034030020350300200000164370
:10439000381900209D030020082803D10121064A76
:1043A000117008E0102803D10221034A117002E0C5
:1043B0000021014A117070478C020020F0B585B0D1
:1043C00009F01AF80546802102F022F90CF040F9B4
:1043D000964908600421964808F0EAFF012817D0A2
:1043E0000421944808F0E4FF012811D000219048EE
:1043F0000068F4F7DBFA0BD38F498D480068F4F7B7
:10440000DFFA05D300218B480068F4F7CFFA04D215
:10441000002087490860874908600221874808F022
:10442000C7FF012802D10020844908804D20FAF7F7
:1044300007FB002843D04D20FAF714FB7F48008883
:10444000F4F7E9F9432109060290F4F709F87C49E9
:104450000390F3F76FFF0746754801683846F3F796
:10446000C2FF0646734801683046F3F763FF05460E
:104470007449F3F747FF7448F3F72CFF03906F4834
:104480000088F4F7C8F9432109060090F3F7E8FF24
:104490006B490190F3F74EFF02906548016802985E
:1044A000F3F7A1FF07466949F3F7DAFF06460399D8
:1044B000F3F740FF05466449F3F724FF3FE05F4808
:1044C0000088F4F7A8F9432109060290F3F7C8FF22
:1044D00007465F49F3F72EFF03905548016803989C
:1044E000F3F781FF0646534801683046F3F722FF91
:1044F00005465449F3F706FF5348F3F7EBFE0390E4
:104500004E480088F4F787F9432109060090F3F735
:10451000A7FF07464E49F3F70DFF01904448016895
:104520000198F3F760FF49490290F3F799FF0646B7
:104530000399F3F7FFFE05464349F3F7E3FE4248CC
:10454000F3F7C8FE0746F4F7D9F90546414AF3F7F1
:10455000E2FE002040490860012040490870002028
:104560003F4908703749091DF3F7CCFE354908313A
:104570000020F3F7C7FE344908310020F3F7C2FEEC
:10458000304930310020F3F7BDFE2E493431002090
:10459000F3F7B8FE2B4938310020F3F7B3FE294971
:1045A0003C310020F3F7AEFE264940310020F3F7FE
:1045B000A9FE002405E00020A1002A4A5050601CFA
:1045C00084B2102CF7DB40212748F3F75CFE00246F
:1045D00005E00020A100254A5050601C84B2102C38
:1045E000F7DB002405E00020A100214A5050601CA8
:1045F00084B2142CF7DB002405E00020A1001D4A42
:104600005050601C84B21E2CF7DB00201A49088031
:104610001A4908701A4908801A4908801A4908700E
:104620001A4908601A49087005B0F0BD64030020FB
:104630000C7F0020087F00200080BB441C7F0020EE
:1046400066661640801900203819002000007A4460
:104650003333B33E9D030020187F00207D030020EC
:104660005203002084170020C417002004180020E3
:1046700044180020941800204C0300204E03002012
:104680004003002042030020440300207803002060
:10469000450300200349C9788900034A891801604D
:1046A000704700009A000020C813002010B50221B6
:1046B000C02000F02BFD012805D10349087002211C
:1046C000C02000F0F7FC10BD840200200349C97827
:1046D000C900034A89180160704700009A00002051
:1046E000C813002005480078002804D000200349A2
:1046F0000870012070470020FCE70000C70300207D
:10470000F8B5044623000FF040FF0D6A080C2A3D5F
:1047100042474C51565B60656A003248F3F7DAFD58
:10472000F8BD30480838F3F7D5FD05460021F4F709
:104730003DF90FD22B4908390020F3F7E3FD294852
:104740000838F3F7C7FD0746F4F7D8F80546264AB8
:10475000F3F7E1FD23480838F3F7BCFDE0E7214813
:10476000001FF3F7B7FD05460021F4F71FF904D247
:104770001C49091F0020F3F7C5FD1A48001FF3F775
:10478000A9FDCDE71748001DF3F7A4FDC8E71548BC
:104790000830F3F79FFDC3E712480C30F3F79AFD9A
:1047A000BEE710481030F3F795FDB9E70D48143017
:1047B000F3F790FDB4E70B481830F3F78BFDAFE744
:1047C00008481C30F3F786FDAAE706482030F3F7C7
:1047D00081FDA5E703482430F3F77CFDA0E7002026
:1047E000C0439DE7401900209D030020002014498C
:1047F0000979134AD27852001143114A5279920032
:1048000011430F4A5278D20011430D4A127A120115
:1048100011430B4A927852011143094AD27992010D
:104820001143074A1278D2011143054A92791202C4
:104830001143034A527A5202114388B27047000072
:10484000D81900200149016070470000C2160020FD
:1048500070B5044623000FF098FE0D4C080C11169D
:1048600023282D3A3F444C494C002348F3F732FDAE
:1048700070BD21480838F3F72DFDF9E71E48001FE9
:10488000F3F728FDF4E70020FBF7B2F905461A49D3
:10489000091DF3F737FD1848001DF3F71BFDE7E787
:1048A00015480830F3F716FDE2E713480C30F3F72C
:1048B00011FDDDE70120FBF79BF905460E4910319C
:1048C000F3F720FD0C481030F3F704FDD0E70A4859
:1048D0001430F3F7FFFCCBE707481830F3F7FAFC86
:1048E000C6E705481C30F3F7F5FCC1E7034800684C
:1048F000BEE70020C043BBE7881900203C0300202E
:10490000FEB505460C462846F3F785FF07468F217E
:10491000C905F3F7A5FD06462046F3F77CFF3146AF
:104920000090F3F760FD0746F3F79EFF01900198B2
:1049300000F094FDFEBD70B504462046F3F76BFF12
:1049400005468F21C905F3F78BFD70BD70B50024B6
:10495000F6F7ACFE012827D12948F3F7BBFCC00FBE
:10496000C0070121C907884210D12548F3F7B2FCDE
:10497000C043461C3046FFF7DEFF0546214801686C
:104980002846F3F7D7FC1F4908600DE01C48F3F7F1
:10499000A1FC0646FFF7CFFF05461A4801682846E6
:1049A000F3F71DFD17490860164800680121C90783
:1049B0004840044614492046F3F7F8FF04D313494E
:1049C0002046F3F7FDFF00D270BD00212046F3F72B
:1049D000EDFF0CD20120C00744402046F9F774FFD8
:1049E000401EC54306492846F3F78CFC06E02046E6
:1049F000F9F76AFF05460249F3F784FC00BFE3E7D5
:104A00004A1A0020B40300200AD723BD0AD7233D49
:104A10000148006870470000107F002010B50D4865
:104A20000078002813D10C48007800280FD10B48DB
:104A3000007801280BD10A480078002807D1FCF73C
:104A4000A9FC04210840042801D1012010BD002048
:104A5000FCE70000B8030020B1030020C4030020DD
:104A60003903002010B50020284988704870C870AC
:104A70000870274908702749087027490870274996
:104A800008702749087005E0F7F798FEFAF780F9F3
:104A9000FCF71AFA234800780028F5D004212248B0
:104AA00008F086FC01280BD000211F480068F3F7AE
:104AB0007DFF05D31D491C480068F3F781FF02D232
:104AC0001B48194908601B4800681B4988420AD0E6
:104AD000184800681949884205D0174815490860E8
:104AE000134811490860134800681449884206D1E8
:104AF0001020FFF751FC0020FAF750F904E00020E5
:104B00000F4908600F49086010BD0000D819002047
:104B10007C03002039030020B1030020C4030020DF
:104B200034030020C6030020387F002000007042BC
:104B30000000A041107F00205A6B7C8D8D7C6B5A49
:104B4000087F00200C7F0020F8B507460C46384649
:104B5000F3F761FE05461549F3F7D4FB1348F3F765
:104B6000B9FB0090F3F7CAFE0546114AF3F7D3FBF1
:104B70000E48F3F7AFFB05460E49F3F7C3FB0B48AE
:104B8000F3F7A8FB0C4908602046F3F744FE0546FE
:104B90000649091DF3F7B6FB0448001DF3F79AFB1D
:104BA00006490860012006490870F8BD3819002040
:104BB0009D0300207E030020007F0020047F002052
:104BC000B0030020FEB5FFF733FBFBF7C7FD08F08D
:104BD000A3FC01F055FE0A2856D17248007800283F
:104BE00002D001284FD122E009F098F808210840AE
:104BF00008281BD1FAF7B6FD012817D1032009F0C8
:104C0000B5F8FAF7B5FDF9F773FE0BF021FD66492B
:104C1000086066480078FCF767FCF9F74BF9002854
:104C200004D10120624908705E4908702BE0FAF750
:104C300099FD012826D1032009F098F8FAF798FD8C
:104C4000F9F756FE0BF004FD57490968401A594917
:104C500008600BF0FDFC544908605648006856494E
:104C6000884202D955485349086050480078FCF7FB
:104C70003BFCF9F71FF9012804D1002049490870CD
:104C80004B49087000BF84E001F0FAFD012819D1FA
:104C9000FAF762FF012815D10BF0DAFC48490860E9
:104CA000FAF760FD012874D1FAF762FDF6F798FD76
:104CB000F9F71EFE3D480078FCF716FC2220F9F7B4
:104CC000D1FE66E001F0DCFD012862D10BF0C0FCF2
:104CD0003B490968401A3B4988425AD32220F9F7D8
:104CE000AFFE002852D1F9F7E5F8012851D1364836
:104CF0000088F3F790FD432109060290F3F7B0FB1B
:104D000007463249F3F716FB06463148016830463C
:104D1000F3F769FB05462F4801682846F3F70AFBBD
:104D200004462D49F3F7EEFA2C48F3F7D3FA029034
:104D300025480088F3F76FFD432109060090F3F73B
:104D40008FFB22490190F3F7F5FA074620480168E6
:104D50003846F3F748FB06462149F3F781FB054641
:104D60000299F3F7E7FA04461C49F3F7CBFA1B481C
:104D7000F3F7B0FA0646F3F7C1FD0446194AF3F714
:104D8000CAFA022004F026FD0FF04AFC2220F9F7AF
:104D900069FEFBF7D3FFFCF71BFAFFF7A7FAF8F75A
:104DA000D9F8FEBDB8030020BC030020700300202A
:104DB000C0030020D40300208096980080841E0049
:104DC00064030020E0C810001C7F00203333B33E92
:104DD0000C7F0020087F0020801900203819002057
:104DE00000007A449D030020012003490870002040
:104DF00002490870704700008D02002085020020E3
:104E0000FEB5054662480668076862480570624854
:104E10000570002D68D02E20F9F712FE002802D070
:104E20000020FAF7B1FC002405E00020A1005B4A55
:104E30005050601C84B2102CF7DB002405E00020E9
:104E4000A100574A5050601C84B2142CF7DB002498
:104E500005E00020A100534A5050601C84B21E2C73
:104E6000F7DB0020504908705049088050490880FD
:104E700050490880504908705049086050490870EE
:104E80005049F3F73FFA50490020F3F73BFA4E49F7
:104E900028310020F3F736FA4B492C310020F3F784
:104EA00031FA494930310020F3F72CFA45493431C1
:104EB0000020F3F727FA434938310020F3F722FAAC
:104EC000002405E00020A100314A5050601C84B24B
:104ED0000A2CF7DB00203D4908703D4908703D4928
:104EE00008703D49086051E02E20F9F7BBFD012014
:104EF000FAF74AFC36480078032840DD00241EE01B
:104F0000A100234A50583146F3F75AFD02D8A000B9
:104F10001F490E58A1001E4A50583946F3F746FD66
:104F200002D8A0001A490F58A000194A11582A485F
:104F30000068F3F7FFF928490860601C84B2244830
:104F400000788442DCDB22490978881EF3F758FC9C
:104F50003146029020480068F3F73DFA3946009048
:104F6000F3F739FA01900299F3F77AFA1A490860CF
:104F700000201749087001201649087006E000203B
:104F8000134908701349087013490860FEBD0000FA
:104F90000C1900207D03002051030020041800207C
:104FA00044180020941800204E0300204C030020D9
:104FB0004003002042030020440300207803002027
:104FC0004503002040190020881900204F030020CD
:104FD00050030020520300205403002010B5052286
:104FE0000D490E480BF008FC00F02AF80C48027836
:104FF0000C490D48F8F7A2FC0C49086008480178F4
:105000000B48F8F7EDFB0B49086006220A490B48EC
:10501000F3F732FF10BD0000C81F0020B41F0020AE
:105020005C040020DC1A0020B41A00206004002078
:10503000DC1F0020640400208C1A0020741A002059
:1050400010B51748F3F746F9164909688900164A5A
:10505000505013480C30F3F73DF9124909688900A4
:10506000124A50500F480068401C0E49086008461C
:1050700000680A2808D00E4800680A2807D00846A9
:1050800000680B49086002E00A20094908600A210B
:1050900004480068F3F73EF80248016010BD0000C4
:1050A0008C19002058040020B41A0020DC1A0020BB
:1050B0005C04002070B504460D46044960180022C7
:1050C000294609F091FF002070BD0000100E02403B
:1050D000F8B504460E4615460548A90040180719BC
:1050E00001223146384609F07FFF0020F8BD00005C
:1050F000300D024070B504460D460349601829463C
:10510000FAF706FD70BD0000040D024070B50446BC
:105110000D46034960182946FAF7FAFC70BD0000F5
:10512000000E024070B504460E461546214960182F
:105130000022314609F058FF00201F496118B200D3
:1051400088502A781B49091F6018314609F04CFF26
:105150006A7818490C396018314609F045FFAA7879
:10516000144910316018314609F03EFFEA781149C0
:1051700014316018314609F037FF2A790D4918318A
:105180006018314609F030FF6A790A492031601809
:10519000314609F029FF094880680121C903884385
:1051A000A979C9030122D203114008430349886049
:1051B000002070BD0C0D0240000C0240000F0240A8
:1051C00010B50346024818188C000251002010BD8B
:1051D000000C024070B504460D46044960180122D7
:1051E000294609F001FF002070BD00000C0D0240AF
:1051F00070B504460D4616460349601832462946E6
:1052000009F0F2FE002070BD080D0240014604299D
:1052100001D1024800E0024870470000000200404F
:10522000004000400146002906D0012907D002298C
:1052300007D0032909D106E00120800706E00448D1
:1052400004E0044802E0044800E000BF00BF7047EB
:1052500000010040006000400064004070B588B06C
:10526000044600250026042C01D0052C71D1102104
:1052700068460FF0E7FF2046FFF7C8FF05463621D6
:1052800061435D4A891808461030F3F723F881B26C
:105290006846418036216143574A891808461430D0
:1052A000F3F718F8C1B2684641703620604352499E
:1052B00040180830007E01281AD1002069468880F5
:1052C0000AF01AFE0290362161434B4A89180846BB
:1052D0001C30F2F7FFFF81B26846C180362161437E
:1052E000454A891808460830F2F7F4FF039013E0A6
:1052F0000320C002694688804B21490202910121A6
:1053000089026846C180362161433B4A89180846B4
:105310000830F2F7DFFF039036206043364940182B
:105320000830407E69460870284601F03FFA0021A7
:10533000284601F005FA0121284601F001FA002172
:10534000284601F01CFA0121284601F004FA51E038
:10535000FFE7102104A80FF075FF2046FFF762FF5A
:10536000064636216143244A891808461030F2F770
:10537000B1FF81B268464182362161431E4A8918D5
:1053800008461430F2F7A6FFC1B2684641740AF02D
:10539000B3FD069036216143174A891808461C3030
:1053A000F2F798FF81B26846818236216143124A42
:1053B000891808460830F2F78DFF079036206043C1
:1053C0000D4940180830417E6846017404A93046F2
:1053D0000CF0BAFC002130460CF080FC0121304674
:1053E0000CF07CFC002130460CF097FC012130468B
:1053F0000CF07FFC08B070BD440E002070B5044670
:105400000A212046F2F79CFE06010A212046F2F707
:1054100097FE7018C5B2284670BD08B500200090F0
:1054200000BF00980028FCD008BDF8B50446002550
:1054300000270FE00A212046F2F782FE8EB23046A6
:10544000B840284385B2381DC7B20A212046F2F77A
:1054500077FE84B2002CEDD12846F8BDF8B504469D
:10546000002500270EE00A212046F2F753FE0E46E3
:105470003046B8400543381DC7B20A212046F2F72E
:1054800049FE0446002CEED12846F8BD10B500F0C8
:1054900089F810BD10B5C046C04610BD70B50446B1
:1054A0000D460126002229462046083009F09CFDC1
:1054B0000026304670BD014601208A6808239A43C1
:1054C0008A60002070470000F8B505460C460127A9
:1054D000244885420CD12448806A102188432249FF
:1054E00088620846806A102108431F4988620BE0E1
:1054F0001D48806A202188431B4988620846806ACB
:1055000020210843184988620020A860207AA860FA
:10551000606800012168884201D90120F8BD207A25
:10552000402814D10120286061682068F2F7F2FD5C
:10553000C008401EC6B2092E03DA0021284600F03A
:105540001FF83146284600F016F8074608E000200C
:105550002860607A4000A17A08436072607A28610E
:105560003846DBE7000400400020004001460020F0
:10557000CA68D0B2704702460120516000207047CF
:1055800070B504460D460126012229462046083002
:1055900009F02AFD0026304670BD02460120D16088
:1055A0000020704710B5F74800780F2871D00CDC48
:1055B0000C284FD004DC00280FD00B286AD117E04C
:1055C0000D2856D00E28F9D192E0153803000EF0C0
:1055D000DCFF05FDFCFBFAF961000521EA480068E3
:1055E000FFF75CFF0421E8480068FFF7C9FF9DE270
:1055F000E5480068406908280FD10521E2480068A5
:10560000FFF74CFF0421E0480068FFF747FFA221A5
:10561000DD480068FFF7C1FF1BE0DB480068406918
:10562000182816D10C20D74908700521D6480068E3
:10563000FFF734FF0421D4480068FFF72FFFD34859
:105640000088FF22120210400112CF480068FFF7C5
:10565000A4FF6BE2CC4800684069282808D10D20DF
:10566000C8490870C9480178C7480068FFF795FF26
:105670005CE2C5480068406928280CD10521C24871
:105680000068FFF77DFF0421BF480068FFF706FFB1
:105690002DE09CE03CE2BC480068406910281ED127
:1056A0000521B9480068FFF7F9FE0421B6480068F3
:1056B000FFF7F4FEA321B4480068FFF76EFFB4487B
:1056C0000088012805D10221AF480068FFF7E6FEF7
:1056D0000DE00221AC480068FFF752FF07E0AA483E
:1056E00000684069402802D10E20A64908701DE2DA
:1056F000A54800684069502831D1A5480088002895
:105700005FD0A1480068FFF731FFA249096808701F
:10571000A0480068401C9F49086005219A4800681D
:10572000FFF7BCFE042198480068FFF7B7FE9848D1
:105730000088401E9649088008460088012808D144
:105740000F209049087002218F480068FFF7A6FEDD
:1057500037E002218C480068FFF712FF31E08A48E9
:105760000068406958282CD187480068FFF7FEFE82
:1057700088490968087087480068401C85490860A6
:1057800083480088401E8249088008460088002817
:1057900017D105217C480068FFF780FE04217A4874
:1057A0000068FFF7EDFE0AF053FF7B4908607B4875
:1057B0000078102188431030784908700020714922
:1057C0000870B3E18CE1C0E078E068E032E06E4858
:1057D0000068406958282CD16B480068FFF7C6FE66
:1057E0006C49096808706B480068401C694908608A
:1057F00067480088401E66490880084600880028DF
:1058000017D1052160480068FFF748FE04215E4873
:105810000068FFF7B5FE0AF01BFF5F4908605F48AC
:1058200000781021884310305C49087000205549E9
:1058300008707BE100205A4908805348006840699D
:1058400008280FD1052150480068FFF727FE0421E2
:105850004D480068FFF722FEA2214B480068FFF781
:105860009CFE1BE0484800684069182816D11620A5
:1058700044490870052144480068FFF70FFE0421E1
:1058800041480068FFF70AFE40480088FF221202E4
:10589000104001123C480068FFF77FFE46E13A489D
:1058A00000684069282808D1172036490870374811
:1058B000017835480068FFF770FE37E1324800682C
:1058C0004069282840D132480088401E3449098860
:1058D000884221D10AF0BCFE324908602D48006898
:1058E0002F4A1288815C28480068FFF756FE2E4830
:1058F000008801280CD12D480088002808D12C48A8
:105900000088002804DD2A480088401E28490880B5
:1059100018201C49087017E01D480088401E2049C7
:105920000988884210DD1720164908701948006858
:105930001B4A1288815C14480068FFF72EFE184845
:105940000088401C16490880F0E00F480068406954
:10595000282816D11448008800282BD1094908703E
:105960000E4800781021884310300C49087005213A
:1059700005480068FFF792FD042103480068FFF71F
:10598000FFFDACE0060000203800002034000020BD
:105990002600002008000020200000203600002003
:1059A000240000201C0000203200002028000020DD
:1059B0002C00002060480088002830D05F48008814
:1059C0005F49098840185D4908805E4800685C4965
:1059D000098840185B4908605B480088002803DD9F
:1059E00040205A49088006E05948008857490880F5
:1059F00000205749088000204F4908801920554948
:105A00000870012054490880052154480068FFF7B8
:105A100045FD042151480068FFF7B2FD5FE04A48A8
:105A2000008800281DDD4548008840304349088033
:105A3000444800684030434908604020434908809A
:105A40001920444908700120434908800521434832
:105A50000068FFF723FD042140480068FFF790FD30
:105A60003DE03B480088002821DD34480088403074
:105A70003249088033480068403032490860344871
:105A800000883249088000203149088019203149B6
:105A90000870012030490880052130480068FFF770
:105AA000FDFC04212D480068FFF76AFD17E0284837
:105AB0000088002813D12A4800781021884310302C
:105AC00027490870002023490870052123480068F1
:105AD000FFF7E4FC042121480068FFF751FD25E0B1
:105AE0001E4800684069102811D115201949087016
:105AF00005211A480068FFF7D1FC04211748006807
:105B0000FFF7CCFCA22115480068FFF746FD0DE029
:105B1000002010490870052110480068FFF7BEFCFE
:105B200004210E480068FFF72BFD00BF00BF0B48A3
:105B30000068FFF7C0FC10BD2800002034000020E2
:105B40002A000020080000202C0000202600002051
:105B500030000020060000202E0000203800002029
:105B60003600002002480078C006C00F70470000D1
:105B700036000020024800788006C00F7047000001
:105B8000360000201CB50220F5F7DCFC0721684632
:105B90000FF058FB002168464170012181700021FF
:105BA000C17001714171012181716A460321002098
:105BB000FFF7B8FA002203211046FFF701FB01228C
:105BC00003210020FFF714FB1CBD10B500F004F802
:105BD0000220F5F7A9FC10BDF0B587B00721684693
:105BE0000FF030FB142102A80FF02CFB00216846B7
:105BF00041706A4603210020FFF794FA0422032132
:105C00000020FFF7DDFA012108200AF0ADF900219C
:105C1000684601724173C1720121817301730021D1
:105C20008172417202A90220F5F79AFC0AF064F928
:105C300007460D49F2F76EFA84B201200004001BFA
:105C400085B229460220F5F727FC01200004001B3D
:105C500086B231460220F5F72FFC01210220F5F72C
:105C600051FC07B0F0BD0000E02801001CB5002188
:105C700008200AF079F90220F5F764FC01220221DC
:105C8000C802FFF7B5FA072168460FF0DBFA0021DA
:105C900068464170012181700021C170017141711C
:105CA000012181716A460B218020FFF73BFA002217
:105CB0000B218020FFF79CFA6A460C218020FFF719
:105CC00031FA01220C218020FFF792FA6A46032163
:105CD0000020FFF727FA002203211046FFF770FA91
:105CE000012203210020FFF783FA1CBD0148007840
:105CF000704700009405002003480078002801D177
:105D0000012070470020FCE78F0400201CB5FFF73E
:105D100063FF072168460FF095FA0021684641703D
:105D2000012181700021C1700171012141718171D6
:105D30006A460221C802FFF7F5F901220221C802D2
:105D4000FFF756FA0BF03BFA0020034908702920B0
:105D5000F9F724F81CBD00008F04002010B52B4873
:105D60000078002804D0012821D0022848D129E059
:105D70002920F8F765FE00280BD02920F8F772FEDD
:105D80004B21C900112009F0FFF801201F490870BC
:105D90000CE000F077F8012808D100F087F8C8215E
:105DA000112009F0F1F80120184908702CE00420B6
:105DB0000BF084F8012804D10BF001FA02201349FA
:105DC000087021E01120F5F71BFC002817D10420F2
:105DD0000BF074F8012812D100F052FD0A280ED100
:105DE000F9F7FAFE00280AD1F8F7C8FF012806D112
:105DF0000BF0A6F900F05AF800200449087003E0FF
:105E000000200249087000BF00BF10BD8F040020B1
:105E100010B507480078012808D11020F5F7F0FBED
:105E2000002803D102490870FFF7ACFE10BD000046
:105E30003C00002010B500240AF00AFC054909685E
:105E4000441A05480068844201D3002010BD012097
:105E5000FCE70000B0020020AC02002010B50024D6
:105E60000AF0F6FB05490968441A054800688442AF
:105E700001D3002010BD0120FCE70000A802002093
:105E8000A40200200148007870470000510400205F
:105E90000146024800780840704700004F04002087
:105EA00001480078704700009F020020002001494F
:105EB0000870704751040020014603480078884369
:105EC000014A1070012070474F040020002801DDB6
:105ED000082800DD7047421E01239340D9B2034ACF
:105EE00012788A43014B1A7000BFF3E79F0200202B
:105EF00003480078002801D1012070470020FCE70A
:105F00009D02002003480078002801D1012070473D
:105F10000020FCE74E04002010B50AF0ADF903F0B4
:105F20000BFC10BD002003490870034908700349A9
:105F3000087070474E0400204F04002050040020D9
:105F400010B586480078002802D001286FD1EEE015
:105F5000FFF7A6FF824908700846007803000EF09C
:105F600014FB09065067CBBBCBCBCB97CB000D20E6
:105F7000F8F770FD000E7B490978884215D00D2096
:105F8000F8F768FD000E774908700D20F8F762FDFC
:105F9000000EAA2803D12C20F8F700FF05E000220C
:105FA000062141208001FFF723F92C20F8F748FD56
:105FB000002822D00D20F8F74DFD000EAA281CD194
:105FC0002C20F8F74FFD0AF09FF9002811D100228C
:105FD00003210220F6F79AFE0022062141208001CB
:105FE000FFF706F90A21202008F0CEFF01205B49C7
:105FF000087000205C49087002E0002057490870D2
:1060000093E00120FFF762FF0020554908705748D0
:10601000007801210843554908700120544908704F
:106020005A20F8F7BBFE00204C4908707DE092E052
:106030000220FFF74BFF00204949087000F014FCD4
:10604000FF21053188420ED11F20F8F703FD0028FB
:1060500009D04648007808210843444908700020C8
:106060003E49087013E000F0FFFB4249884205D129
:106070003E480078202108433C4908703B4800789E
:1060800002210843394908700020344908704CE067
:106090000420FFF71BFF0020314908700DF0D8FBEA
:1060A000042803D00DF0D4FB032811D12E4800782A
:1060B00002280DDA4C20F8F771FE2C4800782021D8
:1060C00008432A49087028480078401C264908706F
:1060D00000202249087028E00320FFF7F7FE002087
:1060E0001F49087021480078042108431F4908709F
:1060F00000201A49087018E00120FFF7E7FE02208F
:10610000FFF7E4FE0320FFF7E1FE0420FFF7DEFEC9
:106110000520FFF7DBFE0620FFF7D8FE0720FFF77C
:10612000D5FE0820FFF7D2FE00BF00BF14E02020FC
:10613000F5F766FA01280DD10122062141208001E0
:10614000FFF756F8012203210220F6F7DFFD0020B9
:106150000249087000E000BF00BF10BD4E040020DF
:106160005004002052040020530400204F0400205B
:10617000510400200203000010B5F8480078030025
:106180000EF003FA0A064C9EBEFAF9F8F7F6F5F49B
:10619000F3480078002812D00020F149087022202E
:1061A000F5F72EFA00280AD12320F5F729FA01285D
:1061B00005D1EC48007808210843EA490870F5F752
:1061C00089FAE949087008460078002814D0084682
:1061D000007800F0D0F9012805D1F5F70DFB00207B
:1061E000DE49087019E0F5F707FB022000F0F2F92C
:1061F0000120DA49087010E03220F8F721FC00286D
:1062000008D03220F8F72EFC0020D84908802C2036
:10621000F8F7C4FD0020D14908709CE1FFF71EFE8D
:10622000002849D1D048007800F0A5F9012806D10E
:10623000022000F0CFF90220C84908703FE0CC48A6
:106240000078401CC0B2CA49087001282DDBC6483E
:106250000078022818D1C5480088401CC34908802E
:10626000084600881E2816DD0022062141208001F4
:10627000FEF7BEFFBB48007804210843B949087007
:106280000020B649087010BDB84800881E2802DDFD
:106290003220F8F783FDB348007801210843B14963
:1062A00008700320AD49087002E00120AB49087076
:1062B000022000F08FF902E00120A84908704AE1AD
:1062C000FFF7CCFD002817D1A748007800F053F95C
:1062D000012808D10020A6490870F5F78DFA0020A2
:1062E0009E4908700BE0F5F787FA022000F072F97A
:1062F00001209A49087002E00220984908702AE1BA
:10630000FFF7ACFD00285BD19748007800F033F927
:10631000012806D1022000F05DF904208F490870A1
:1063200051E093480078401CC0B291490870C828D9
:106330003FDB8D48007802281FD18C480088401C24
:106340008A490880084600881E281DDD0022062193
:1063500041208001FEF74CFF824800780421084369
:106360008049087000207D4908708CE7EFE0D4E098
:10637000A6E08EE070E044E026E07C4800881E281D
:1063800002DD3220F8F70AFD764800780221084342
:10639000744908700120724908700021222008F019
:1063A000F3FD9621232008F0EFFD05206B490870CE
:1063B00002E0032069490870022000F00BF902E0B6
:1063C000032066490870C6E0FFF748FD002814D195
:1063D0006548007800F0CFF8012805D10020644915
:1063E00008705E4908700BE0F5F706FA022000F02D
:1063F000F1F803205949087002E004205749087059
:10640000A9E0FFF72BFD002822D15748007800F0C3
:10641000B2F8012806D1022000F0DCF806204F492E
:10642000087018E0FFF73CFD02210840002808D161
:106430004F4908701E2000F0BBF80720474908703C
:1064400009E0022000F0C6F805204449087002E087
:106450000520424908707EE0FFF700FD002814D1B6
:106460004148007800F087F8012805D10020404914
:1064700008703A4908700BE0F5F7BEF9022000F009
:10648000A9F805203549087002E006203349087054
:1064900061E0FFF7CFFC00280BD135490870314887
:1064A0000078042108432F49087000202B49087008
:1064B00005E0022000F08EF80820284908704AE024
:1064C000FFF7CCFC002824D12748007800F053F8CF
:1064D000012806D1092021490870022000F07AF82D
:1064E0001AE023480078401CC0B221490870642893
:1064F0000BDB002008701B48007802210843194973
:10650000087007201549087006E007201349087035
:1065100002E00820114908701DE0FFF79FFC0028E9
:1065200011D11148007800F026F8012805D100208B
:106530000F4908700949087008E0F5F75DF9072070
:106540000649087002E009200449087003E00020B1
:106550000249087000BF00BF00BF94E69D02002002
:10656000A00200209F020020B4020020B6020020FA
:106570009E020020704710B50446022C04D10A2167
:10658000802000F007F810BD0B210120000300F06F
:1065900001F8F8E770B504460D4629462046FEF797
:1065A000A9FD002801D0012070BD0020FCE70000FB
:1065B00010B5044604486043044908600AF048F8EE
:1065C0000349086010BD000040420F00AC020020EB
:1065D000B002002010B504467D20C0006043810059
:1065E0004018034908600AF033F80249086010BDFA
:1065F000A4020020A8020020704710B5C046C04683
:1066000010BD10B502F038FFC046C04610BD0000F6
:106610003EB504460D460A2168460EF013FE0121E0
:10662000092009F0A1FC0721684601700021C17012
:106630008170002C03D003206946487002E00220DC
:1066400069464870002168460171417101218171DC
:106650000804401B81B2684601816946094802F07E
:106660004CFF084802F024FF0121064802F033FFE6
:10667000012203211120F6F749FB0121014802F014
:1066800020FF3EBD000F004010B50446012C08D18C
:106690000121092009F068FC0121064802F011FFE0
:1066A00007E00021092009F05FFC0021014802F009
:1066B00008FF10BD000F00400149096888B270470B
:1066C000400F00403EB504460A2168460EF0BAFD70
:1066D0000121242009F048FC0721684601700021AF
:1066E000C1708170002C03D003206946487002E01D
:1066F000022069464870002168460171417181712C
:1067000001816946094802F0F8FE084802F0D0FE0F
:106710000021064802F0DFFE012203211120F6F7D6
:10672000F5FA0121014802F0CCFE3EBD400F0040C9
:1067300010B502F0B3FE10BD10B502F0B4FE10BDEE
:1067400070B504460D46002229462046143008F054
:106750004BFC002070BD70B504460D460022294652
:10676000201D08F041FC002070BD70B504460D46A8
:1067700001222946201D08F037FC002070BD70B5AD
:1067800004460D4601222946201D08F02DFC00205C
:1067900070BD70B504460D460026294620461030CF
:1067A000F9F7B6F90646304670BD0000F0B587B07F
:1067B00005460C460127224A07CA04AB07C300203E
:1067C0000390002C02D1042007B0F0BD00206860C7
:1067D000608861780843E1880843A18808432178EC
:1067E000084368602078402802D02078C02824D14F
:1067F000E088C117C90D09184912890004AA515A25
:106800008EB2E168B1400846F2F705F80290A06840
:10681000F2F701F801900299F1F722FE03903F216F
:1068200009060398F1F786FD0290F2F71DF880B291
:10683000A86104212846FFF798FF00273846C3E7E0
:10684000C0BD020001460868C0B270470246106829
:10685000000A0002CBB2184310600020704710B548
:1068600002F0B6FE10BD00000348007800020349A4
:106870000978084370470000230400202404002006
:1068800003480078042801D1012070470A20FCE762
:106890002304002010B50120174908701749002073
:1068A000F1F730FD1321002001F0F6FB1321012048
:1068B00001F0F2FB1321022001F0EEFB1321032073
:1068C00001F0EAFB1321042001F0E6FB132105206F
:1068D00001F0E2FB1321062001F0DEFB132107206B
:1068E00001F0DAFB1321082001F0D6FB1321092067
:1068F00001F0D2FB10BD0000C3020020C402002042
:10690000032803D0072801D0082833D14F49096A4A
:1069100082004F4B9A58120991434C4A11628100F0
:106920004C4A5158090982004B4B9A58120911439D
:10693000464A526A8A4345494A628100474A515849
:1069400009098200464B9A58120911433F4A926A3C
:106950008A433E498A628100424A515809098200AD
:10696000414B9A5812091143384AD26A8A4337492F
:10697000CA626AE002283CD13449C96A8200394BB4
:106980009A5812099143314AD1621146896A8200AC
:10699000324B9A58120991432C4A91621146496A26
:1069A00082002C4B9A5812099143284A5162114691
:1069B000096A8200264B9A5812099143234A1162B0
:1069C000114649688200244B9A5891431F4A5160EE
:1069D0001146C9688200244B9A5891431B4AD160E2
:1069E0001146896882001E4B9A589143174A91605C
:1069F0002BE0164909688200154B9A589143134AB7
:106A000011608100134A51588200134B9A58114368
:106A10000E4A52688A430D494A6081000F4A515814
:106A200082000F4B9A581143084A92688A430749DB
:106A30008A6081000B4A515882000B4B9A581143CF
:106A4000024AD2688A430149CA607047405C0040EC
:106A500000BD0200D8BC020028BD0200B0BC02008C
:106A600078BD020088BC020050BD0200F8B50546A2
:106A70000C462B000DF089FD140B2532485E728701
:106A8000A1B0CFF4F2F1F0EFEEEDECEBEAE9A0000B
:106A9000D4490858A100D44A515808430090A00096
:106AA000D24E3058A600D24FBE5930430246A00005
:106AB000D04E3358A000D04E3158204602F0FEFB95
:106AC0008EE100200090A000CA490B58A000C749E1
:106AD0000A580021204602F0F1FB81E1A000C149E3
:106AE00008580090A000C34E3058A600C34FBE59AE
:106AF00030430346A000BE4E3258A000BE4E31586F
:106B0000204602F0DBFB6BE1A000B649085800907C
:106B1000A000B84E3058A600B84FBE5930430346C7
:106B2000A000B24E3258A000B34E3158204602F0B9
:106B3000C5FB55E1A000AC4908580090A000AD4944
:106B40000858A100AD4E715808430346A000A7495C
:106B50000A580021204602F0B1FB41E1A000A14902
:106B60000858A100A04A515808430090A000A34E25
:106B70003358A0009D4E3258A0009F4E31582046F9
:106B800002F09CFB2CE1A00096490858A100964A0F
:106B9000515808430090A000944E3058A600944FDE
:106BA000BE5930430246A000944E3358A000924E86
:106BB0003158204602F082FB12E1A00089490858B2
:106BC0000090A0008B490B58A00088490A5800216A
:106BD000204602F073FB03E1A00082490858A1009F
:106BE000814A515808430090A000824E3058A600B8
:106BF000824FBE5930430346A0007C4E3058A60059
:106C00007B4FBE5930430246A0007B4E3158204690
:106C100002F054FBE4E0A00072490858A100724A57
:106C2000515808430090A000724E3058A600734F90
:106C3000BE5930430346A0006C4E3258A0006E4E41
:106C40003158204602F03AFBCAE0C8E0C3E0B7E0A2
:106C5000A5E08CE078E062E048E034E01DE0FFE78A
:106C6000A00060490858A1005F4A515808430090AD
:106C7000A00060490858A100604E715808430346BF
:106C8000A0005A490858A100594E715808430246BD
:106C90000021204602F012FBA2E0A0005249085851
:106CA0000090A000514E3058A600514FBE593043BD
:106CB0000246A000514E3358A0004F4E3158204696
:106CC00002F0FCFA8CE0A00046490858A100464AB0
:106CD000515808430090A000454B1A58A000464B5D
:106CE00019580023204602F0E9FA79E000200090CC
:106CF000A000404E3058A600404FBE5930430346D6
:106D0000A0003A4E3058A600394FBE5930430246D3
:106D1000A000394E3158204602F0D0FA60E0A000C1
:106D200030490858A100304A515808430090A0004B
:106D3000324E3358A0002E4E3258A0002E4E3158FD
:106D4000204602F0BBFA4BE0A00026490858A100FB
:106D5000254A515808430090A00028490B58A0002C
:106D600023490A580021204602F0A8FA38E0A00082
:106D70001C490858A1001C4A515808430090A00023
:106D80001C490858A1001D4E715808430346A00035
:106D900017490A580021204602F090FA20E0A0008E
:106DA000114908580090A000144E3358A000104E0E
:106DB0003258A000104E3158204602F07FFA0FE002
:106DC00000200090A0000D490B58002211462046DB
:106DD00002F074FA04E02046FFF792FD00E000BFE5
:106DE00000BFF8BD88BC020050BD0200D8BC020044
:106DF00028BD0200B0BC020000BD020078BD020048
:106E000010B5FDF7F3FC514908705148007800288F
:106E100002D0012878D145E005F0FEFB4D49097804
:106E2000884206D005F0F8FB4A490870012048491D
:106E30000870464800782021084047490978884270
:106E400008D04248007820210840434908700120BA
:106E50003F49087013F0ACF940490978884206D0E0
:106E600013F0A6F93D49087001203949087013F064
:106E70007BF93B490978884206D013F075F9384907
:106E800008700120324908700CF0E8FC3549097897
:106E9000884206D00CF0E2FC3249087001202C49EF
:106EA000087050E005F0B8FB0A2803D1012001F07A
:106EB000CDFB02E0002001F0C9FB27480078202824
:106EC00003D1012001F006FB02E0002001F002FBEB
:106ED00022480078012802D101F086F802E0002063
:106EE00001F082F81E480078012802D101F0EAF88A
:106EF00002E0002001F0E6F81B480078002804D1E9
:106F0000012001F043F803E019E0002001F03EF811
:106F100014480078032807D012480078042803D0CA
:106F200010480078052803D1012001F06FFB02E032
:106F3000002001F06BFB00200549087003E00020F1
:106F40000349087000BF00BF10BD00002B040020E3
:106F5000200400202504002026040020270400200F
:106F6000280400202A04002029040020F3B583B05F
:106F70000E46092700BF0398029000210298F1F7FE
:106F800015FD03D2F90702984840029033000DF036
:106F9000FCFA06040F1C2937455358480299F1F7AB
:106FA00022FA029001F072FB019001F0ABF84BE085
:106FB00053480299F1F717FA029001F067FB514923
:106FC0000843019001F09EF83EE04F480299F1F726
:106FD0000AFA029001F05AFB4C490843019001F073
:106FE00091F831E04A480299F1F7FDF9029001F079
:106FF0004DFBE121C9040843019001F083F823E02F
:1070000044480299F1F7EFF9029001F03FFB61214A
:1070100009050843019001F075F815E03E48029912
:10702000F1F7E1F9029001F031FB21214905084314
:10703000019001F067F807E00298029001F026FB4A
:10704000019001F05FF800BF00BF0298F1F720FC4B
:1070500004460D462046294600235840594008431F
:1070600020D016E00A22002320462946F1F77CF8BA
:10707000D0B239467A1E57B20190C8B2019901F0D8
:107080000BF80A22002320462946F1F76DF8044642
:107090000D460021084661406840014306D0002F9C
:1070A000E0DA03E00021092000F0F6FF002E15DDF4
:1070B000062E13DA01F0EAFA0121C906B1400843AD
:1070C000019001F01FF806E039467A1E57B2C8B2A7
:1070D000002100F0E1FFF01CB842F5DD002F0BDBD2
:1070E00000210398F1F762FC06D239467A1E57B2A6
:1070F000C8B2122100F0D0FF05B0F0BD00247449E1
:107100000050C3470000C20700401C46000084072F
:1071100000007A440000C84200002041F8B507464C
:107120000C460825002F16D010E00A213846F0F74B
:10713000F1FF009129466A1E55B2C8B2009900F0CD
:10714000ABFF0A213846F0F7E5FF0746002F19D0BC
:10715000002DEADA16E00620001BC6B208E0294638
:107160006A1E55B2C8B2002100F096FF701EC6B26A
:10717000002E01D0002CF2D1002C03D100210820D8
:1071800000F08AFF23000DF000FA05040A131C2505
:107190002E0001F07BFA009000F0B4FF29E001F02E
:1071A00075FA012149040843009000F0ABFF20E08C
:1071B00001F06CFA012189040843009000F0A2FF5D
:1071C00017E001F063FA0121C9040843009000F0C0
:1071D00099FF0EE001F05AFA0121090508430090D9
:1071E00000F090FF05E001F051FA009000F08AFFF6
:1071F00000BF00BFF8BD0000F8B50446FFF74AFB2A
:1072000023000DF0C2F906CE042B7998CBCE0120D5
:10721000400200F077FF02206B49087008460078B2
:10722000F8F750FB69490860084600680090684913
:107230000098F1F7BBFB08D266490098F1F710F906
:1072400005460121FFF792FE07E062490098F1F739
:1072500007F905460321FFF789FEB3E05E4800F019
:1072600051FF03205849087008460078F8F72AFBB8
:107270005649086008460068009058490098F1F7A0
:1072800095FB0BD253490098F1F7EAF80121C907A1
:10729000484005460321FFF769FE2CE0504900985D
:1072A000F1F784FB0BD24B490098F1F7D9F8012193
:1072B000C907484005460421FFF758FE1BE049492D
:1072C0000098F1F773FB0BD242490098F1F7C8F828
:1072D0000121C907484005460521FFF747FE0AE09E
:1072E0003C490098F1F7BCF80121C9074840054620
:1072F0000621FFF73BFE65E00720400200F002FF99
:1073000001203149087008460078F8F7DBFA2F4968
:10731000086008460068F1F77EFA07468F21C90524
:10732000F1F79EF806462A49F1F79AF80546012139
:10733000FFF71CFE46E00120C00200F0E3FE5520EE
:107340002149087008460078F8F7BCFA1F49086020
:10735000084600680A280DD20021072000F09CFE94
:107360000021062000F098FE002118480068FFF771
:10737000D5FE12E015480068642809D200210620D5
:1073800000F08AFE002111480068FFF7C7FE04E004
:1073900000210E480068FFF7C1FE13E000F044FE34
:1073A00010E00E21022000F077FE0E21032000F0F5
:1073B00073FE0A21042000F06FFE0121052000F079
:1073C0006BFE00BF00BFF8BD2C040020300400207D
:1073D00000007A440000C8420002000800247449FA
:1073E0008096184B20BCBE4CFEB50446FFF752FAFF
:1073F00001F04CF9054600F085FE23000DF0C5F8BC
:107400000FFD0945819FD0FCFBFAF9F8F7F6F5F47A
:10741000FD001120FE49087008460078F8F772FA5E
:10742000FC490860084600680002010F012000F0D6
:1074300033FEF84800680003010F022000F02CFE24
:107440001221032000F028FEF24800880004010FFA
:10745000042000F021FEEF4800880005010F052000
:1074600000F01AFE1221062000F016FEE94800780E
:107470000006010F072000F00FFEE6480078010724
:10748000090F082000F008FE56E32220E0490870AA
:1074900008460078F8F736FADE49086008460068C2
:1074A0000002010F012000F0F7FDDA480068000338
:1074B000010F022000F0F0FD1221032000F0ECFD8E
:1074C000D44800880004010F042000F0E5FDD148F5
:1074D00000880005010F052000F0DEFD12210620C6
:1074E00000F0DAFDCB4800780006010F072000F01D
:1074F000D3FDC84800780107090F082000F0CCFD33
:107500001AE30121084600F0C7FD1221022000F015
:10751000C3FD0120BE49087008460078F8F7F2F96B
:10752000BC490860096809090A225143B94A12781E
:107530001207120F88180021FFF7F0FDFCE202216C
:10754000012000F0A9FD1221022000F0A5FD02207B
:10755000AF49087008460078F8F7D4F9AD490860DB
:107560000120C00400F0CEFDAA480068010F0520EC
:1075700000F092FDA74800680001010F062000F00E
:107580008BFDA44800680002010F072000F084FD75
:10759000A04800680003010F082000F07DFDCBE249
:1075A0000321012000F078FD1221022000F074FD7B
:1075B00003209749087008460078F8F7A3F9954921
:1075C0000860084600680002010F032000F064FD17
:1075D000904800680003010F042000F05DFD8D4815
:1075E00000880004010F09E07CE149E116E1EBE0CD
:1075F000C7E0A3E07FE05BE019E09CE2052000F03B
:107600004BFD844800880005010F062000F044FD72
:10761000804800780006010F072000F03DFD7D48FE
:1076200000780107090F082000F036FD84E20420ED
:107630007749087008460078F8F764F975490860DA
:1076400008460068010F012000F026FD714800681F
:107650000001010F022000F01FFD6E4800680002CB
:10766000010F032000F018FD6A4800680003010FB5
:10767000042000F011FD674800880004010F052078
:1076800000F00AFD634800880005010F062000F0A5
:1076900003FD604800780006010F072000F0FCFCA5
:1076A0005C4800780107090F082000F0F5FC43E270
:1076B0000421012000F0F0FC1221022000F0ECFC7B
:1076C00005205349087008460078F8F71BF951491E
:1076D000086008460068F1F7B9F800224E4B0191A6
:1076E0000090F1F715F80546F1F744F90746032134
:1076F000FFF73CFC20E20521012000F0CDFC122127
:10770000022000F0C9FC06204149087008460078B4
:10771000F8F7F8F83F49086008460068F1F796F86E
:1077200000223D4B01910090F0F7F2FF0546F1F782
:1077300021F907460321FFF719FCFDE1062101208D
:1077400000F0AAFC1221022000F0A6FC072030491C
:10775000087008460078F8F7D5F82E490860084602
:107760000068F1F773F8054600222B4BF0F7D0FFC5
:1077700001910090F1F7FEF807460321FFF7F6FBB1
:10778000DAE10721012000F087FC1221022000F03D
:1077900083FC08201E49087008460078F8F7B2F804
:1077A0001C49086008460068F1F750F800221A4B9F
:1077B00001910090F0F7ACFF0546F1F7DBF80746C2
:1077C0000321FFF7D3FBB7E10821012000F064FC9F
:1077D0001221022000F060FC09200D4908700846C3
:1077E0000078F8F78FF80B49086008460068F1F751
:1077F0002DF80022084B01910090F0F789FF054613
:10780000F1F7B8F807460321FFF7B0FB94E1000059
:107810002D040020340400200000F0400921012044
:1078200000F03AFC1221022000F036FC0A20C34985
:10783000087008460078F8F765F8C149086001202B
:10784000C00400F05FFCBE4800880004010F052062
:1078500000F022FCBA4800880005010F062000F065
:107860001BFCB74800780006010F072000F014FC4D
:10787000B34800780107090F082000F00DFC5BE118
:107880000A21012000F008FC1221022000F004FC73
:107890000220AA49087008460078F8F733F8A8498A
:1078A00008600120C00400F02DFCA54800880004F9
:1078B000010F052000F0F0FBA14800880005010F32
:1078C000062000F0E9FB9E4800780006010F072023
:1078D00000F0E2FB9A4800780107090F082000F049
:1078E000DBFB29E10B209549087008460078F8F782
:1078F00009F8934908600846006801900846007836
:10790000012836D10B21002000F0C6FB12210120F6
:1079100000F0C2FB68460179022000F0BDFB122195
:10792000032000F0B9FB694648790A21F0F708FC0A
:10793000C5B22946042000F0AFFB694648790A2108
:10794000F0F7FEFBCDB22946052000F0A5FB122181
:10795000062000F0A1FB68468179072000F09CFB1F
:107960001221082000F098FB6846C179092000F038
:1079700093FB73480078022836D10B21002000F0D9
:107980008BFB1221012000F087FB68460179022061
:1079900000F082FB1221032000F07EFB694648794B
:1079A0000A21F0F7CDFBC5B22946042000F074FB94
:1079B000694648790A21F0F7C3FBCDB22946052074
:1079C00000F06AFB1221062000F066FB6846817910
:1079D000072000F061FB1221082000F05DFB6846E3
:1079E000C179092000F058FB55480078032878D168
:1079F0001221002000F050FB694648796421F0F71D
:107A00009FFBC5B22946012000F046FB6946487934
:107A10000A21F0F795FB06460A21F0F791FBCDB25B
:107A20002946022000F038FB694648790A21F0F720
:107A300087FBCDB22946032000F02EFB69468879EA
:107A40008021084000281CD01221042000F024FBD3
:107A5000694689794806400E0A21F0F771FBC5B2E4
:107A60002946052000F018FB694689794806400E32
:107A70000A21F0F765FBCDB22946062000F00CFB89
:107A800017E01321042000F007FB694688790A21DA
:107A9000F0F756FBC5B22946052000F0FDFA69460D
:107AA00088790A21F0F74CFBCDB22946062000F078
:107AB000F3FA1321072000F0EFFA6946C8790A218A
:107AC000F0F73EFBC5B22946082000F0E5FA69460A
:107AD000C8790A21F0F734FBCDB22946092000F01D
:107AE000DBFA17480078042824D10B21002000F08D
:107AF000D3FA1221012000F0CFFA68464179022022
:107B000000F0CAFA1221032000F0C6FA694688790B
:107B10000A21F0F715FBC5B22946042000F0BCFA93
:107B2000694688790A21F0F70BFBCDB2294605207A
:107B300000F0B2FA00E000BF00BFFEBD2D0400203F
:107B40003404002070B50446FEF7A4FE00F09EFD4C
:107B5000054600F0D7FA012C02D0022C79D14DE075
:107B60000121084600F098FA1221022000F094FA50
:107B700001204B49087008460078F7F743FF494950
:107B80000860084600784007C00F002804D0012193
:107B9000052000F081FA03E00021052000F07CFAC6
:107BA000404800780007C00F002804D001210620BB
:107BB00000F072FA03E00021062000F06DFA394867
:107BC0000078C007C00F002804D00121072000F072
:107BD00063FA03E00021072000F05EFA31480078E4
:107BE0008007C00F002804D00121082000F054FABB
:107BF00003E00021082000F04FFA4FE002210120AD
:107C000000F04AFA1221022000F046FA022024492C
:107C1000087008460078F7F7F5FE22490860084624
:107C20000078C006C00F002804D00121052000F014
:107C300033FA03E00021052000F02EFA19480078FD
:107C40008006C00F002805D00121062000F024FA8C
:107C500004E022E00021062000F01EFA114800781E
:107C60004006C00F002804D00121072000F014FABC
:107C700003E00021072000F00FFA0A480078000610
:107C8000C00F002804D00121082000F005FA03E00D
:107C90000021082000F000FA00E000BF00BF70BD26
:107CA0002E04002038040020F0B587B00546FEF70A
:107CB000F1FD2B000CF069FC07FD052755A8E3FC3E
:107CC000FD00A848407A552804D10120400200F068
:107CD00019FA03E00520C00100F014FA0220A249BD
:107CE000087008460078F7F7E5FEA04908600846E6
:107CF000006805909E490598F0F7B2FB0646012101
:107D0000FFF734F92AE19748407A552804D1072033
:107D1000400200F0F7F903E01D20C00100F0F2F985
:107D200001209149087008460078F7F7C3FE8F4993
:107D3000086008460068F0F789FD064600228D4B72
:107D4000F0F7E6FC00228C4B01910090F0F7E0FC8C
:107D500003910290F0F70EFE01210490FFF706F95F
:107D6000FCE08048407A552804D10120C00200F090
:107D7000C9F903E01120C00100F0C4F90A207A49D2
:107D8000087008460078F7F795FE784908600846BD
:107D900000680121C907884219D3744800688843E4
:107DA0007249086008460068F0F750FD0646002258
:107DB000704BF0F7ADFC0022704B01910090F0F792
:107DC0003FFC03910290F0F7D5FD044613E06748AD
:107DD0000068F0F73BFD06460022664BF0F798FC82
:107DE0000022674B01910090F0F72AFC039102906A
:107DF000F0F7C0FD044663492046F0F731FB064624
:107E00000021FFF7B3F8A9E05648407A552804D17D
:107E10000120C00200F076F903E01120C00100F05B
:107E200071F90121084600F037F91221022000F013
:107E300033F904204C49087008460078F7F73AFEF9
:107E40004A49086008460068F0F700FD064600222F
:107E5000484BF0F75DFC0022494B01910090F0F790
:107E6000EFFB03910290F0F785FD0446464920465A
:107E7000F0F7F6FA06460021FFF778F86EE0394889
:107E8000407A552804D10120C00200F03BF903E0FC
:107E90001120C00100F036F90221012000F0FCF8A9
:107EA0001221022000F0F8F807202F49087001E0A5
:107EB00023E042E008460078F7F7FCFD2B49086014
:107EC00008460068F0F7C2FC06460022294BF0F78E
:107ED0001FFC00222A4B01910090F0F7B1FB0391A7
:107EE0000290F0F747FD044627492046F0F7B8FA1C
:107EF00006460021FFF73AF830E01A48407A552844
:107F000003D1202000F0FEF802E0A02000F0FAF8F3
:107F10000F21012000F0C0F80E2013490870084618
:107F20000078F7F7C7FD114908600846006805901A
:107F300003210598FFF71AF810E00E21032000F046
:107F4000ABF80E21042000F0A7F80A21052000F06C
:107F5000A3F80421062000F09FF800BF00BF07B07F
:107F6000F0BD00002E2700202F0400203C0400203C
:107F70000050C3470000F04000408F40000039C06F
:107F8000000039400000C84200401C4612490870F9
:107F900012490978104A127891421BD00E4909788B
:107FA0000E4A117001210E4A1170002809D00A4AA8
:107FB00011700C49097804229143091D094A117076
:107FC00008E00021044A117006490978042291430F
:107FD000044A117070470000C1020020C202002054
:107FE000C3020020C402002001210C4A11700028A5
:107FF00009D00B4A11700B49097849084900491CFE
:10800000084A117008E00021054A117005490978F5
:1080100049084900034A117070470000C30200205C
:10802000BF020020C402002010B5012017490870CB
:1080300017491848F0F766F90821002000F02CF8DD
:108040000821012000F028F80821022000F024F87F
:108050000821032000F020F80821042000F01CF87B
:108060000821052000F018F80821062000F014F877
:108070000821072000F010F80821084600F00CF84D
:108080000821092000F008F810BD0000C3020020FC
:10809000C4020020FFFFFF0F0A280EDA01228240EF
:1080A000064B1B881A43054B1A80142902DA044A2E
:1080B000115402E01322024B1A547047BA020020F6
:1080C0000B15002001210C4A1170002809D00B4A21
:1080D00011700B49097802229143891C084A1170DA
:1080E00008E00021054A11700549097802229143F0
:1080F000034A117070470000C3020020C002002034
:10810000C402002070B50446012046490870464864
:108110000078002807D14022214691430846434970
:10812000F0F7F0F809E040480078012805D1402137
:10813000214308463D49F0F7E5F83D48007800281E
:1081400009D03A48F0F7C6F81021084305463749E8
:10815000F0F7D8F808E03548F0F7BCF8102188436C
:1081600005463249F0F7CEF832480078002809D0A9
:108170002E48F0F7AFF80821084305462B49F0F7E1
:10818000C1F808E02948F0F7A5F80821884305461A
:108190002649F0F7B7F828480078002809D0234886
:1081A000F0F798F80121084305462049F0F7AAF8AE
:1081B00008E01E48F0F78EF845086D001B49284678
:1081C000F0F7A0F81D480078002809D01748F0F70C
:1081D00081F80221084305461449F0F793F808E0B6
:1081E0001248F0F777F80221884305460F49F0F767
:1081F00089F813480078002809D00C48F0F76AF88D
:108200000421084305460949F0F77CF808E00748CF
:10821000F0F760F80421884305460449F0F772F846
:1082200070BD0000C3020020BC020020C402002078
:10823000BD020020BE020020BF020020C0020020BC
:10824000C102002010B59E48007800281CD10120F2
:108250009B490870FCF7DCFB9A4988420AD104204C
:108260009949087001209949087008460078FFF77D
:108270001BFD23E1012094490870944908700846C9
:108280000078FEF7B9FF19E10220FDF701FE002892
:1082900034D000208E4908700220FDF70DFE8A4878
:1082A0000078042810D18948007803280CD10120D7
:1082B00085490870002085490870FEF7EBFA82486E
:1082C000007800F027F9F9E07F4800780428D0D042
:1082D00003217D480078EFF733FFC8B27A49087070
:1082E00008460078401C0870002078490870FEF7A6
:1082F000D1FA7548007800F00DF9DFE00120FDF7B4
:10830000C7FD00285AD0002071490870FEF7C2FA54
:108310000120FDF7D1FD6C48007801280FD105211F
:108320006A480078EFF70CFFC8B268490870084641
:108330000078401C087008460078FEF75DFF624830
:10834000007802280FD10E2160480078EFF7F8FE80
:10835000C8B25E49087008460078401C087008469C
:108360000078FFF741F858480078032811D15749A1
:108370000878C10F091849104900411A534A117071
:1083800010460078401C1146087008460078FFF738
:10839000D9FB4D480078042895D106214B48007838
:1083A000EFF7CEFEC8B24949087008460078401C75
:1083B000087008460078FFF777FC7FE00420FDF79F
:1083C00067FD002815D00020414908700420FDF702
:1083D00073FD3D480078042870D0FEF75BFA012059
:1083E000394908703949087008460078FEF704FFDB
:1083F00064E00820FDF74CFD002819D00020344926
:108400000870FEF747FA0820FDF756FD04202E49B4
:10841000087000202D4908702B48007800F07AF889
:1084200000F034F9802108430446FFF76BFE45E075
:108430001120F6F705FB002812D00020244908700F
:10844000FEF728FA1120F6F70DFB01201E490870EF
:1084500005201E49087008460078FEF7CDFE2DE085
:108460000020F6F7EDFA002812D000201849087015
:10847000FEF710FA0020F6F7F5FA0420124908700A
:1084800001201249087008460078FFF70DFC15E03E
:108490001020F6F7D5FA002810D000200C490870FB
:1084A000FEF7F8F91020F6F7DDFA0120064908700A
:1084B0000649087008460078FEF79EFE10BD0000D1
:1084C000220400208D7C6B5A230400202404002009
:1084D0002104002001210C4A1170002809D00B4A08
:1084E00011700B490978082291430831084A11702C
:1084F00008E00021054A11700549097808229143D6
:10850000034A117070470000C3020020BE02002021
:10851000C402002070B50446FEF7BCF9002C17DD3C
:10852000052C15DA00F0B2F80546FFF7EBFD122135
:108530000320FFF7B1FD0A210420FFF7ADFD21461E
:108540000520FFF7A9FD12210620FFF7A5FD0FE08A
:108550000E210320FFF7A0FD0E210420FFF79CFD54
:1085600012210520FFF798FD0A210620FFF794FD50
:1085700070BD000010B521480078002802D0012805
:1085800036D123E01E480078012803D11D48007829
:10859000012807D11A480078022803D0184800782B
:1085A000032807D13C21012005F096FD0120134945
:1085B00008700AE012480078042806D11249012008
:1085C00005F08AFD01200D49087015E0012005F035
:1085D000B5FB00280BD10120094908700949087032
:1085E00008460078FEF708FE00200449087003E002
:1085F00000200249087000BF00BF10BD2104002008
:108600002304002024040020302A000001210C4A09
:108610001170012809D10B4A11700B4909784022C9
:1086200091434031084A117008E00021054A117059
:108630000549097840229143034A117070470000B0
:10864000C3020020BC020020C402002001210C4A09
:108650001170002809D00B4A11700B4909781022BB
:1086600091431031084A117008E00021054A117049
:108670000549097810229143034A117070470000A0
:10868000C3020020BD020020C402002010B5024831
:10869000EFF720FE10BD0000C402002010B5092134
:1086A0000020FCF797FD0A210020FCF793FD0B2129
:1086B0000020FCF78FFD0C210020FCF78BFD04212E
:1086C0008020FCF787FD05218020FCF783FD002139
:1086D0004020FCF77FFD01214020FCF77BFD0221BB
:1086E0004020FCF777FD0C2101200003FCF772FD10
:1086F0000D2101200003FCF76DFD0E210120000378
:10870000FCF768FD0A214020FCF764FD0B214020A6
:10871000FCF760FD0C214020FCF75CFD0D214020A2
:10872000FCF758FD0E214020FCF754FD0F2140209E
:10873000FCF750FD0821C020FCF74CFD0921C020AA
:10874000FCF748FD0A21C020FCF744FD0B21C020A6
:10875000FCF740FD06218020FCF73CFD072180202E
:10876000FCF738FD08218020FCF734FD092180202A
:10877000FCF730FD08210020FCF72CFD03214020F0
:10878000FCF728FD04214020FCF724FD05214020B2
:10879000FCF720FD06214020FCF71CFD10BD000069
:1087A00007480078002809D106480078002805D13C
:1087B00005480088002801D1012070470020FCE70F
:1087C000B8020020C3020020BA0200200D48007841
:1087D000022805D10C480078022801D100207047FA
:1087E00008480078042805D107480078002801D0FF
:1087F0000020F4E705480078002801D00020EEE7CB
:108800000120ECE7230400202404002020040020A1
:108810001FB5082102A80CF015FD082168460CF0D0
:1088200011FDFFF73BFF0121162007F09DFB2E48AD
:108830000090001401900F21490501988843019090
:108840000121090301988843019001980009000162
:10885000019049000198884301904900019888439C
:10886000019049000198884301904900019888438C
:10887000019089000198884301904900019888433C
:1088800001904900019888430190684600F0D8FDA6
:108890000121684601720321417200218172C17277
:1088A0000321017301214173002181730121C173EF
:1088B00002A800F067FD00F057FD00200B4908708A
:1088C0000B4908800B4908700B4908700B49087068
:1088D0000B4908700B4908700B4908700B49087068
:1088E0000B49EFF70FFD1FBD0000FFFFB80200208E
:1088F000BA020020BC020020BD020020BE020020FF
:10890000BF020020C0020020C1020020C3020020DC
:10891000C402002010B500201549087015490870E0
:1089200015490870FCF774F81449884206D10420F0
:108930001349087001201349087004E00120104910
:1089400008701049087001200F49087000200F4975
:1089500008700F4908700F4908700F49087001200E
:108960000E49087000200E4908600E49086010BDCD
:108970002004002021040020220400208D7C6B5A5A
:1089800023040020240400202504002026040020C5
:1089900027040020280400202A04002029040020A5
:1089A000300400203C04002010B5022005F0C6F978
:1089B000002814D10121022005F08EFBFEF720FAD9
:1089C000FFF7D8FD00F012FCF5F774FA012803D187
:1089D0000020FFF7DBFA02E00120FFF7D7FAFFF7EC
:1089E00031FC10BD10B5FE480078002806D00128E3
:1089F00014D002287ED003287DD1FFE2F948007808
:108A0000002803D1F8480088002806D00120F44946
:108A1000087007F01DFEF5490860D4E3F1480078BE
:108A2000002869D0F2480078C107C90FF1484078A2
:108A30008006C00F81420BD0EE4840782021884349
:108A4000EB4909784901202211400843E94948705F
:108A5000E74800788007C10FE64840780007C00F5C
:108A600081420DD0E348407808218843E0490978E5
:108A70008907C90FC900082211400843DD49487021
:108A8000DB4800784007C10FDA4820308078400783
:108A9000C00F81420FD0D74820308078042188430E
:108AA000D34909784907C90F8900042211400843B6
:108AB000D04920318870CE4800780007C10FCD48DA
:108AC00040784007C00F81420DD0CA484078042149
:108AD0008843C74909780907C90F89000422114052
:108AE0000843C4494870C2480078C006C00FC14955
:108AF000097B02E07EE265E3AAE18907C90F8842AB
:108B00000DD0BC48007B02218843B9490978C906C9
:108B1000C90F4900022211400843B6490873B448FE
:108B200000788006C00FB34909798907C90F8842C8
:108B30000DD0B048007902218843AD4909788906F3
:108B4000C90F4900022211400843AA490871A848E8
:108B500000784006C00FA749097A8907C90F8842E3
:108B60000DD0A448007A02218843A149097849061A
:108B7000C90F49000222114008439E4908729C48CF
:108B80000078C0099B49097A4907C90F88420DD06E
:108B90009848007A04218843954909780906C90F45
:108BA0008900042211400843924908729048407895
:108BB0008007C00F8F4909788907C90F88420DD0F7
:108BC0008C48007802218843894949788907C90F70
:108BD00049000222114008438649087084484078C1
:108BE0004007C00F834909784907C90F88420DD053
:108BF00080480078042188437D4949784907C90F96
:108C000089000422114008437A4908707848407866
:108C10000007C00F774909794907C90F88420DD06D
:108C20007448007904218843714949780907C90FBC
:108C300089000422114008436E4908716C4880780D
:108C40008007C10F6B484078C007C00F81420AD02F
:108C50006848407840084000654989788907C90F0D
:108C6000084364494870624880784007C00F6149F2
:108C7000097BC907C90F88420AD05E48007B4008BB
:108C800040005B4989784907C90F0843594908736F
:108C9000574880780007C00F5649097AC907C90F9D
:108CA00088420AD05348007A4008400050498978E9
:108CB0000907C90F08434F4908724D488078C0061C
:108CC000C00F4C490979C907C90F88420AD04948E1
:108CD00000794008400046498978C906C90F084311
:108CE00044490871424880788006C00F414909789C
:108CF000C907C90F88420AD03E48007840084000A2
:108D00003B4989788906C90F08433A4908703848B1
:108D100080784006C00F374909784906C90F884254
:108D20000DD034480078402188433149897849067C
:108D3000C90F89014022114008432E4908702C4870
:108D40008078C1092B4820304078C00981420FD07B
:108D500028482030407880218843254989780906B1
:108D6000C90FC901802211400843224920314870AF
:108D70001F48C078C107C90F1E48203040788006C0
:108D8000C00F81420DD01B482030407820218843FD
:108D90001749C9784901202211400843154920315B
:108DA00048701348C0788007C00F12490978C90677
:108DB000C90F88420DD00F480078102188430C4914
:108DC000C9788907C90F09011022114008430949D0
:108DD00008700748C0784007C00F0649097B0BE0C0
:108DE000B8020020C3020020BA020020C8020020FE
:108DF000C4020020405C00404907C90F88420DD0E2
:108E0000F248007B04218843F149C9784907C90F1A
:108E10008900042211400843EC490873EC48C078EB
:108E20000007C10FE9484078C00981420DD0E748EA
:108E3000407880218843E649C9780907C90FC901EC
:108E4000802211400843E14948700020E149087040
:108E5000E148008800287DD0DF480078C007C00FB7
:108E600000280DD0DC48008840084000DA4908801E
:108E70000020FDF745FDD94908780021FDF7F6FDF2
:108E8000D54800880221084000280CD0D24800882C
:108E90008843D14908800120FDF732FDCF49487849
:108EA0000121FDF7E3FDCC4800880421084000289B
:108EB0000CD0C94800888843C74908800220FDF7C4
:108EC0001FFDC64988780221FDF7D0FDC248008801
:108ED0000821084000280CD0BF4800888843BE49BC
:108EE00008800320FDF70CFDBC49C8780321FDF77D
:108EF000BDFDB94800881021084000280CD0B648B4
:108F000000888843B44908800420FDF7F9FCB34980
:108F100008790421FDF7AAFDAF4800882021084008
:108F200000280CD0AC4800888843AB490880052055
:108F3000FDF7E6FCA94948790521FDF797FDA6480C
:108F400000884021084000280ED0A34800888843AC
:108F5000A14900E046E008800620FDF7D1FC9F49CA
:108F600088790621FDF782FD9B4800888021084012
:108F700000280CD09848008888439749088007202B
:108F8000FDF7BEFC9549C8790721FDF76FFD9248B2
:108F90000088FF210131084000280CD08E4800884D
:108FA00088438D4908800820FDF7AAFC8B49087A80
:108FB0000821FDF75BFD884800880121490208402F
:108FC00000280CD084480088884383490880092001
:108FD000FDF796FC8149487A0921FDF747FD0020FD
:108FE0007D49088002207E49087007F031FB7D49E9
:108FF0000860E8E003207A490870E4E074480078EB
:10900000C107C90F714840788006C00F81427DD1E9
:109010006F4800788007C10F6C4840780007C00F88
:109020008142F4D16A4800784007C10F6748203078
:1090300080784007C00F8142E9D165480078000779
:10904000C10F624840784007C00F81425ED160483E
:109050000078C006C00F5D49097B8907C90F8842A7
:1090600054D15B4800788006C00F584909798907B8
:10907000C90F88424AD1564800784006C00F53496C
:10908000097A8907C90F884240D151480078C00940
:109090004E49097A4907C90F884237D14C48407870
:1090A0008007C00F494909788907C90F88422DD127
:1090B000474840784007C00F444909784907C90F1D
:1090C000884278D1424840780007C00F3F4909796B
:1090D0004907C90F88426ED13D4880788007C10F8B
:1090E0003A484078C007C00F814264D13848807840
:1090F0004007C00F3549097BC907C90F88425AD1BB
:10910000334880780007C00F304900E053E0097A07
:10911000C907C90F88424ED12D488078C006C00FBC
:109120002A490979C907C90F884244D1284880785B
:109130008006C00F25490978C907C90F88423AD16E
:10914000234880784006C00F204909784906C90F96
:10915000884230D11E488078C1091C4820304078B0
:10916000C009814227D11A48C078C107C90F1748E2
:10917000203040788006C00F81421CD11448C0784E
:109180008007C00F11490978C906C90F884212D15A
:109190000F48C0784007C00F0C49097B4907C90F29
:1091A000884208D10A48C0780007C10F07484078B4
:1091B000C009814202D001200649087000200849F8
:1091C000087000E000BF00BF10BD0000405C004020
:1091D000C4020020C3020020BA0200200B150020A8
:1091E000B8020020C80200207047000010B52848CF
:1091F000007801280FD12748007800280BD0264896
:109200000078F6F75FFB25490968884203D02148BA
:109210000078FDF7F1FF1E48007802280FD11D48A5
:10922000007800280BD01E480078F6F76BFB1D492C
:109230000968884203D017480078FEF7D5F814482B
:10924000007803280FD11348007800280BD0164867
:109250000078F6F7D7FB15490968884203D00D4816
:109260000078FEF76FFC0A48007804280FD10948FF
:10927000007800280BD00E480078F6F71BFC0D494B
:109280000968884203D003480078FEF70DFD10BD41
:1092900023040020240400202C040020300400209B
:1092A0002D040020340400202E0400203804002067
:1092B0002F0400203C0400207047000070B5049C7F
:1092C0008DB2002D05D0274D2D688EB23543254E29
:1092D000356095B2002D05D0224D6D6896B23543AC
:1092E000204E75609DB2002D05D01E4DAD689EB21A
:1092F00035431C4EB560A5B2002D05D0194DED6863
:10930000A6B23543174EF5600D0C2D04002D06D086
:10931000144D2D6A0E0C36033543124E3562150C72
:109320002D04002D06D00F4D6D6A160C3603354303
:109330000C4E75621D0C2D04002D06D0094DAD6A32
:109340001E0C36033543074EB562250C2D04002D47
:1093500006D0044DED6A260C36033543014EF56206
:1093600070BD0000405C004000210549002004E081
:1093700000220A60091D421CD0B21028F8DB704799
:10938000405C00402D49096807225202914302784F
:10939000520207235B021A401143284A116011460A
:1093A0000968DA10914342789201DB101A401143A8
:1093B000224A1160114609682022914382785201A5
:1093C00020231A4011431D4A1160114609681822D2
:1093D0009143C278D20018231A401143174A1160F2
:1093E00011460968062291430279520006231A4069
:1093F0001143124A1160114649689215914342790E
:109400001202FF2301331A4011430C4A51601146E6
:109410004968802291438279D20180231A40114306
:10942000064A51601146096849084900C279D207C5
:10943000D20F1143014A116070470000005C0040E8
:10944000024A0168D160416811617047005C0040C8
:1094500010B511F019FD03E0F3F780F8F3F7AEF95A
:1094600010F038FA0028F7D100F088F900210148FF
:10947000017210BD2E27002010B5064800F035F807
:10948000002805D0034800F013F8012002490870B5
:1094900010BD0000000F0040F602002010B50420AF
:1094A00007F026FC10BD10B5052007F021FC10BD0B
:1094B00010B50446002211462046143005F094FDF4
:1094C00010BD70B505460C462246002128460C30DA
:1094D00005F08AFD70BD70B505460C4622460A218E
:1094E00028460C3005F080FD70BD10B50446002103
:1094F00020461030F6F70CFB10BD30B502467D2338
:10950000DB00D0680724E402A0430C78E4020725BE
:10951000ED022C402043D060D0683024A0434C782A
:10952000240130252C402043D060D06801246402FF
:10953000A0438C78640201256D022C402043D0604A
:10954000D0686C10A043CC7824026D102C402043CE
:10955000D060D0680824A0430C79E40008252C4092
:109560002043D060D0680424A0434C79A400042593
:109570002C402043D060D0680224A0438C79640042
:1095800002252C402043D06005E0D0680006C00FC3
:10959000002800D004E018465C1EA3B20028F4D1D5
:1095A00000BF002B01D1092030BD5068000C000421
:1095B0000C89204350600020F6E700000348C06A91
:1095C000400840000149C862704700000024004084
:1095D00010B5FFF7F3FF10BD10B507F070F80028C5
:1095E0007ED0F1F74DFA0028FAD004F00FFC0028E5
:1095F000F6D003F01DF80028F2D0F3F771F8002838
:109600007ED0042007F068FC002879D0052007F000
:1096100063FC002874D0FCF76BFC002870D0FFF7C7
:10962000BFF800286CD0F9F745FD002868D0FCF79A
:1096300063FB002804D10F20F5F702FA01285FD15F
:10964000FCF760FC00285BD0F5F798FB002804D1FC
:109650000F20F5F7F5F9012852D1FFF7B7F80028E8
:109660004ED0FBF7DBF9002804D10F20F5F7E8F91D
:10967000012845D106F066FE002841D006F0A0FD85
:10968000002804D10F20F5F7DBF9012838D100F0CC
:109690008DFD002804D10F20F5F7D2F901282FD134
:1096A000F1F7A2FE002804D10F20F5F7C9F901282F
:1096B00026D10AF0E1F8002822D005F00FFB00289F
:1096C00004D10F20F5F7BCF9012819D1042007F0C7
:1096D000CFFE002814D0052007F0CAFE002800E0C5
:1096E0000EE00DD0042008F08BF9002808D00520EA
:1096F00008F086F9002803D0F2F71EFF002801D1F8
:10970000002010BD0120FCE710B502460023002018
:10971000002100BF0BE0074C0419237D002B04D06F
:10972000072902DA53544C1CE1B2441CE0B20A2867
:10973000F1DB10BD600E10001CB5072168460BF070
:1097400081FD01216846417081700021C170017165
:109750004171012181716A460B2101200003FBF751
:10976000E1FC03220B2101200003FBF7B1FC0122E5
:1097700003210220F3F7CAFA1CBD00000748006865
:1097800007490840884205D10448006880B203496F
:10979000086002E00020014908607047247F002033
:1097A00000005AA50248006880B20149086070476D
:1097B000247F00200548006805490840884203D1FD
:1097C0000248006880B270470020FCE7207F00203C
:1097D00000005AA507490968074A1140914202D082
:1097E0001146044A1160034909680143014A1160A6
:1097F00070470000207F002000005AA510B504F03B
:109800008DFA02210840022813D1012004F0AEFA9B
:10981000032004F057FC072004F054FC4A20F5F71D
:10982000BDFA01200349087003490870062004F0BE
:1098300049FC10BD3A0500203B05002070B50446E8
:1098400006F074FD0546204670BD0EB50C21684635
:109850000BF0F8FC002168460170082141700321DB
:10986000090341800121490281800021C180012139
:109870008903018100218172F1F770FA0EBD10B5E4
:1098800005210020FBF7A6FC00218020FBF7A2FCAD
:1098900002218020FBF79EFC03218020FBF79AFC2D
:1098A00010BD000010B55848FCF7CCFF57490870B0
:1098B00008460078F0F75EFF54480078F0F760FA49
:1098C00052480078EFF78CFC50480078F0F742FBE4
:1098D0004F48007A03000AF058FE3C1F2122235013
:1098E000464B8C412487258C8C2627288C8C8C29F0
:1098F0002A2B8C558C8C8C8C5A393134366E3782AD
:109900002C7838205F2D2E333573642F30698C8C82
:109910003A327D8C3B8C3C8C00BF00BF00BF00BF47
:1099200000BF00BF00BF00BF00BF00BF00BF00BF3F
:1099300000BF00BF00BF00BF00BF00BF00BF00BF2F
:1099400000BF00BF00BF00BF00BF00BF00BF00BF1F
:1099500000BF2E480078F0F765FE4BE02B480078FA
:10996000EFF7F0FB46E029480078EFF773FB41E0A2
:1099700026480078EFF7DCFA3CE024480078EFF75F
:109980009FFD37E021480078F0F7E4FB32E01F4804
:109990000078F0F729F82DE01C480078EFF712FE68
:1099A00028E01A480078EFF7C3FF23E01748007853
:1099B000F0F796FE1EE015480078F0F773F919E00D
:1099C00012480078F0F7B2FF14E010480078F0F782
:1099D0007DF80FE00D480078F0F706FB0AE00B4831
:1099E0000078F0F7F3F805E008480078F0F764FB3A
:1099F00000E000BF00BF054800780649087001215B
:109A0000044802F02BFF10BD004000406407002016
:109A1000332E00207334002030B503460C46154623
:109A2000002D10D115480360154804801548C07EEC
:109A3000012802D102F028FA01E0F2F753FB0020DE
:109A40001149087012E0012D07D110480360104839
:109A50000480012008F004FD08E0022D06D10D4825
:109A600003600D480480022008F0FAFCB0200B4986
:109A7000087002200A49087030BD0000A4050020CB
:109A8000A805002070290020BA050020AC050020A0
:109A9000B0050020B4050020B80500208E05002088
:109AA0008D05002010B5002204218802FBF7A0FBE1
:109AB00000200149087010BD9405002010B5012256
:109AC00004218802FBF794FB01200149087010BDB6
:109AD0009405002070B50546002D04D0012D05D059
:109AE000032D22D11EE01348C07970BD0026114815
:109AF0004A304078002803D00E484A3046780FE0BC
:109B000000240BE00B48801CEEF7E4FBE040C007AC
:109B1000C00F002801D0701CC6B2641C202CF1DBE1
:109B20003046E2E70448007ADFE700BF00BF0020CC
:109B3000DBE70000E4260020B644002070B50546AF
:109B40000C46002D04D0012D05D0032D16D112E0B6
:109B50000C48C47113E006F0C1FA0A49891C20467A
:109B6000EEF7D0FB002107484A3041700121052063
:109B700011F06EF903E00448047200E000BF00BF7A
:109B800070BD0000E4260020B644002010B5FFF7A9
:109B900089FF00200549487648778877C877B02044
:109BA0000349087000200349087010BD7029002087
:109BB0008E0500208D0500201CB5072168460BF09E
:109BC00041FB002168464170012181700021C17074
:109BD00001714171012181716A4604218802FBF7FC
:109BE000A1FA6A46002141208001FBF79BFA6A46F0
:109BF00002210020FBF796FA6A46012141208001EC
